:020000040800F2
:1000000000500020D58B0008818C0008357700084F
:10001000818C0008818C0008818C000800000000A1
:10002000000000000000000000000000818C0008BB
:10003000818C000800000000818C000825770008F2
:10004000818C0008818C0008818C0008818C00085C
:10005000818C0008818C0008818C0008818C00084C
:10006000818C0008818C0008818C0008818C00083C
:10007000818C0008818C00088D760008818C000836
:10008000818C0008818C0008818C0008818C00081C
:10009000818C0008818C0008818C0008818C00080C
:1000A000818C00089D750008818C0008AD750008E2
:1000B0008D7500087D7500086D750008D5760008FF
:1000C000CD760008D1760008C9760008818C00083A
:1000D000818C000849760008BD750008818C0008F5
:1000E000818C0008818C0008818C000800000000D1
:1000F0000000000000000000000000000000000000
:0C01000000000000000000005FF808F1A3
:100110002DE9F04F674B684C99B023600023636072
:1001200006F08EFE18B903F05DFD06F0ABFE03F09D
:1001300051F900230893614C09930A934FF4E0139B
:100140000B9323685E4943F480338A7B2360A36961
:10015000894643F01003A361236803F40033099335
:10016000089B01330893099B1BB9089BB3F5A06F4B
:10017000F2D12168514B11F4003101D0022315E076
:10018000186840F0010018600891236803F002032A
:100190000993089B01330893099B1BB9089BB3F58E
:1001A000A06FF2D12368980739D501230A93454BF4
:1001B000454E1968454F41F010011960196821F04A
:1001C00003011960196841F00201196063686360F6
:1001D00063686360636843F4806363603C4B1968E1
:1001E00021F0704119603B49B161616821F47C11D3
:1001F0006160196841F000411960FB6823F4004315
:10020000FB60BB68190449BF334B4FF4E013B36183
:100210004FF480130B930A9B012B01D117E0FEE7EB
:10022000022B18D16AB10B9BB3F5801F02D14FF49A
:10023000A01305E00B9BB3F5E01F02D14FF40013B0
:100240000B9362680B9B134343F4803302E06368B3
:1002500043F460136360236843F080732360226873
:10026000164B9201FBD55A6822F003025A605A6875
:1002700042F002025A606368104A03F00C03082B34
:100280000693F8D15168154B01F00C01042903D0F5
:10029000082904D00F4A00E0B2691A602AE05168C8
:1002A0005068C1F38341C50301F102011AD40C4A1D
:1002B0001EE000BFC1210008080500200010024018
:1002C000A410002000200240100000200010014077
:1002D0000410014000127A00001BB70080000020CB
:1002E00000093D00526812F4003FB26918BF52087D
:1002F000514319606268DFF848A3C2F30312324425
:1003000092F81CB01A6818AD22FA0BFBC3F800B0C3
:10031000BB4B4FF00008CAF80C30A369B94843F052
:100320000103A361636A43F080736362A36943F0CE
:100330001C03A3614FF6FF7325F82C3D29468DF869
:10034000368002F081FAB048294602F07DFA29464B
:10035000AE4802F079FAAE4B28465A6842F0007275
:100360005A6004F03DFF0D9BAA4AAB48B3FBF2F381
:100370004FF47A728360BBFBF2FBA84B0BF1FF32A8
:100380005A60F0228AF823200722C3F808806420EC
:100390001A6001F006FEA022A14841460AF0C5FD00
:1003A000E369424643F00703E361A36943F4006352
:1003B00043F00C03A361984B4FF0000803F10C01CC
:1003C00002F8018001320E2AF5D1FF229A76DA7600
:1003D0001A775A77934B4FF0100A0FCB85E80F002E
:1003E000A3690D9843F01003A361A3690EA943F01C
:1003F0001003A3614FF400533B614FF480433B6112
:1004000002F022FA10A90F9802F01EFA404606F0F8
:10041000FBFE854FD9F808B041460BF40063524605
:10042000384605930AF081FD042302223B70072120
:1004300001231BF4004F8DF832208DF83380ADF886
:1004400030A0BB70F97008D01220ADF830003B71BD
:100450007B71BB71F971904600E0984669480CA920
:1004600004F008FF059B93B1022367480CA9ADF87F
:10047000303004F0FFFE092301223B73BA7308F108
:100480000103072287F80D80FA735FFA83F8636926
:10049000664843F001036361A369DFF890A143F468
:1004A0000073A36101F058FA614B00240D93614B76
:1004B000B8F1010F0E930CBF2346802312934FF423
:1004C000807313934FF4806314932023294615936C
:1004D00050464FF4005316930F94CDF8408011947A
:1004E000179401F01BFADAF80030B8F1010F43F06D
:1004F0000103CAF80030504B98BF00215A6888BFEA
:10050000012122F4702222F4807242EA01225A6010
:1005100099684A4A20460A4042F4602242F00202A8
:100520009A60D96A08F1FF3221F47001D2B241EA2F
:100530000252DA62012339188A78002A5AD03A5CCA
:100540005C1C092A91F803E0E4B23B4911D9A2F1FD
:100550000A0505EB45054FF0070C0CFA05FC0EFAF1
:1005600005FED1F80C8028EA0C0C4CEA0E05CD6093
:100570000EE002EB42054FF0070C0CFA05FC0EFAF8
:1005800005FED1F8108028EA0C0C4CEA0E050D612E
:10059000062B29490ED8013B03EB83034FF01F0EB6
:1005A0000EFA03FE9A404D6B25EA0E0545EA02035A
:1005B0004B6320E00C2B0ED8073B03EB83034FF07B
:1005C0001F0E0EFA03FE9A400D6B25EA0E0545EA52
:1005D00002030B630FE00D3B03EB83034FF01F0E91
:1005E0000EFA03FE9A40CD6A25EA0E0545EA02039B
:1005F000CB6200E01C460430102823D023469AE743
:100600000005FA0500080140000C014000100140FF
:100610000000014040420F000805002010E000E00B
:10062000580F0020B0CB0008DC0300200800024077
:100630004C240140EC03002000240140FDF7F1FFB1
:1006400000ED00E0A84B9A6842F480729A609A68C4
:1006500042F001029A609A6842F008029A60996832
:10066000A14A0807FBD4936843F0040393609E4AB1
:10067000936813F00403FAD19168B9F8E60041F4E5
:10068000A0019160994A50B9B2F9E83033B9B2F992
:10069000EA30D3F1010338BF002300E0034613F032
:1006A000010340F0898086F82C3000B207F0FCFC92
:1006B0008F4907F04DFD8D4E0546B6F9E80007F06D
:1006C000F3FC8B4907F044FD0446B6F9EA0007F055
:1006D000EBFC874907F03CFD804628460AF054FEB3
:1006E000064628460AF0C4FE074620460AF04CFE9D
:1006F000054620460AF0BCFE044640460AF044FE89
:10070000814640460AF0B4FE31468046484607F02E
:100710001FFD31468346404607F01AFD49460590C5
:10072000384607F015FD41460790384607F010FDA2
:1007300029468246484607F00BFD6E49086241464D
:1007400005F1004007F004FD6A4A214650629462B8
:10075000079807F0FDFC0146059807F0F1FB654B93
:100760002146D862504607F0F3FC0146584607F090
:10077000E5FB60490863294607F1004007F0E8FC03
:100780005C4A21465063584607F0E2FC0146504659
:1007900007F0D4FB574B21469863059807F0D8FC27
:1007A0000146079807F0CCFB5249C86328463146FA
:1007B00007F0CEFC4F4A10644F4DDFF860912B6874
:1007C0004A4C43F00A032B60D9F800304B4E49489D
:1007D000B3F852B00023B4F8EE8094F8ED703370A3
:1007E000436405F025FD002800F00781444B454A8D
:1007F000B8F1BB0F1A60444A444E5A60444ADA606A
:1008000001D9012312E0B8F1610F01D902230DE0F3
:10081000B8F1290F01D9032308E0B8F1130F01D96A
:10082000042303E0B8F1090F07D9052386F82D301A
:100830002B6843F001032B600CE00623F6E70A2F38
:100840000ED097B1334B1B78002B40F08180002FE6
:100850007AD01F46304B0022022F1A70EFD104E0ED
:100860002B6823F002032B60ECE7DFF888804FF061
:1008700000094146C1F8449005F0DAFC0028E1D0B7
:1008800006210DAB68200A4606F0C6FD9DF83730FC
:100890009DF839C003F001035B000CF0010C43EA42
:1008A0008C0C9DF8353003F001035CEA030A09D093
:1008B000BAF1010F02D188F8489034E0BAF1020F82
:1008C0000BD12DE00CAB68200C21012206F0A4FD19
:1008D0009DF8303013F00F0301D105208EE0042B7A
:1008E0001ED188F848A01EE000240140A41000207A
:1008F00035FA8E3C080500200C0200204E02002034
:100900003802002055610008B95F0008100000207F
:1009100090C1793D5D170020B6020020340200200E
:10092000012388F84830B04BB04A1A60B04A5A6088
:10093000B04A92F84820002A14BF6E226F221A7221
:10094000AD4B02221A707DE72B6823F002032B6067
:100950002B680DF1600823F004032B60002308F8D6
:100960002C3D1E200A210122434606F055FD18B1F8
:100970009DF83430482B03D02B6823F008032B60FC
:1009800094F8E2300BB19D4A137094F8E3300BB148
:100990009B4A137094F8E4300BB19A4A13702B6899
:1009A000990702D5904B1B689847974B914F1B684E
:1009B00098472B6813F0080F1CD00FFA8BF34FF0F9
:1009C000640A93FBFAF94846049307F06DFB049B15
:1009D00083460AFB193000B207F066FB8B4907F02B
:1009E000B7FB0146584607F0ABFA894907F0B0FB60
:1009F000F86405E00023FB6402E0032001F01AFB29
:100A0000844B4FF480425A614FF400521A614FF008
:100A10000A0A9946D9F80C30192083F48043C9F8A2
:100A20000C30D9F80C300AF1FF3A83F40053C9F8BE
:100A30000C3001F0B6FA192001F0B3FA1AF0FF0AEF
:100A4000DFF8D0B1E6D14FF40053CBF810304FF4BB
:100A50008043CBF81030704BDFF8E8A11B6893F9A6
:100A60000C0007F021FB6D4907F072FB0AF08CFCCB
:100A70008346BAF8000007F017FB594607F068FBF9
:100A80000AF0B8FC664B1880BAF8000007F00CFBBF
:100A90000146644807F010FC634907F00DFC5A4B0F
:100AA00038655E49D86807F053FB604907F050FB92
:100AB0005F4B627918605F4B5F491A705F4B01EBC7
:100AC000C202527C7B655E4B1A60A268920644BFEC
:100AD00001221A602B681B0740F1FF804FF480430E
:100AE000C9F81430322001F05CFA002111221E20D6
:100AF00005F0E4FA012160221E2005F0DFFA6420EF
:100B000001F04FFA4FF0000A404605F057FBD3467C
:100B10004FF00A0C5346022101221E200493CDF807
:100B20000CC005F0CBFA322001F03BFA404605F04C
:100B300045FBBDF93410BDF93600049BBDF93820E2
:100B40000B448842B8BF014692449142B8BF0A465E
:100B500012F5805F8344DDF80CC00BDDD9F80C2062
:100B6000BCF1010C82F48042C9F80C20D3D10121E0
:100B7000059101E0002005901E200021122204931F
:100B800005F09CFA049B4FF00A0C022101221E2062
:100B90000493CDF80CC005F091FA322001F001FA6F
:100BA000404605F00BFBBDF93410BDF93600049B3F
:100BB000BDF938205B1A8842B8BF0146C2EB0A0A69
:100BC0009142B8BF0A4612F5805FC0EB0B0BDDF80F
:100BD0000CC039DDD9F80C20BCF1010C82F4804244
:100BE000C9F80C20D1D131E0A4020020C14900088D
:100BF000795F0008080500205D1700204E020020E4
:100C0000B60200205A170020380200208988883C4C
:100C10000000204100100140F002002035FA8E3C17
:100C2000140300200AE81C4100401C46BD378635ED
:100C3000EC02002000050020B0CB0008B41000201A
:100C4000FC0400200000002000220592DFF8CCC147
:100C50001846CDF80CC007F027FA0146674807F0A0
:100C60002BFB20F000403063584607F01DFA014688
:100C7000624807F021FB20F000407063504607F007
:100C800013FA01465E4807F017FB20F00040B063FE
:100C9000002170221E2005F011FA012120221E20C1
:100CA00005F00CFA022100221E2005F007FA64204C
:100CB00001F077F9059BDDF80CC03BB94FF07E538E
:100CC000CCF83030CCF83430CCF838304FF48043A6
:100CD000C9F810304B4B01221A704B4E4B4BB346A8
:100CE000336004F0C1F83068494B0590FF21184685
:100CF00016220AF01AF9002202702A68DFF814E1BD
:100D0000012112F0020F8EF80010734604D04170DA
:100D10000321197002218170550704D519784D1CE3
:100D20001D700325455412F00A0F0CD01A780421C7
:100D30008154511CC9B205254554D11C0232197089
:100D4000D2B206218154A268910604D519784D1CAF
:100D50001D70072545546179082901D00E2904D159
:100D600019784D1C1D700B25455419784D1CEDB29A
:100D70001D700C234354530705D5264B02311970BF
:100D8000234B10215955234B12261978465494F8B9
:100D900041614D1CEDB2002E0CBF002602F0010691
:100DA0001D7026B102311970194913264E5596054A
:100DB00004D51A78511C1970152383541648002144
:100DC00098220AF0B2F8144D05F1980A95F84A30C5
:100DD000002B30D1059999464A68002603230096D6
:100DE0000120314605F008F90346C8B9B9F1000FF2
:100DF00024D14FF496424FF00109EEE700406F46D0
:100E000001C05E462C020020B8040020CC11002056
:100E1000BF040020BE0400201804002010000020A1
:100E2000284631464C2204930AF07FF8049B2B603D
:100E3000012385F84A304C355545C7D1BB4BDBF80B
:100E40000020197A02290AD0187D022806D08D07C1
:100E500005D400F0020000F0FF0108B10C3359681E
:100E6000B34DA96531B9009102209268032305F0C2
:100E7000C3F8A8654046002114220AF056F86379A9
:100E80000E2B01D0082B02D101238DF83F30A3682F
:100E9000A848C3F38041C3F340028DF83A10A64935
:100EA0008DF83920C3F380128DF83B200968C3F315
:100EB00040328DF83420C3F3C03200318DF8362033
:100EC000C3F3C02218BF01218DF83720C3F30042BD
:100ED0008DF83C208DF83D1003F0010201688DF87B
:100EE000352091F8B011B4F8E000C1F380018DF81D
:100EF0003E10ADF84200B4F8DE104FF47A70ADF851
:100F00004400D804ADF8401004D58C4BB3F8DA3067
:100F1000ADF84430B1F5FA7F84BF0023ADF844301A
:100F2000B4F81A318649ADF8463094F8223185F884
:100F30005C30002385F85D304B709DF83F30002B0E
:100F400014BF0223002302B101337E4A4FF0000890
:100F500002EB8303D3F8C830C1460593059931F8F5
:100F600008304FF6FF718B42DAB20AD195F85D3046
:100F700085F85F30744B1F78162F40F039810024BC
:100F800028E19DF8381019B1911E012940F20D8118
:100F90009DF8361011B1012A00F007811B0A022BBF
:100FA00002D19DF8341003E0012B04D19DF83510D7
:100FB000002900F0FA80654C9DF83E104FEA021AB5
:100FC000544431B19DF83F1019B9043A032A40F254
:100FD000D580012B39D1FF2387F8A43087F8A530BD
:100FE000A3680026E27B6068ADF830300CA90223CC
:100FF00087F8A860C7F8B4408DF833308DF83220F8
:1010000087F860607E66BE66FE66C7F8A06087F8F7
:10101000A66087F8A76001F017FC4C4A217B52F8C4
:101020000A00324603F0B0FF204604F0A3FC484B10
:101030004849C7F8B830484BC7F8C060C7F8BC305B
:1010400020460A1D04F060FDAFE0022B36D15FFAA6
:1010500089F21C20424341494FF0000B8E180120B9
:1010600086F8019086F802B086F80AB08854A16824
:10107000E27B6068ADF83010F4600CA98DF8322086
:101080008DF8333001F0E0FB304B217B53F80A0040
:101090005A4603F079FF204604F06CFC304BC6F84A
:1010A00018B033612F4B2046736106F1100106F131
:1010B000140204F029FD09F1010976E0032B5BD14C
:1010C0009DF83A20BDF8443032B195F85E60204674
:1010D00008214FF6FF721AE0BDF8402095F85E60D7
:1010E000B2F5FA7F0DD920492046B1FBF2F292B257
:1010F000082103F0F5FC05EB8606C6F888011B4BBA
:101100000CE01B492046B1FBF2F292B2012103F040
:10111000E7FC05EB8606174BC6F88801C36095F817
:101120005E30013385F85E303FE000BF10000020E4
:101130000805002034020020FC040020A410002038
:1011400065050020B0CB00080005002074DE000813
:10115000B9170008C005002095180008B005002048
:10116000855100088D17000800127A00B518000894
:1011700040420F00A5180008042B16D1BDF84230DC
:10118000874A204692FBF3F20121BDF8463092B225
:1011900097F85D6003F0A4FC97F85D3007EB8606D6
:1011A0000133C6F8B80187F85D3008F10208B8F1DC
:1011B0001C0F7FF4D3AED9E67A4E98E80F00264490
:1011C00086E80F00784B10341A78C02C02F1010227
:1011D0001A7008D06B6D0021185903EB040807F052
:1011E0004BF90028E8D0714EB368D9041DD418E03B
:1011F0006F486D4A00EBC70393F810E0D3F814C0B2
:1012000082F800E0BCF1000FEDD000247445EADA6A
:10121000644E23011E4463440FCB013486E80F0063
:10122000F4E7082F634C28D129E05F4B93F8009036
:10123000B9F1010FF5D9604C4FF00008C84504F131
:101240001004EEDA54F8100C4FF07C5106F080FFD9
:101250004FF07C5144F8100C54F8140C06F078FF51
:101260004FF07C5144F8140C54F80C0C06F070FF4D
:1012700008F1010844F80C0CE0E70E2F03D12378A5
:1012800043F0100302E0237823F01003237005F0ED
:1012900035FF4A4A4A484B494B4B02604B48C5F818
:1012A0009C3201600023B6F81A01C5F89812A5F81F
:1012B000A23285F8A432C5F8A82245495852023313
:1012C000242BFAD1434B1A60B3681A0740F1B4805B
:1012D000364B002293F81831042B00F2A780DFE888
:1012E00003F003032A4F9100012B4FF003013A4A08
:1012F00008D185F8AC12072185F8AE3285F8AD1219
:101300000C2308E0022385F8AC32002385F8AE32C6
:1013100085F8AD12072313700023009310200123DA
:101320002E494FF4E13204F067FE2D4BC5F8B002B0
:10133000C5F8B43276E001232A4A2B4900931020E5
:10134000052304F059FEC5F8B8020746B6F81A019D
:1013500006F0AAFE254906F0FBFE254906F0EEFD43
:1013600007F0E2F80023234A98500433402BFAD1C7
:10137000214B1022C5F8B432174B381C1A7052E0BA
:10138000009201234FF4E13210201C4904F034FE96
:101390001B4BC5F8BC02C5F8B432102240E000BFB8
:1013A00040420F00E006002034170020A410002067
:1013B000B0CB00081A020020E8060020A407002095
:1013C0000C040020B411002088CC0008FC00002090
:1013D0006203002000020020D5040020251E000822
:1013E00029150008A0860100311F0008CDCCCC3F94
:1013F0000000B0441C010020DD150008BD1E0008DF
:10140000CD150008009201234FF4E1321020384935
:1014100004F0F2FD374BC5F8C002C5F8B43208221B
:10142000354B1A70003018BF012028B9082001F090
:1014300088F90023C5F8B432B2682F4B12F4804FFC
:1014400004D0082119702D49C5F8B41242F20101E7
:10145000114002F0010002F4005741B1284AC5F8DA
:10146000B4220FB108221A7008B10C221A701A782F
:10147000043A5A7000F0BCFC224B18607379052BBB
:1014800003D1214B4FF4C8721A80204B4FF47A726B
:101490001A80237843F0080323701D4B1A7822F03A
:1014A00002021A70B3689B071ED51A4B1A4A1C46D3
:1014B0001A6000F081FB282000F073FD069A013AC3
:1014C0000692F6D12168154B48781D780246012313
:1014D000954203D30133082B0244F9D1104A13700B
:1014E0008A7853430F4A138019B0BDE8F08F00BFCC
:1014F000711E0008B9150008D5040020091600085F
:10150000151600085C030020B802002058170020C0
:101510005C170020D0030020A8110020CD0300207C
:101520007C000020CE0300201E4B2DE9F0431A78EA
:101530001D460AB31C4B07781E781C4B93F800C05D
:1015400002231B4A03F10108D45C344104F00F0468
:10155000BC420CD20B2C0AD812F8039012F8088067
:1015600002EB840209EA0C0408EB04241461023340
:10157000102BE6D100232B7003788B420FD90C4B34
:1015800093F8400060B10B4A890012780B44186947
:1015900002B1400800F5777080B2BDE8F08300200A
:1015A000BDE8F08300010020B4070020B50700204B
:1015B000CC070020B607002007299ABF024B33F85A
:1015C00021000020704700BFDC010020024B53F8CF
:1015D0002100C0F3CF0070478401002008B5074BFD
:1015E00053F8210006F05CFD054906F0B1FD054900
:1015F00006F0A6FC06F098FF80B208BD1C01002092
:101600000000203F00005C44014B33F8110070479C
:1016100062030020014B33F811007047880A002054
:10162000032810B5114B0FD8114A126894888C42C8
:101630000AD2D2888A4207D9012202FA00F093F82E
:101640004120104383F8410093F841300F2B0CD117
:10165000064B002283F84120064B998808B21428D3
:1016600002DD1439998010BD9A8010BDCC0700208E
:10167000CC080020A4070020024B9A8801329A80EF
:10168000704700BFA4070020074B1A68074B11786A
:10169000B3F9040053780B4403EB83039842D4BF9F
:1016A00000200120704700BFCC080020A4070020C4
:1016B000064BB3F90400064B1B681B7803EB83034E
:1016C0009842D4BF00200120704700BFA40700202B
:1016D000CC08002010B50446FFF7EAFF002814BF2D
:1016E0002046002000F0010010BD024B01221A72BA
:1016F000704700BFA4070020014B187A704700BF55
:10170000A4070020034BB3F90400D0F1010038BF57
:1017100000207047A4070020014B00229A807047E8
:10172000A4070020016B0346C26810B5406941B1AF
:10173000196C541A005D013918BF0A46C0B21A6408
:1017400010BD196A405C0131914228BF0021C0B22E
:10175000196210BD036B13B15A68036C01E0C269D2
:10176000036A9A4237BFC068C3EB02008018C3EB1C
:101770000000C0B27047436B13B190F8440070474B
:10178000826A436AD31A58425841704710F80A3C9B
:101790000133DBB20A2B00F80A3C0AD910F8123CDC
:1017A00023B910F8131C034A22F81130002300F863
:1017B0000A3C7047880A0020334A10B5136C9068C1
:1017C0001944081A40F68C2398429160D060516009
:1017D00013463CD9127893F945108A420BD1111F58
:1017E000082908D893F84610182901D8013103E0D8
:1017F00083F8442002E0002183F8461093F9441056
:101800008A421CD1204991F84710C1B10021914270
:101810001E4806DA03EB8104246920F811400131E7
:10182000F5E7511E00EB41011630814203D0002440
:1018300021F8024FF9E7164908780130087083F85B
:101840004520002201211A7083F8471010BD92F83C
:101850004710B9B1A0F2EF2440F2DA518C4208D817
:1018600011780B2905D80B1D0131117042F82300A6
:1018700010BD002283F84720991804320020302A36
:101880000861F9D110BD00BF68050020880A00205A
:10189000D80E0020024B1A6C0132114419647047B3
:1018A00068050020024B53F820301B6819807047F0
:1018B00090060020074BA1F57A7153F820304FF4C1
:1018C0007A701A681B894B4393FBF0F39BB2138029
:1018D000704700BF9006002038B50C6805462046CA
:1018E00009F064FB214602462868BDE8384009F04B
:1018F00065BB094BDA68D10709D4DA68520708D406
:10190000DB6813F0100F0CBF042003207047012088
:1019100070470220704700BF002002408A6810B55F
:101920000C6A036814430A6923F4FF4314434A69A9
:1019300023F0700314438A691443CA6914434A6A42
:1019400014438A6A224313430360CB6843600B68E5
:1019500083604B68C36010BD02684FF6FE7313408E
:1019600003600023036043608360C3602A4B984296
:1019700022D02A4B984229D0294B984230D0294B6B
:10198000984237D0284B98423ED0284B984206D1F7
:1019900053F8682C42F4700243F8682C7047244BCB
:1019A000984206D153F87C2C42F0706243F87C2CAC
:1019B0007047204B984206D153F8042C42F00F0296
:1019C00043F8042C70471C4B984206D153F8182C4E
:1019D00042F0F00243F8182C7047184B984206D199
:1019E00053F82C2C42F4706243F82C2C7047144BA3
:1019F000984206D153F8402C42F4704243F8402CF0
:101A00007047104B984205D153F8542C42F4702281
:101A100043F8542C704700BF080002401C000240ED
:101A20003000024044000240580002406C00024076
:101A300080000240080402401C04024030040240BE
:101A400044040240580402402DE9F843574B0C4629
:101A50000168013AC3F842108188A3F84610072AAA
:101A600042D8DFE802F0040A101822292F35B3F813
:101A700042202280B3F8442013E0B3F844202280AF
:101A8000B3F8422005E0B3F8422052422280B3F876
:101A90004420524205E0B3F8442052422280B3F879
:101AA00042206280B3F846301DE0B3F84220524233
:101AB0002280B3F8442012E0B3F844202280B3F827
:101AC00042200CE0B3F842202280B3F8442005E025
:101AD000B3F8442052422280B3F84220524262803E
:101AE000B3F846305B42A380314B1B78002B5AD1B0
:101AF000B4F9000006F0D8FA8046B4F9020006F006
:101B0000D3FA0746B4F9040006F0CEFA294D06468A
:101B10002968404606F01CFBE9688146384606F015
:101B200017FB0146484606F00BFAA9698146304684
:101B300006F00EFB0146484606F002FA09F05AFC90
:101B400069682080404606F003FB296981463846D3
:101B500006F0FEFA0146484606F0F2F9E9698146C8
:101B6000304606F0F5FA0146484606F0E9F909F074
:101B700041FCA9686080404606F0EAFA696980463F
:101B8000384606F0E5FA0146404606F0D9F9296ADA
:101B90000746304606F0DCFA0146384606F0D0F932
:101BA00009F028FCA080BDE8F88300BFCC07002026
:101BB0003C0000202805002010B5194B93F8482060
:101BC000511C83F84810174902F00702487816495B
:101BD00003EB420331F81010A3F84A100023184613
:101BE000124A9A5A02331044102B80B2F8D1C0081E
:101BF00006F05AFA0E4906F0ABFA0E4906F05CFB05
:101C00000D4B04461B68187806F04EFA0146204634
:101C100006F09EFA06F088FC084B187010BD00BF55
:101C2000CC070020DC030020EC0300201608002075
:101C30003333534000F07F45D0030020CD03002014
:101C4000034B1B68DA79511CD9711344187A704719
:101C5000B004002010B5FFF7F3FF0446FFF7F0FFD4
:101C600004EB002080B210BDF0B5137C012B29D805
:101C70000C255D43144C013305EB040C9CF8086003
:101C800030421DD02D5D1DB1012D14BF022501254F
:101C90000E4C4E7B04EB0514277B3740B7420FD127
:101CA0004F686668B7420BD38F68A668B74207D8FB
:101CB00015709460C2F804C0D16013741046F0BD72
:101CC000DBB2D3E70020F0BD1000002048D10008AF
:101CD0002DE9F0478278C6781E4BC2F1640802EB0A
:101CE000820C54425FFA88F84FEA4C0CC6F1640942
:101CF000A4B203F11807A5B228B2002804DC002D15
:101D000014BF1546012500E0454600FB00FA6D436F
:101D10000AFB06FA9AFBF5F54D4468434FF00A0AB0
:101D200090FBFAF0604480B258800D88B1F802A0B0
:101D300000B2C5EB0A0A00FB0AF04FF47A7A90FB76
:101D4000FAF0054423F8025F0A34BB42A4B2D2D1B0
:101D5000BDE8F087AA03002010B54478007800237E
:101D600003FB03F11939614301F6C411594341439F
:101D700040F6C41291FBF2F1034A22F8131001332A
:101D8000072BEDD110BD00BF8C03002010B5044C13
:101D90002068FFF7E1FF20680249BDE8104097E79F
:101DA0008803002074110020104B043033F91030E8
:101DB000B3F5617F05DB40F633029342A8BF1346BB
:101DC00001E04FF4617308781922504300F2833028
:101DD000984208DA4878504300F283309842B4BF02
:101DE0000020012070470020704700BF62030020E0
:101DF00010B5094A094913688C6812689342F8D1F2
:101E0000074A106811684FF47A725043001BB0FB08
:101E1000F1F002FB030010BDA010002010E000E074
:101E20001005002038B5104C0123054684F84030D9
:101E3000FFF7DEFFE36D41F28832C31A9342236657
:101E400084BF002384F8643094F86430EDB20F2B23
:101E5000E065E55403D1054B01221A7038BD024AF2
:101E6000013382F8643038BDCC0700200001002027
:101E700010B50446FFF7BCFF0D4B41F288319A6E56
:101E80009866821A8A42DA6684BF002283F870203C
:101E900093F87030074A142BD45403D1064B012217
:101EA0001A7010BD024A013382F8703010BD00BFB5
:101EB000CC070020C5010020C401002010B5044655
:101EC000FFF796FF164A536F5067C31AB3F57A6F40
:101ED00084BF002382F8783092F8783023B9A82C98
:101EE0001CD110490B7006E0022B02D10E490C7078
:101EF00001E0242B01D80D49CC540133DBB282F828
:101F00007830094A127852000532934206D1044BC8
:101F1000002283F87820034B01221A7010BD00BF05
:101F2000CC0700205C010020820100205D01002020
:101F300038B50446FFF75CFF114B40F6C411DA6F69
:101F4000D867821A8A4284BF002283F8802093F8DF
:101F500080200AB90F2C11D10A480021017052B11A
:101F6000094D182A154405F8014C04D1012283F8C3
:101F70008010027038BD013283F8802038BD00BF68
:101F8000CC070020010100200201002038B50446E2
:101F9000FFF72EFF0546FFF72BFF401BA042FAD3A9
:101FA00038BD10B504462CB14FF47A70FFF7EEFF40
:101FB000013CF8E710BD2DE9F04106460F4690467A
:101FC0000025EBB2434512D20024E3B2B34209D25A
:101FD000084B3846DA68013482F40052DA60FFF7C1
:101FE000E0FFF2E73C20FFF7DCFF0135E9E7BDE861
:101FF000F08100BF001001400B490B7813F0010F76
:1020000003F004020AD072B9980707D443F004031E
:102010000B70064B1A88064B1A8070471AB90220BB
:10202000FF210122C7E770475C1700203003002022
:10203000C603002040F2DB1568430C4C08B54FF492
:10204000804363614FF400532361851EE368284693
:1020500083F48043E360E36883F40053E360FFF7B5
:10206000A0FF1920FFF79DFFF0E700BF001001401F
:1020700008B503681B68984708BD064B10B50446B1
:1020800021461868FFF7F4FF034B1B689A79544008
:102090009C7110BDB4040020B004002038B5044683
:1020A00024200D46FFF7E9FF4D20FFF7E6FF002C47
:1020B000084C0CBF3E202120FFF7DFFF23680022E1
:1020C00028469A71FFF7D9FF236893F84900BDE8C5
:1020D0003840D2E7B004002001460020DEE7F8B522
:1020E0000E4E0F4C0F4DC1B20746306884F8811078
:1020F000FFF7BEFF2B6894F881109A7930684A4048
:102100009A71C7F3072184F88110FFF7B1FF2B689C
:1021100094F881109A794A409A71F8BDB40400206D
:10212000CC070020B0040020F8B51B4D1B4C1C4F01
:102130000646C1B2286884F88210FFF799FF3B6811
:1021400094F882109A7928684A409A71C6F3072158
:1021500084F88210FFF78CFF3B6894F882109A791C
:1021600028684A409A71C6F3074184F88210FFF745
:102170007FFF3B6894F882109A7928684A409A71E8
:10218000310E84F88210FFF773FF3B6894F88210D9
:102190009A794A409A71F8BDB4040020CC07002017
:1021A000B004002010B5441E14F8011F21B1034BE8
:1021B0001868FFF75DFFF7E710BD00BF600500205E
:1021C000014B186854E700BF08090020054B1B6845
:1021D00003EBC00090F9063019420CBF01204FF00C
:1021E000FF307047D00800200A4B1A6802EBC0028B
:1021F000D379FF2B07D008490978994203D9074AB8
:1022000032F8130004E00728D4BF908840F2DC5075
:1022100000B27047D0080020D504002062030020DF
:102220002DE9F04F0C68836889B0D0F800A0D0F891
:1022300004800646204603938B4609F0A5F807461E
:10224000204609F015F9DBF804408146204609F0E4
:102250009BF80546204609F00BF9DBF808200446F8
:102260001046019209F090F8019A8346104609F051
:10227000FFF839460290584605F06AFF3946049047
:10228000029805F065FF59460590484605F060FF45
:1022900002990690484605F05BFF2946079058468C
:1022A00005F056FF0146504605F052FF2146834691
:1022B000069805F04DFF0146059805F041FE0146E0
:1022C000404605F045FF0146584605F039FE2146D7
:1022D0008346049805F03CFF0146079805F02EFE62
:1022E0000146039805F034FF0146584605F028FEE4
:1022F0003060029905F1004005F02AFF0146504682
:1023000005F026FF21468346079805F021FF014688
:10231000049805F013FE0146404605F019FF0146FA
:10232000584605F00DFE21468346059805F010FF3E
:102330000146069805F004FE0146039805F008FFE3
:102340000146584605F0FCFD21467060504605F0F8
:10235000FFFE2946044609F1004005F0F9FE01465A
:10236000404605F0F5FE0146204605F0E9FD3946F8
:102370000446284605F0ECFE0146039805F0E8FE09
:102380000146204605F0DCFDB06009B0BDE8F08FE5
:102390002DE9F84F2E4E04463768384608F0F4FF12
:1023A0000546384609F064F876688046304608F0FD
:1023B000EBFF8346304609F05BF8D4F804900646FC
:1023C0002946484605F0C4FEA7688246414638467D
:1023D00005F0BEFE0146504605F0B0FD216882467C
:1023E000584605F0B5FE41460446484605F0B0FEA5
:1023F000314605F0ADFE0146204605F0A1FD31460F
:102400000446384605F0A4FE294605F0A1FE014623
:10241000204605F095FD0146504609F0B7F80D49F4
:1024200005F096FE0C4905F047FF0C4B196805F0C6
:1024300087FD0B4905F040FF08F0DCFF83B21A046A
:1024400044BF00F5B4739BB218B2BDE8F88F00BF6B
:10245000180300200000E144DB0F49405405002030
:1024600000002041034B1A78510744BF22F00402B8
:102470001A7070475C17002070B5FFF719F938B370
:10248000144C237A0BB9A38070BD134D2E78C6F37C
:102490008000FFF71FF990B1104B46F002061A6852
:1024A0000F4B51892E7019805189598052899A8019
:1024B0000C4A12685288DA80E3880133E380FFF720
:1024C000E3F810B92B785B0702D4BDE87040C9E788
:1024D00070BD00BFA40700205C170020A0070020EB
:1024E00062030020CC0800202DE9F0410278034669
:1024F000202A00F10100F9D0092AF7D02D2A02D1B3
:102500000346414D04E02B2A08BF03464FF07E5599
:102510001E460024334616F8012BA2F13007F9B20B
:1025200009290DD83949204605F012FE04463846DF
:1025300005F0BAFD0146204605F002FD0446E9E734
:102540002E2A17D1314F334616F8010B3038C2B25C
:10255000092A0FD805F0A8FD394605F0ADFE014661
:10256000204605F0EDFC29490446384605F0F0FD0B
:102570000746E8E71A7802F0DF02452A38D15A7890
:102580002D2A02D10233012604E02B2A14BF013385
:1025900002330026013B002713F8012F303AD1B255
:1025A000092903D80A2101FB0727F5E7B7F59A7F28
:1025B00028BF4FF49A77B8464FF07E51B8F1070F15
:1025C00007D90846124905F0C3FDA8F108080146DD
:1025D000F4E707F0070737B108460C4905F0B8FDE6
:1025E000013F0146F7E72EB1204605F065FE04E005
:1025F0004FF07E51204605F0ABFD0146284605F020
:10260000A7FDBDE8F08100BF000080BF00002041B1
:1026100020BCBE4CF0B50124B0FBF4F58D4201D3D3
:102620004C43F9E70026DCB1B0FBF4F504FB1500E0
:10263000B4FBF1F41EB9002D01DC002CF3D1092DFF
:1026400003F101075FFA85FC04DD002A0CBF572562
:10265000372500E0302565441D7001363B46E2E732
:102660001C70F0BDF0B50124B0FBF4F58D4201D330
:102670004C43F9E70026DCB1B0FBF4F504FB150090
:10268000B4FBF1F41EB9002D01DC002CF3D1092DAF
:1026900003F101075FFA85FC04DD002A0CBF572512
:1026A000372500E0302565441D7001363B46E2E7E2
:1026B0001C70F0BD70B50646B6FBF2F40846154630
:1026C00014B12046FFF7F6FF05FB1464024B1B5DB7
:1026D00000F8013B70BD00BF54DF00082DE9F04158
:1026E000069C002B06460F460CBF4FF020084FF00B
:1026F0003008234613F8011B09B9154603E0002AE8
:10270000FBDD013AF6E7002D04DD30464146B847CF
:10271000013DF8E714F8011B11B13046B847F9E75D
:10272000BDE8F08180EAE073A3EBE0738B4206DB47
:10273000002801DD401A704702D00844704700208D
:102740007047034B9A6822EA00009860704700BF08
:10275000A41000202DE9F041038A87890446BFB206
:102760000D461F40002F36D0B7FA87F34FF00042D6
:10277000DA40D24391B21B3B21821740042BF1D89F
:10278000DFE803F0221F1C1903006B6A33B103F169
:10279000FF3800231FFA88F86B6203E0B4F82C803E
:1027A0001FFA88F82E6A002EDCD033683046414686
:1027B00098477668F7E72868A18E08E06868218F57
:1027C00005E0A868A18F02E0E868B4F8401003684B
:1027D00089B29847C6E7BDE8F0810C4B800A984261
:1027E0000CD003D8B0F5801F0ED00BE0084B9842F8
:1027F00006D04933984205D1002070470220704727
:1028000003207047FE207047012070470100100030
:1028100002001000044B53F820301BB107289CBF66
:102820001B681980704700BFC006002010B5054C1A
:1028300000202188FFF7EEFF61880120BDE81040ED
:10284000E8E700BF620000202DE9F0410F88002377
:1028500047FA03F2D2072BD58A7803F0070512F066
:10286000100F18BF91F803C002F00F0618BF46EA18
:102870000C06AD004FF00F0C0CFA05FC06FA05F53E
:10288000DC0850F82480282A28EA0C0C45EA0C05BC
:1028900040F8245005D101229A40C46824EA02027B
:1028A00005E0482A04D101229A40C4682243C2604C
:1028B0000133102BCCD1BDE8F08100BF08B504F086
:1028C000E1FA00F087FDBDE808400F201421012245
:1028D000FFF771BBA04A2DE9F04F13689F4903F53C
:1028E0009C439F4D20330B60AB6885B013F4807F11
:1028F000174604D09B4B1B681B681B699847AB6845
:1029000042F201041C405CB9974E337873B1954B89
:102910001B681B681B68984704F060FB347005E077
:10292000924B1A7801321A7004F058FBAB68DA0443
:1029300005D58F4B1B68DB0701D4FFF793FD8D4B4B
:102940003C681868037C83B18B4A013B32F9130061
:10295000A0F57A70B0F57A7FA8BF4FF47A7020EABC
:10296000E07005F0A1FB85492FE0AA68170435D572
:102970007E4A5168611A002930DB04F59C41203100
:1029800051607F494E797F4931F81660417CB6B27B
:1029900096FBF1F0117A013101F00F0111720A4436
:1029A00050721846784A9A5C01331044102B80B25A
:1029B000F8D100B290FBF3F000B26428A8BF642005
:1029C00020EAE07005F070FB704905F075FC704975
:1029D00005F0BEFB05F0A8FD6E4B1880AB68DE0568
:1029E00010D56D4B9C426D4C08D923681B681B6A3F
:1029F000984718B923681B685B6A984723681B6867
:102A00005B699847AA68564BD404B5F8DC100AD520
:102A10005948B3F81A31B0F90620581A82420ADD33
:102A200019448A4205E05449B3F81C31B1F9062033
:102A30009A42C0F2C1830122002395F823A195F8A0
:102A40002411B5F81C41B5F81E619B464A4F4FEA68
:102A50009B0BF85E0233A042C4BF6BF07F0B5FFAA2
:102A60008BFBB042B8BF4BF0400B082BEED13F4C74
:102A7000637E5B4504D1A37EF92B03D8013300E0CC
:102A80000023A376464B84F819B093F80080384FA2
:102A90009946B8F1000F14D13B68D80707D582B921
:102AA000404B1B78DB070CD5FFF7A6FA09E03D4B3E
:102AB0001B785E0705D511B1FFF7D4FC01E0002AB1
:102AC000FAD0A37E2949142B374E40F0A280354B13
:102AD0001AF1000A1B7818BF4FF0010A03F0040333
:102AE00003F0FF0293B1B8F1000F00F09280BBF148
:102AF0005F0F02D1FFF7B6FC8BE0BAF1000F00F0D8
:102B00008880BBF17D0F40F08480F3E7BBF1570F65
:102B10000BD1264B4FF47A721A80254B1B6813F0A9
:102B2000080376D1234A138073E0AB68580749D570
:102B3000BBF15A0F46D1204B187818B11A700122F8
:102B40001E4B54E0CA7E1E4B82F00102CA760AB1C7
:102B500004224CE006224AE0501700200402002024
:102B6000A410002000020020F800002050080020DF
:102B700004040020FC0000206203002000007A44CE
:102B8000DC030020EC030020590800200000C842AC
:102B900000C07F44D8040020404B4C00B007002008
:102BA0004C0000205C170020340200205817002041
:102BB0000C02002030030020E5020020E702002084
:102BC000E6020020BBF15D0F00F09C82BBF15B0FC1
:102BD00000F09A82BBF15E0F0BD1032295E2BBF1AC
:102BE000A70F40F0B282AE4B1A7842F004021A707E
:102BF0000FE0BBF1560F01D1FFF760FE99F80030EE
:102C0000002B00F09982BBF16F0F40F08E82FFF72E
:102C1000F3F9AB685B0732D5E37EA3B1A14B1B7818
:102C2000580710D5A048A14BB0F90620B3F81C31C5
:102C30009A4208DD3B6813F0010304D19C4A32211B
:102C400011809C4AD3763B68D9030AD59A4B1A78EF
:102C50002AB99A4A127812B9954A32211180012272
:102C60000CE0964B1A7852B18E4A127802F00402A8
:102C700002F0FF011AB91970914B01221A70D6F8AF
:102C80000090002309F1750A3B6009F17706984628
:102C90000AF1020303EB080113F808204B7816F839
:102CA000010C9A420AD23146FFF77EF830B116F88D
:102CB000023C01229A403B6813433B6008F1040840
:102CC000B8F1A00F06F10406E2D17E4B1B7843B1A8
:102CD0003B68DFF8088213F0020F7B4E40F0A181C1
:102CE00096E109F21512019209F58B769846019A40
:102CF00016F8010C531C03EB080113F808204B785D
:102D00009A4229D23146FFF74FF828B396F802C00D
:102D100030796E4B0CF1FF3C4FF00C090CEB4C0C76
:102D200009FB00F99C44634B96F803B003F11C0ABD
:102D30000AEB09014A6862450ED000220AF809B080
:102D40008A60012202FA00F093F84C20C1F804C016
:102D500022EA000083F84C0008F10608B8F1480F99
:102D600006F10606C3D15A4B5A4A1E68D2F800A093
:102D7000DFF86C814FF000099B46D8F80030002B3B
:102D800000F03D811978002900F03981D8F804203D
:102D9000C2EB0A02002A0CDB0AF5FA72C8F804201A
:102DA000012202FA09F294F84C0020EA020284F8A7
:102DB0004C2018F8040C5A780430C0B2002A40F0B5
:102DC000E580394A32F910000190B5F81A01019AEC
:102DD00000F1C80C624501DD9B7814E0019AC83807
:102DE000824202DA9B785B420DE0012303FA09F389
:102DF00094F84C2022EA030384F84C300AF5FA7365
:102E0000C8F80430FBE094F84C2042FA09F2D207EB
:102E100000F1F580002B304ACCBF0220012001399F
:102E200010700A2900F2E380DFE801F0060F1B288A
:102E3000315C6E80929CA60032781344FA2BA8BFB6
:102E4000FA2323EAE373337007E072781344642BA8
:102E5000A8BF642323EAE37373703046FEF77CFF58
:102E6000C5E0F27830461344642BA8BF642323EAFC
:102E7000E373F370216DFEF72BFFB8E03279134452
:102E8000642BA8BF642323EAE3733371AFE0727944
:102E90001344642BA8BF642323EAE3737371A6E091
:102EA0001A0200205C17002062030020A4100020FA
:102EB000CC02002050080020E4020020E50200209F
:102EC000E70200205B170020C403002068D100083F
:102ED00088030020A0100020E60200200C02002041
:102EE00070080020616D4A781A44C82AA8BFC82219
:102EF00022EAE2724A700A781344C82BA8BFC8239A
:102F000023EAE3730B7072E0616DCA7A1A44C82A2F
:102F1000A8BFC82222EAE272CA728A7A1344C82B76
:102F2000A8BFC82323EAE3738B7260E0616D4A7D1A
:102F30001A44C82AA8BFC82222EAE2724A750A7D4A
:102F40001344C82BA8BFC82323EAE3730B754EE0D4
:102F5000626D91780B44C82BA8BFC82323EAE373A2
:102F6000937044E0626D117B0B44C82BA8BFC8234B
:102F700023EAE37313733AE0626D917D0B44C82B2F
:102F8000A8BFC82323EAE373937530E0012A2ED14A
:102F90009B784FF4966292FBF3F38F4A32F910005C
:102FA000B0F5617F05DB40F633029042B8BF0246C0
:102FB00001E04FF46172A2F5617292FBF3F3DBB2B0
:102FC000864A581C0C29107011D194F858209A4246
:102FD0000DD0042B824A28BF02230A2184F85830DE
:102FE00001FB03230633CBF80030FEF7CFFE0123AD
:102FF00003FA09F394F84C20134384F84C3009F198
:103000000109B9F1040F08F10C087FF4B6AE5FE6D0
:10301000AB68D80514D5734B1B681B689B68984731
:1030200070B1D8F800309B070AD5338813F001023D
:103030000CD16D4943F00103E26522660B8006E086
:103040003388012223F00103338000E000223B6833
:10305000590710D57AB1328822F0010102F002023C
:1030600089B292B2318052B9E26522665E4A41F07D
:103070000201118003E0328822F00202328032889D
:103080005A4912F0030F4FF4804014BF48610861A1
:10309000D8F8001011F00A0F21D0DF0609D5540727
:1030A0000AD442F004023280514A1188514A1180F8
:1030B00002E022F0040232809806328806D55106DA
:1030C00007D4494942F040020A8002E022F040025F
:1030D00032805A0603D5464A1188474A118013F4B4
:1030E000006F338814BF43F4807323F480733380FC
:1030F0006B79082B01D00E2B6AD1338823F0400363
:10310000338065E0012200E002225FFA82F808F1D4
:10311000FF3385F86C3603F0B5FE00F05BF9022052
:1031200028214246FEF747FF73E5BAF1000F03D0AE
:10313000BBF17E0F3FF46BADBBF1970F7FF44FAD4A
:103140002E4B4FF4C8721A8063E50023BBF1BB0F0E
:10315000039301D1022304E0BBF1B70F04D14FF672
:10316000FE73ADF80E300CE0BBF1BE0F01D10223AF
:1031700005E0BBF1BD0F7FF44CAD4FF6FE73ADF82B
:103180000C303368BDF80C10B3F854200A44A3F88F
:103190005420BDF80E10B3F856200A44A3F8562068
:1031A00003F070FE00F016F90F2014210122FEF743
:1031B00002FF0023A3762CE5114B00220021DA65E3
:1031C0001A665A669A66DA6619675967996733E428
:1031D00005B0BDE8F08F00BF62030020E6020020CA
:1031E0000C170020B0070020C4030020001001408D
:1031F00030030020DA040020C6030020B8020020BB
:103200005008002000230E49DAB2595C4F2903D040
:1032100001330A2BF7D11A460A4B83F828210022E2
:1032200083F829214FF4E132C3F82C21C3F830216F
:10323000C3F83421C3F83821522283F83C21704767
:1032400079DF0008A410002007B5064B064800935C
:10325000064B074A1968074B03F0DFFC03B05DF823
:1032600004FB00BFADDD000883DF00088400002000
:1032700098DD0008A4DD000810B50446204607F0DC
:1032800095FE10F0FF0F06D10C4B0D481978BDE8E4
:10329000104003F0C2BC204607F0DDFE02280CD827
:1032A000064B0A221870074B074C02FB0030074BF5
:1032B00006301860FEF76AFDE0E710BDA8080020A0
:1032C0009FDF00080C170020D5E1000888030020CC
:1032D000234B70B519684FF47A73B1FBF3F1214BAE
:1032E00021481A78214B224D1B7803F096FC214B84
:1032F00021481968214B2E68B1FBF3F103F08DFCD6
:1033000000241F4BE2B253F8221049B1012303FA03
:1033100002F2324202D01B4803F07FFC0134F0E796
:103320002A6892070DD5184A1848127803EB8203D1
:10333000196A03F072FC164B197A11B1154803F0A3
:103340006CFC1548FEF72EFFBDE87040134B144887
:103350001A88144B92B219884FF4D26303F05DBC03
:10336000A0100020CD030020B0DF00087C0000206A
:103370000C02002080000020EEDF000840420F0019
:103380008CD100080CE000085D17002010E0000858
:10339000A40200201AE000087FE60008BC04002018
:1033A0001EE000086003002010B50748FEF7FAFE93
:1033B0000024064B0648E218E15852680C3403F02A
:1033C0002CFCD82CF5D110BD50E0000838D30008F3
:1033D00066E000082DE9F84303F032FD10B90A2039
:1033E000FEF728FEA64D4FF4D2622846A54907F005
:1033F00093FD95F86C364FF4DA72022B84BF0023EC
:1034000085F86C3695F86C369F4E02FB035303F536
:10341000A87393F850203360022A84BF002283F8F7
:10342000502093F85030994A13700A2202FB03533C
:10343000974A03F26E631360AB6842F201021A40CE
:103440003AB944F208021A401AB98D4A43F40053BB
:103450009360AB68DB0703D54FF40050FFF771F9B9
:10346000AB685F0409D50820FFF76BF94FF40050F3
:10347000FFF767F90120FFF764F9AB681C0706D571
:103480004FF40050FFF75DF90120FFF75AF9AB68E0
:1034900098040ED54FF40040FFF753F94FF4006045
:1034A000FFF74FF94FF48030FFF74BF94020FFF75B
:1034B00048F9784C784B27461C6001F0D5FC774BD7
:1034C00004F1180201201A6001F06EFC014601208F
:1034D00003F07EFC002849D0022001F065FC014683
:1034E000022003F075FC002840D0202001F05CFC95
:1034F0000146202003F06CFCAB68190601D50028BA
:1035000034D0102001F050FC0146102003F060FC84
:10351000AB681A0700D548B3042001F045FC01460A
:10352000042003F055FC30B9082001F03DFC0146B1
:10353000082003F04DFCAB685B0503D400231A465A
:10354000194609E00028F9D110E079B90121C00736
:1035500008D40C33182B0BD051481844007A840738
:10356000F5D5F2E70132D2B2022AF2D9FFF74AFECC
:10357000FEF70CFC4B494C4B366819604B4B06F17F
:103580000409C3F8009006F1750200238846D15C57
:1035900039B9D0188478C078844202D2444B19706B
:1035A00002E00433A02BF2D1424A434B1A60327836
:1035B000424B012A03D0022A03D0414A02E0414A89
:1035C00000E0414A414C1A6006F5D3732360404B3A
:1035D00000229A803F4B404A06F5D771136006F5EA
:1035E000B3726260A3F12202A2602E333B4A2361D0
:1035F00006F5D8731160A361C4F80C806761B5F853
:10360000F00004F04DFD2062B5F8F20004F048FD32
:1036100096F8583004F11C02237796F874306062F3
:10362000637795F82531C4F82C9084F828302C4B1A
:10363000C4F838801A602B4B06F160021A6006F15C
:103640006403236306F25D136363B6F8620104F05A
:103650002BFD0146244804F02FFE244904F078FD98
:10366000234B24491860F06D04F072FD01464FF0C1
:103670007C5004F021FE204B1860BDE8F88300BFA9
:10368000A410002000F8000834020020A808002040
:1036900088030020B4110020FC000020B8040020A2
:1036A0001000002074110020A0080020A4080020B1
:1036B0004C000020981100205002002074000020CF
:1036C000493F0008AD41000825430008CC08002010
:1036D000A40700209C110020BC020020040500204B
:1036E000F00200204C030020000061444C3D0F44D8
:1036F000F8040020DB0F49403C03002010B50446CD
:10370000204607F053FC10F0FF0F07D10B4B0C487D
:1037100093F86C16BDE8104003F07FBA204607F01E
:103720009AFC022808D8054B064C83F86C0603F077
:10373000A9FBFFF74FFEE3E710BD00BFA410002078
:10374000A3DF0008D5E100082DE9F04F7E4985B0E0
:10375000054607F0F3FB7D49002828460CBF0124ED
:10376000072407F0EBFB7A490028284608BF02240B
:1037700007F0E4FB002808BF0424E10740F1B28011
:10378000744803F04AFA0020FFF75EFD724F734859
:1037900003F043FA724803F040FA7A79714B7248A9
:1037A00003EB8203D96C03F038FA3869002104F086
:1037B00063FE00285CD13D460646D5F81080002106
:1037C000404604F059FE00284ED101366748314684
:1037D000D5F814B0D5F818A0D5F81C9003F01DFA50
:1037E0004046002104F052FE10B1614803F015FA82
:1037F0006946404601F05EFB01465E4803F00DFA63
:103800005846002104F042FE10B1594803F005FA71
:103810006946584601F04EFB0146564803F0FDF953
:103820005046002104F032FE10B1514803F0F5F982
:103830006946504601F03EFB01464E4803F0EDF963
:103840004846002104F022FE10B1494803F0E5F992
:103850006946484601F02EFB0146474803F0DDF972
:103860000C2E05F11005A8D14448711C03F0D5F9C0
:10387000434803F0D2F9434DD7F8088055F8041FA8
:1038800019B1414803F0C9F9F8E70D463F4B53F829
:10389000256056B10123AB4013EA080F03D03C4822
:1038A000314603F0BAF90135F0E73A4803F0B5F9CB
:1038B00031467B1893F8103104AA1344364A8A5CC7
:1038C0000131082903F8102CF3D10023334869464D
:1038D0008DF8083003F0A1F9314803F09EF940203B
:1038E00003F066F9A2071AD52E4803F096F92E4880
:1038F00003F093F92D48FFF701FF2D4803F08DF9F0
:103900002A4803F047F82B4803F087F9274803F0CB
:10391000B5F8234803F081F9802003F049F96307E3
:103920000FD5254803F079F9244803F076F91F48AC
:10393000FFF7A2FC1A4803F070F94FF4807003F00F
:1039400037F905B0BDE8F08F6EE00008EDEC000837
:1039500075E000087BE00008A410002089E0000862
:103960009BE000088CD10008A7E00008B2E0000846
:10397000A4E1000817E0000869E00008BAE00008C8
:10398000CCE00008E4D20008DCE00008E8D200083F
:10399000EAE00008F7E0000815E3000803E100088A
:1039A0007FE600080CE100081FE10008D5E10008EF
:1039B0002DE1000837E1000846E1000857E1000862
:1039C0002DE9F047784B86B01A789A46DFF8EC91EB
:1039D000BAB901238AF80030744BD9F8002059682D
:1039E000914204D019690C33914218BF002302217F
:1039F00059726F4B6F48DA63FEF7D4FB6E48FEF7DF
:103A0000D1FBD9F8000003685B689847002800F0F4
:103A1000C7806A4B664C186803689B6898470928FA
:103A2000014601D03F2853D14FF00008266C644F67
:103A300045462EB163483968324607F0BFFA10B9DF
:103A4000B84605B93D46604B0C379F42F1D3EDB106
:103A5000D5F800E0D8F800C0236C55481EF8037074
:103A60001CF80310B94211D15A1C51B92D2B08D89A
:103A7000026403442027024483F8447082F844100F
:103A800004E0234483F844702264E5E7236C0BB11F
:103A9000454512D04D48FEF785FB454509D855F8F8
:103AA0000C0BFEF77FFBD9F800000921FEF7E0FAC6
:103AB000F3E74148FEF776FB0026236C9E42A0D236
:103AC000404BD9F80000995DFEF7D2FA0136F4E7D1
:103AD000236C33B904283DD104F1440003F02AFBE0
:103AE0005EE00C2801D13A4886E70A2901D00D2969
:103AF0004CD13848FEF756FB236CE218002382F8BD
:103B0000443094F84420232A17D00493324B2D4E8E
:103B1000009303A82A4912220C23039607F09FFA68
:103B2000054638B1006807F041FA0130AB6830440F
:103B3000984702E02948FEF735FB22480021302251
:103B400007F0F3F9002323649AF80030002B7FF488
:103B500055AF25E00C28C6D07F2903D151E72F2B84
:103B60003FF64FAFA1F12002D2B25E2A3FF649AF35
:103B700013B920293FF445AF5A1C2264D9F800003C
:103B80001C4484F84410FEF773FA3AE77F29E6D123
:103B9000013B23640022234483F8442010482EE78D
:103BA00006B0BDE8F08700BF5B17002010000020C2
:103BB000CC08002069E10008A1E1000860050020B0
:103BC00038D300081009002010D40008A6E100082E
:103BD000ABE100087FE60008D9180008B6E100084C
:103BE000D2E100082DE9F04FC24AC34C87B01068FB
:103BF000516804AB03C3DFF8249300214FF4D26271
:103C0000204607F092F904F5A873C9F80030BB4BC1
:103C10000025DFF80CB31D7004F26E63CBF80030A2
:103C20005623237003236371A3604FF41673A4F823
:103C3000F030FA23A4F8F2302A23A4F8EE304FF43F
:103C4000FA73A4F8F630202384F8F4306E2384F855
:103C500004312B2384F805314FF4C873A4F80831DC
:103C600040F24C43A4F81C3140F26C73A4F81E31AE
:103C700040F27E43A4F8D03040F23A73A4F8D23038
:103C80004FF47A73A4F8D43040F27E53A4F8D630BF
:103C900040F2EA53A4F8D83040F2B4530127322658
:103CA000212240F2DC514FF01E0A1920A4F8DA302C
:103CB0004FF47A5384F80621A4F81A1184F82501E8
:103CC000A4F8DE30019084F8EC7084F821A184F827
:103CD000247184F82771A4F8DC60A4F8E0600291F4
:103CE0000392FFF78FFA40F6AC53A381D9F8003066
:103CF0004FF0170E83F818E083F819E04FF0550ED7
:103D0000A57383F806E04FF00F0E83F808E04FF03C
:103D1000220E83F809E04FF00E0E4FF0280883F8CA
:103D200013E04FF02D0C4FF0350E83F80EA083F802
:103D30000FA083F810C0DE7183F81DE01D7083F8BA
:103D4000048083F805809D765D74DD769D741D7713
:103D500001984FF05A0E9872039A69481A755322C7
:103D60009A776422DA774FF00A0A782283F80BE018
:103D70005A7383F817C083F815A083F80C8083F872
:103D80002170D86318644FF08240D8624FF07C50A5
:103D90009863DFF890C15B48C3F824C0C3F828C01B
:103DA0005864594A5948DFF880C102991A635A6326
:103DB0009864C3F84CC084F86EE64FF0410E84F866
:103DC0007066A4F8761684F86FE684F8725684F864
:103DD000735684F8715684F874569A664C4A0421D6
:103DE000DA664C4A83F858101521D86583F8747048
:103DF000A3F85450A3F85650A3F8525083F86080AB
:103E000083F8618083F864101A67434800F0B4FFB8
:103E1000D9F800604FF44873A6F86231C82386F8D9
:103E2000A7314FF49663A6F8A83140F2D933A6F82B
:103E3000AA3140F6430386F86071A6F8AC3186F8E3
:103E40005D5186F85E5186F85F8186F8645186F888
:103E5000A6A133465F464FF47F72A3F866214FF464
:103E6000FA62A3F8682104A940F2DC52A3F86A219F
:103E70004A5D013583F86C21082D4FF0FF0283F86D
:103E80006D2103F10803E6D1012386F8AE3186F8EF
:103E9000AF3186F8B0310023E21810330021C02B77
:103EA000154D1161F8D1314605F541704FF4DA72C4
:103EB00007F032F8314605F597604FF4DA7207F0F3
:103EC0002BF83B6805F5CF625968186803C2198959
:103ED00022F8021B1968C5F88216596851601B89BF
:103EE0001381012385F85433022385F8083507B080
:103EF000BDE8F08F38D20008A4100020A8080020E8
:103F00008FC2753DCDCC4C3D9A99193F0000A04021
:103F1000F6287C3F3D0A773FD6E1000834020020B6
:103F200088030020000020400000404008B50548FC
:103F3000FEF738F9FFF756FE02F0A4FFBDE808408F
:103F400001F035BDDFE100082DE9F04F8BB009939A
:103F50008A4B0792B3F90220B3F90030002AB8BFA8
:103F60005242002BB8BF5B429A42B8BF1A46844BFC
:103F700003921B88814603F00302069203F00202BB
:103F800003F0010392B205930023089219461E46DE
:103F9000184604931F461A46069C002C41D0022A5C
:103FA0003FD0764C079F0D5F7C426D00A54203DB3E
:103FB0003C46A542B8BF2C46724DDDF824A031F92D
:103FC00005C03AF90150CCEB040404EB050C99F858
:103FD0000750642405FB0CF595FBF4F599F81B409C
:103FE0006FF004076743BD4205DB04EB8404A54280
:103FF000B4BF2F462746644D5C59644442F2107C9E
:104000006445A8BF6446DFF898C16445B8BF6446FC
:104010005C5199F811506C4324130494069C012CB4
:104020003BD05A4D55486D5E594C85EAE576A6EB76
:10403000E576B6F5206F085E19F802C053F80480E3
:104040001DDC022A15D05026464396FBFCFC0426B4
:1040500095FBF6F5C5EB0C0CE0444E4EB8F57A5FD7
:10406000A8BF4FF47A58B045ACBF44F80380E6507F
:1040700007E080EAE076A6EBE076642EE3DD00253B
:10408000E550434C1E597D2496FBF4F609EB0204DF
:10409000A47A6643402496FBF4F6089CB4B1022A45
:1040A00068D0DDF80CA0DDF810B00AFB00F40AFBC4
:1040B00006F8CAF5FA7505FB074405FB0B854FF4B6
:1040C000FA7C94FBFCF495FBFCF506E0059C002CC7
:1040D00050D0022A4ED0049D3C46DFF8B0C04FF0CD
:1040E000040B31F80CC00FFA8CF898FBFBFADFF8E0
:1040F000B4B012F80BB00BFB0AFA6FF04F0B9AFB3F
:10410000FBFAA244CDF804A0DFF89CA0042431F906
:104110000AB021F80AC0CBEB08080AF1080C98FB9A
:10412000F4F80AF114041C5953F80CB00AF1140AFB
:10413000A34453F80C40C34443F80A40164CDDF83E
:1041400004A0145D013204FB0BFB20249BFBF4FB59
:10415000CBEB050B114DDA44032A43F80C8021F810
:1041600005A003F1040301F102017FF415AF0BB0C8
:10417000BDE8F08F35460446AFE700BF9A03002044
:10418000C403002020030020AC08002054030020BA
:10419000B408002080C1FFFFA8030020A00A00206F
:1041A000F0D8FFFFA2030020400900202DE9F04FC6
:1041B00089B00793524B0291B3F9043001920393F3
:1041C000504B06461B8803F0010103F002039BB22B
:1041D00004934D4B0691B3F800A04FF6FF714FEAE0
:1041E0001A13B1FBF3F1002305911D461946022D68
:1041F00008D1029FDDF80CC07C791B340CFB04F461
:10420000641129E03E4C019A31F9048057424FEA8B
:104210004804BC4203DB1746BC42B8BF27463B4CB0
:10422000DDF81CC00C5F3F1B3CF901403A19069CAD
:104230007CB9029C277907F11B0408FB04F4049F56
:1042400024114FB190F811C00CFB02F704EB2724A6
:1042500002E0C479544324112D4FDFF8C48031F9B2
:1042600007C004279CFBF7FCCCEB040C0AFB0CF406
:1042700096F80AB053F80870E4120BFB0474254F4B
:10428000B4F5001FA8BF4FF40014BC42B8BF3C46B1
:10429000214F10F80590DA5943F8084043F807C059
:1042A000C2EB0C0809FB0CF9DDF814C001350CFB5E
:1042B00008F807F10C0C1837DA5953F80CB04FEA2C
:1042C000A818934453F80C20C344DA51377D032DCA
:1042D00007FB0BF74FEA272707EBE91707EB6434D7
:1042E0000E4F43F80C80CC5306F1010601F1020198
:1042F00003F104037FF47BAF09B0BDE8F08F00BF8A
:104300009A030020C4030020600300202003002043
:10431000540300200000E0FF60090020A00A0020F4
:10432000B40800202DE9F04F89B00793714B814606
:1043300018880492039103F0B3FE6F4903F008FF5D
:10434000029002994FF07E5003F0B6FF00240690D1
:104350004E462546A046B8F1020F684B0BD1039993
:10436000B3F904004A790A32504303F09DFE6449D0
:1043700003F0A2FF35E0049A5F5F53429F4203DBE4
:1043800013469F42B8BF3B465E4AAA5E9B1A079AF5
:10439000505F184403F088FE5B4903F08DFF5B4BD0
:1043A0008346B3F800A01AF0010F04D0D9F84410E6
:1043B00003F0CEFE15E0039B18791430784303F028
:1043C00073FE4F4903F078FF1AF0020F074609D039
:1043D000D9F84810584603F0BBFE0146384603F0B2
:1043E000AFFD07464A4BDFF84CB1585F03F05CFE67
:1043F000484BD96803F0ACFE82465146384603F07C
:104400009DFD316A074603F0A3FE029905903846E8
:1044100003F09EFEF16A03F09BFE54F80B1003F0CC
:104420008FFD3D49074604F031F830B938463B4925
:1044300004F04AF810B1394F00E0374F4BF80470E0
:10444000DFF8F4B0504654F80B1003F077FD44F851
:104450000BA0069903F07CFE0BF10C03E2580BF164
:10446000180B54F80B10824610460192009303F08B
:1044700067FD514603F064FD019A009B44F80B2050
:1044800044F803A0264903F017FFB16B03F060FE68
:104490002449824603F0FAFF38B95046224904F015
:1044A00013F820B1DFF880A001E0DFF878A00598CC
:1044B000394603F045FD514603F040FD06F09AFFF2
:1044C0001A4BB0F57A7FA8BF4FF47A709842B8BF04
:1044D000184608F10108164BB8F1030FE85204F131
:1044E000040405F1020506F104067FF434AF09B0B7
:1044F000BDE8F08F60030020BD3786359A030020A9
:10450000000048422003002000002041C403002096
:10451000540300203802002000007AC300007A43D0
:1045200000004040000096C30000964318FCFFFFC7
:10453000A00A0020C00800208409002070B50E46A3
:104540002021154606F025FD0446B8B1441C20463E
:1045500006F081FDB0F5617F05DB40F6340398423B
:10456000A8BF184601E04FF461701923A0F56170EF
:1045700090FBF3F030702B7801332B702046202114
:1045800006F007FD0446B8B1441C204606F063FD62
:10459000B0F5617F05DB40F634039842A8BF1846AA
:1045A00001E04FF461701923A0F5617090FBF3F006
:1045B00070702B7801332B70204670BD30B51049D8
:1045C000104A0C78104B8CB19C6E15680444A542BF
:1045D00015D3126800209A660C4A0870117809B148
:1045E00001391170012283F86C2030BD986E146877
:1045F000C830844203D31268012008709A6630BD27
:1046000011040020A010002040090020E602002034
:1046100037B5204D8DF8073095F86D308DF80620B0
:1046200002AA8DF804008DF805101A4412F8042C23
:10463000443AD2B20F2A09D81749022B31F8124056
:1046400008D89CB12046FFF7B9FF0FE0022B4FF0CE
:10465000C804F7D9114B1A68AB6E121B934205D2EE
:104660000C4A002382F86D300D4A137095F86C30B7
:10467000012B00D064B995F86D30022B03D8054AA0
:10468000013382F86D30074A002385F86C301370CF
:1046900003B030BD4009002040D20008A010002027
:1046A000E602002011040020F0B5934C934A2368E1
:1046B0009D8AADB2E9B211F0010F36D0198821F40C
:1046C00000610904090C1980198889B241F48061DC
:1046D0001980002182F86E10894908788949B8B19B
:1046E00092F86F0018B988480078FF2810D101208F
:1046F00082F86F0085480078022804D1188880B2BB
:1047000040F400601880097841F00101198216E137
:10471000097801F0FE0119827B4B1B78FF2B00F01A
:104720000E81FF2382F86E3009E18F0740D5BFF379
:104730005F8F76490878C0B2012816D1704D2D7868
:104740009DB192F86F5085B1198821F480610904F8
:10475000090C1980BFF35F8F198B198882F87000DC
:1047600089B241F4007119801DE0188BBFF35F8F8F
:10477000087802280CD16248007848B192F86F009E
:1047800030B1198821F480610904090C1980D0E046
:104790000978032907D15A49097821B192F86F1095
:1047A000002940F0C680998889B241F48061C5E053
:1047B0004E0764D5012182F870105149097800290B
:1047C0003ED092F86F1000293AD0504992F86E000E
:1047D00009784F4D022919881FD921F480610904F5
:1047E000090C19801F8A2E68C1B2FFB240B237543B
:1047F000188880B240F4007018808B1C82F86E30EC
:10480000236828681D8A013149B2EDB24554998860
:1048100089B241F4806199802CE089B241F4007141
:1048200019801E8A2D68C1B2F6B240B22E541B8A7E
:10483000481C40B2DBB203312B5482F86E1019E0F1
:1048400092F86F1011B93349097851B1198889B2BA
:1048500041F40071198092F86E30013382F86E30A5
:1048600008E0198889B241F480711980234B012135
:1048700083F86F1021680B88D805FCD45FE001F045
:10488000400101F0FF06214809B32149B3F810C0E7
:104890000F6892F86E105FFA8CFCCDB26E1C49B2B4
:1048A000F6B207F801C082F86E60077876B2F11CA4
:1048B0008F4205D1998821F480610904090C9980FF
:1048C0000378B3423BD1023582F86E5037E02906B7
:1048D00035D592F86E104DB26F1C1FD00E4E0131BF
:1048E0003668C9B2755D82F86E10EDB21D8200782F
:1048F00049B2884223D11CE0C00E002040090020AC
:10490000B30E0020B00E0020B10E0020BC0E00201F
:10491000B80E0020B20E0020B40E0020144982F818
:104920006E600978C9B219821249097809B901780B
:1049300029B9998821F480610904090C99800E4BEA
:1049400092F96E1018780D4B421C91420FD1002243
:1049500083F86F2093F8703033B12268938823F482
:1049600040731B041B0C9380054B00221A70F0BD92
:10497000B10E0020B30E0020BC0E00204009002024
:10498000BD0E00200C4B07B51B68196819B10B4A06
:104990009069014391619A889868ADF804200222D9
:1049A0008DF8072004220DEB02018DF80620FDF79B
:1049B0004BFF03B05DF804FB4C05002000100240E3
:1049C00010B50A4C23681BB1FFF7DCFF00232360FE
:1049D000074B1B7813B1012B03D010BD4FF40062BD
:1049E00001E04FF48052034B1A8010BD4C050020AB
:1049F00050050020000000200D4B0278D968437854
:104A0000C943C1F30221C1F1040103FA01F1094BC9
:104A10000901C9B21A4482F8001302780120510931
:104A200002F01F0200FA02F243F82120704700BF93
:104A300000ED00E000E100E0254B10B55343254AAE
:104A4000254C12680139B2FBF3F20388013AA04207
:104A500089B292B29BB212D004F50064A0420ED08B
:104A6000B0F1804F0BD0A4F59834A04207D004F5E4
:104A70008064A04203D004F58064A04202D123F0F8
:104A800070039BB2154CA04206D004F58064A0428E
:104A90001CBF23F440739BB203800F4B8185984267
:104AA00002850FD003F5006398420BD003F54063F5
:104AB000984207D003F58063984203D003F58063E2
:104AC000984201D1002303860123838210BD00BFD9
:104AD00040420F0080000020002C014000100040E8
:104AE0002DE9F74FA24E0C4637780546114600686F
:104AF00091469B4622467B1C06F8043BFFF79CFF31
:104B0000AB686868ADF8043018238DF8063001A949
:104B100002238DF80730FDF797FE2B7B3F0106EB54
:104B2000070A2C680C2B00F2F280DFE813F00D006E
:104B3000F000F000F0004D00F000F000F000820006
:104B4000F000F000F000B600238C8A4823F0010347
:104B50001B041B0C2384218CA288238B844223F00A
:104B600073034FEA03434FEA134389B292B243F00F
:104B7000700314D000F50060844210D000F540604E
:104B800084420CD000F58060844208D000F580603B
:104B9000844204D021F0020141F0030107E021F03A
:104BA0000E0122F4407241F0030142F48072A280AF
:104BB0002383A4F834B02184238B23F008031B043F
:104BC0001B0C43F0080332E0238C6A4823F01003E7
:104BD0001B041B0C2384218CA288238B844223F486
:104BE000E6434FEA03434FEA134389B292B243F4D8
:104BF000E04308D000F50060844204D021F0200199
:104C000041F0300107E021F0E00122F4406241F080
:104C1000300142F48062A2802383A4F838B021845A
:104C2000238B23F400631B041B0C43F400632383D6
:104C30006DE0238C4F4823F480731B041B0C2384EA
:104C4000218CA288A38B844223F073034FEA034391
:104C50004FEA134389B292B243F0700308D000F5D3
:104C60000060844204D021F4007141F4407107E0F7
:104C700021F4606122F4405241F4407142F48052C8
:104C8000A280A383A4F83CB02184A38B23F0080363
:104C90001B041B0C43F0080338E0B4F820C0354A6D
:104CA0002CF4805C4FEA0C4C4FEA1C4CA4F820C05A
:104CB000B4F820C0A388B4F81C802CF4005C28F45D
:104CC000E6484FEA08484FEA0C4C4FEA18484FEACA
:104CD0001C4C94429BB248F4E0484CF4405C03D036
:104CE00002F50062944203D123F4804343F48043ED
:104CF000A380A4F81C80A4F840B0A4F820C0A38B23
:104D000023F400631B041B0C43F40063A383AB7BFD
:104D100043B1B4F844306FEA43436FEA53439BB264
:104D2000A4F8443023889BB243F0010323802B7BFB
:104D30000C2B14D8DFE803F0071313130A13131313
:104D40000D131313100004F1340307E004F13803CA
:104D500004E004F13C0301E004F14003F351504648
:104D6000AAF80890CAF8044003B0BDE8F08F00BF6D
:104D7000B4090020002C014070B50546441E14F80B
:104D8000011F61B1064E304606F003F90028F6D047
:104D9000861B0448631B304480F81031EFE770BD78
:104DA00015E30008A410002070B50022064628492B
:104DB0001301585CB04204D00132072AF7D1002019
:104DC00070BD244D0B4405F1C404102E0FCB84E8B4
:104DD0000F002B4617D007D8012E0DD0022E34D14C
:104DE0001D4B1B689B680BE0202E27D0402E2CD13A
:104DF000194B1B681B6903E0174B1B685B6820E0BD
:104E0000C5F8C8301DE0154A1268127A042A1CD869
:104E1000DFE802F00A0A030A0A00114AC5F8C820AE
:104E2000C5F8CC20032206E04FF4E132C5F8C820D3
:104E3000C5F8CC20012283F8D12006E0064B1B6880
:104E4000DB68C5F8CC30204670BD064870BD00BF99
:104E500060D20008B4090020B8040020FC00002043
:104E6000A0860100780A00200F4970B500230C7855
:104E70001A46D8B2844205D00D7B854208BF012076
:104E80000CD100E000200C2505FB0010074D084E5A
:104E9000154495F828510132755D05720133052BD3
:104EA00001D0012AE5D970BD10000020A410002017
:104EB00079DF000830B587B005460C4603A800210D
:104EC0000C2206F032F82846002103F0FDFA20B14A
:104ED00028462A4903F034F803E02846274903F01E
:104EE0002DF8274903F034F903F0F8FA054685EA6E
:104EF000E570A0EBE57069460A22FDF7DBFB0023B5
:104F00009D420370ACBF20232D2368468DF80C30E2
:104F100006F04CF8012807D130238DF80D308DF8BC
:104F20000E308DF80F300CE0022805D130238DF8BB
:104F30000D308DF80E3004E0032804BF30238DF8C7
:104F40000D30694603A806F017F803A806F02EF8FE
:104F50000338C5B22A4603A9204606F051F80023BB
:104F600063552046074906F007F803A9204629445F
:104F700006F002F8204607B030BD00BF6F12033ABA
:104F800000007A442AE300087C4B70B51B78012BA3
:104F90000CBF0325002599BB048C24F001042404D4
:104FA000240C0484038B048C9BB223F0F30343F0A2
:104FB000010343EA0515724BA4B2984215D003F5DC
:104FC0000063984211D0B0F1804F0ED0A3F5983312
:104FD00098420AD003F58063984206D003F58063B7
:104FE000984218BF24F00A0401D124F0020444F0CE
:104FF0000104224305830284038B23F00C033AE06F
:1050000004293FD1048C5E4B24F010042404240CAA
:105010000484018B048C21F440710905090D41F4CD
:1050200080719842A4B241EA053512D003F50063BD
:1050300098420ED0B0F1804F0BD0A3F59833984230
:1050400007D003F58063984203D003F5806398424C
:1050500007D124F0200444F0100444EA021292B272
:1050600004E024F0A00444F01004224305830284E9
:10507000038B23F440631B041B0C0383038B9BB241
:10508000038370BD0829018C37D121F48071090494
:10509000090C0184838B048C9BB223F0F30343F04F
:1050A000010343EA0515364BA4B2984212D003F52A
:1050B000006398420ED0B0F1804F0BD0A3F5983327
:1050C000984207D003F58063984203D003F58063CC
:1050D000984207D124F4007444F4807444EA022214
:1050E00092B204E024F4206444F480742243858363
:1050F0000284838B23F00C0338E021F480510904EF
:10510000090C0184838B068C23F440731B051B0D53
:1051100043F4807343EA0535194BB6B2984212D076
:1051200003F5006398420ED0B0F1804F0BD0A3F589
:105130009833984207D003F58063984203D003F573
:105140008063984207D126F4005646F4805646EA1A
:10515000023292B205E047F6FF54344044F48054E2
:10516000224385830284838B23F440631B041B0C3E
:105170008383838B9BB2838370BD00BF6405002053
:10518000002C014038B510F80E2C044650F8043CB1
:1051900052B9012200F80E2C20F80C1C197B18685B
:1051A0000222BDE83840EFE630F80C2C20F80A1C4B
:1051B000891A89B220F8081C084A10F80F0C00253B
:1051C00002EB4002A2F8D41004F80E5C1868197BB8
:1051D0002A46FFF7D9FE04F8065C38BDB409002062
:1051E0001F4B10B55A6802F00C02042A03D0082A9B
:1051F00004D01C4A14E01C4A126811E05A6859682D
:10520000C2F38342C90302F1020201D4174906E046
:10521000596811F4003F1449096818BF49084A4306
:1052200002605968124AC1F30311545C0168E140FD
:1052300041605C68C4F30224145D21FA04F48460C4
:105240005C68C4F3C224145DE140C1605B68C3F3D1
:1052500081331A44137CB1FBF3F1016110BD00BF2F
:105260000010024000127A002800002000093D00D2
:105270004D000020CB78F0B5DA0648BF8A7809885F
:1052800003F00F0548BF154311F0FF0F1DD0046850
:1052900000220127974007EA0106BE4211D197007C
:1052A0004FF00F0C0CFA07FC05FA07F724EA0C0480
:1052B000282B44EA070401D1466102E0482B08BFCD
:1052C00006610132082AE4D10460FF291FD944682D
:1052D000002202F108060127B74007EA0106BE4294
:1052E00011D197004FF00F0C0CFA07FC05FA07F7E5
:1052F00024EA0C04282B44EA070401D1466102E0A9
:10530000482B08BF06610132082AE2D14460F0BD93
:1053100010B50446FCF7EDFA012806D11CB1FCF7E4
:10532000E8FA013CF8E7052010BD002C08BF052075
:1053300010BD00BF2DE9F04FAE4E85B03778032F7A
:1053400014D9AD4BAD48B3F90410B0F904200029CD
:10535000B8BF49426FF063035B1A9A4204DB01F164
:1053600064039342A8BF134683801FE0012F1DD81A
:10537000A34BA44C1B78013B142B00F2DF81DFE828
:1053800013F09100DD01DD0168009F00DD01DD010A
:105390002F01DD01DD01DD01DD01DD01BD00DD01EC
:1053A000DD01DD01DD01DD019F01B601924B964972
:1053B000B3F806A0914B0968B3F80280B3F80090E7
:1053C000B3F904B0914C02910025BD4204F11004E0
:1053D000CED20FFA8AF002F067FE54F8101C02F0E9
:1053E000B7FE03460FFA88F0019302F05DFE54F811
:1053F000081C02F0ADFE019B0146184602F0A0FD1C
:1054000003460FFA89F0019302F04EFE54F80C1C8B
:1054100002F09EFE019B0146184602F091FD029AA1
:10542000034692F90000019340420BFB00F002F0AA
:105430003BFE54F8041C02F08BFE019B014618460B
:1054400002F07EFD03F04AF8714B23F81500013598
:10545000BBE702210420FCF7B9FE684D0121AF88AB
:1054600078431FFA80F80420FCF7B0FE6D8800FB3B
:1054700005801FFA80F80420FCF7B6FE4044208126
:1054800002210520FCF7A2FE7843012187B2052006
:10549000FCF79CFE00FB057087B20520FCF7A4FE1C
:1054A00038440BE005200121FCF790FE534B9D880A
:1054B000684385B20520FCF797FE284460813DE1F2
:1054C000544B00201D68FCF78FFEDFF8608195F9D2
:1054D0000630B8F902203227534393FBF7F3184400
:1054E00020800120FCF780FE95F90E30B8F90020ED
:1054F000534393FBF7F7384460801FE1464B1B781A
:1055000013F0040F454B02D11B689B880BE0196810
:10551000394A0B88B2F9062049889A4203DB914246
:10552000B4BF0B461346E381E289394B394F1A80E9
:105530003B4B1B681D7845B30220FCF755FE3A68CB
:10554000B2F91030518A984203DB0BB29842B8BFCF
:105550000346344909684889C3EB000E274B0FFA0C
:105560008EFED9880FFA81FCF44501DA0D4401E082
:1055700001DD4D1BDD8092F91620B3F9063053434F
:10558000642293FBF2F31844A080274B1B88DB05B1
:105590000CD5194B1A88D7F80090E28022819A889E
:1055A000184F62815B880325A38101E0134BF1E76B
:1055B00009EBC50393F90630B7F90680284608FBC6
:1055C00003F8642398FBF3F8A7F80680FCF70CFEB9
:1055D00001354044072DF88007F10207E8D1ADE01E
:1055E0000D4B1B7813F0040F0C4B21D11B689B88CB
:1055F0002AE000BF341700209A030020A00A0020F0
:10560000000500206200002004050020E0060020C4
:1056100036170020D00800205C170020D808002092
:10562000DC080020E0080020C40300202003002044
:105630001968AD4A0B88B2F9062049889A4203DB03
:105640009142B4BF0B461346E381E289A74BA84DB4
:105650001A80A84B03201B880121DF0503D5FCF726
:10566000B5FDA14F02E0FCF7B1FDA34FB7F80280F2
:10567000022100FB08F01FFA80F90320FCF7A6FDC9
:105680003F88012100FB0790E8800420FCF79EFD85
:1056900000FB08F002211FFA80F80420FCF796FDB9
:1056A00000FB078028810320FCF79EFDE388184457
:1056B000E0800420FCF798FD2389184420813DE018
:1056C00001210420FCF782FD8B4D6F88784387B25F
:1056D00004202781FCF788FD384420810121052022
:1056E000FCF774FD2D88684385B26581E2E6824B44
:1056F0000325B3F80490984628460221FCF766FD7E
:1057000000FB09F0012187B22846FCF75FFDC5F1D7
:1057100006035B0838F8133000FB037087B224F8E7
:1057200015702846FCF760FD384424F81500013553
:10573000072DE1D16C4BDA886C4B1A806F4DDFF886
:10574000E491AB6813F0200F34D00020FCF74CFD3F
:10575000208080460120FCF747FD694B644F1B68A1
:1057600060801A0626D5674B1B681B7813F0020F62
:10577000654B23D0D9F800C0B3F900109CF90E2076
:105780009CF906C0B3F902304A43CCF1000C03FB8C
:105790000CF3322192FBF1F26FF0310C92B293FBD9
:1057A000FCFC9444E04493FBF1F1A7F800800A4428
:1057B00010447880D9F80010002319E0D9F80010BF
:1057C000B3F902C091F90620B3F900300CFB02FCDA
:1057D00032229CFBF2FCE044A7F8008091F90E1005
:1057E0004B4393FBF2F2E3E7E2520233102B0CD06F
:1057F000E05E31F9232001EB830790427F88F3DBE1
:105800003AB28242A8BF0246EEE73E4B1B681B78C5
:105810005B0704D435493478088801231BE03B4BEF
:1058200000241F780423043FFFB25FFA87F84FFA81
:1058300088F2D4420BD4364A03F10109381932F800
:1058400013105FFA89F9C0B2FCF7E4FF4B4601344C
:10585000042CECD1DEE7A34208D231F9132000B2C8
:105860008242A8BF104680B20133F4E7294B4FEAC9
:1058700044081A68AB6803F480550395244D03F07F
:105880001009254BB5F90660244D1B782F68244D6F
:1058900003F00403DBB2D5F800C0029300234345B4
:1058A00062D0B2F802A004B2544505DD0F4CC0EB43
:1058B0000A0A1D5B55441D53039D0C4C002D33D02B
:1058C0007D8931F903A0AE42CBBFBCF80250958868
:1058D000B2F802B0BCF800B0AA4503DBDA45B4BFA9
:1058E00055465D46E55238E09A0300203617002001
:1058F00062000020C4030020A00A0020A4100020A1
:1059000004040020E4080020200300206705002094
:1059100062030020D80800205C170020E008002067
:10592000D4080020D008002031F903A01588B2F86F
:1059300002B0AA4503DBDA45B4BF55465D46E552E1
:1059400004EB030ABC89A64207DAB9F1000F01D1C2
:10595000148800E09488AAF80040029C14B9044C12
:105960001C5BCC5202339AE705B0BDE8F08F00BF54
:10597000DC04002013B50122044600210068FFF773
:105980005BF8236801A81A8892B242F001021A80DB
:10599000637B00228DF8043001238DF805308DF8EB
:1059A00006208DF80730FFF727F802B010BD10B5BC
:1059B0000848FCF7F7FB084B1C68236820461B6966
:1059C000984718B90A20FCF7ECFAF6E7034A044BAB
:1059D000DA6010BD2CE30008600500200400FA0521
:1059E00000ED00E0826A8169436B1144D960416A2D
:1059F000914203D98A1A5A60816204E001698A1AC5
:105A00005A6000228262002280F844201A6842F024
:105A100001021A60704770B5046D4279A38902F0E3
:105A2000040123F400531B041B0C0546866886B052
:105A3000A38101F0FF0021B14FF480604FF40051C9
:105A400000E0014612F0010F14BF0423002312F0FE
:105A5000020F1CBF43F008039BB212F0080F228A0A
:105A600018BF0C2392B222F4405211432182A28922
:105A700092B222F4B05222F00C02104303439BB2C4
:105A8000A381A38A01A823F440731B041B0CA382E7
:105A9000FFF7A6FB1949049A039B8C4208BF1346E3
:105AA000A2891921594312B2002AB4BF7600B60068
:105AB000B1FBF6F16423B1FBF3F21201100903FB11
:105AC0001011A08900B2002806DAC9003231B1FBFA
:105AD000F3F303F0070305E009013231B1FBF3F3FF
:105AE00003F00F031A4392B22B6D22819A8992B26E
:105AF00042F400529A8106B070BD00BF00380140E8
:105B0000417188E7816086E7F8B50468054620465C
:105B10000E461746FCF761FE032845D82B7B9B08F1
:105B20009AB246B94FF0020C0CFA03F3A18989B27C
:105B300021EA0303A3810A2101FB00211B4B43F847
:105B40002160043143F8217046B12A7B0225920876
:105B500005FA02F2A1890A4392B2A281282202FB2D
:105B6000003000F12002EFF31286502383F31288F5
:105B70000023C1180D6915B115600A690432043398
:105B8000102BF6D100231360F3B283F31188036A5C
:105B900023B1A3899BB243F0010304E0A38923F05E
:105BA00001031B041B0CA381F8BD00BF580F00208C
:105BB0002DE9F0411D46A24B8CB09842884617460D
:105BC0005CD1A04CA04BA2602360A04B2065636118
:105BD00003F58073A3614FF48073E36023619C4BF2
:105BE000A907A364E36403F5484303F15403236363
:105BF000A3F11403D3F8D42F636342F48042C3F8B3
:105C0000D42FD3F8D02F42F00102C3F8D02F4FF099
:105C100002038DF803304FF40073ADF800304FF0FD
:105C200018038DF8023003D58A486946FCF70CFE4C
:105C30001C232A078DF8023003D586486946FCF7F5
:105C400003FE4FF48063ADF8003048238DF8023036
:105C5000EB0703D57F486946FCF7F6FD0E238DF868
:105C600004300022012301A88DF805308DF80620AC
:105C70008DF80730734CFEF7BFFE54E0764B984228
:105C800040F0DA80754B704A9F601A604FF4807262
:105C9000DA601A61724A18655A6102F580729A6177
:105CA000704AAE079A64DA646F4BDA6942F40032E4
:105CB000DA615A6942F001025A614FF002038DF82D
:105CC00003304FF00403ADF800304FF018038DF8A7
:105CD000023003D55F486946FCF7B6FD1C232C074C
:105CE0008DF8023003D55B486946FCF7ADFD08230B
:105CF000ADF80030E8074FF048038DF8023003D5C7
:105D000054486946FCF7A0FD26238DF80430002294
:105D1000012301A88DF805308DF806208DF8073095
:105D2000FEF76AFE4D4C0026012384F844302662BB
:105D3000E661A6626662C4F82C806571A760A671F0
:105D40002046FFF768FE15F0090F31D0206B0028C0
:105D500026D0E36C039601934FF480530A9380237B
:105D60000693E368059604932023099363690796D5
:105D7000029308960B96FBF7EFFD01A9206BFBF74A
:105D8000CDFD236B1A6842F001021A60226D918AE0
:105D900089B241F0400191825B689BB2236407E0C5
:105DA000236D4FF6DF721A80DA6842F02002DA6063
:105DB00015F00A0F2CD0606B28B3A36C002601935A
:105DC0004FF480530A938023069323690296049329
:105DD0001023039305960796089609960B96FBF7F2
:105DE000BBFD606B01A9FBF799FD636B1A6842F07C
:105DF00002021A605E605E60236D9A8A92B242F07F
:105E000080029A8204E0236DDA6842F08002DA6050
:105E1000236D29079A8992B242F400529A819A8A94
:105E200003D592B242F0080203E022F00802120405
:105E3000120C9A82204600E000200CB0BDE8F081F0
:105E4000003801404C100020D0D20008A80A0020E1
:105E5000043801400008014000440040F80F0020D1
:105E6000A80C002004440040001002402DE9F04737
:105E7000054605F09BF8324B0446D3F808809A4655
:105E800090B93048FCF78EF92F4B53F8241049B1E4
:105E90000123A34013EA080F02D02C4800F0BDFEF6
:105EA0000134F1E72A4821E028462A49224605F034
:105EB00085F858B92848FCF775F9284C54F8041FA0
:105EC0000029EFD0214800F0A8FEF7E72B78002644
:105ED0002D2B03BF013504F1FF344FF001094FF0C2
:105EE0000009194B53F8267027B91D48BDE8F04743
:105EF000FCF758B928463946224605F05FF8E8B95C
:105F00000120B040020601D51648EFE7830501D510
:105F10001548EBE7B9F1000F03D0FCF712FC13486A
:105F200004E040EA0800CAF808001148FCF73AF912
:105F300039461048BDE8F04700F06FBE0136D0E7A3
:105F4000A410002038E30008E8D200080CE00008A4
:105F50007FE60008CCE400084BE30008E4D2000828
:105F600060E3000877E3000889E300089DE3000888
:105F7000A7E3000869E0000813B5062204463B21A8
:105F800068206B4601F048FAA0B19DF800209DF80A
:105F9000013043EA022323809DF802209DF803305C
:105FA00043EA022363809DF804209DF8053043EA0C
:105FB0000223A38002B010BD13B50622044643217C
:105FC00068206B4601F028FAA0B19DF800209DF8EA
:105FD000013043EA022323809DF802209DF803301C
:105FE00043EA022363809DF804209DF8053043EACC
:105FF0000223A38002B010BD2DE9F04F87B099466F
:106000000746884615469DF840B0FEF7CDFE02AE25
:106010000446034600F1100E18685968324603C260
:10602000083373451646F7D1237B0BB903950495C6
:10603000384602A900F0CCFE044608B9002031E041
:106040004368586828B1384602A92246FBF70CFE7F
:10605000F2E7A36894F800A01E781EB9CDF800B04E
:10606000124804E0012E1DD11148CDF800B04B4676
:1060700041462A46FFF79CFD03460028DED00D4A24
:10608000067102EB8A02C2F80004626850600A4896
:1060900042689A4204D002690C309A4218BF00202C
:1060A0004772184607B0BDE8F08F00BF00380140C6
:1060B00000440040A80A00201000002013B5244B23
:1060C0004000C0B283F8080402ACD3F8180483F887
:1060D000091404F8012D0021012283F80A24C3F8D1
:1060E0000C4483F80B14C3F8104483F8142483F889
:1060F000152483F8161448B38288920515D40288B3
:10610000D4050DD447F230520188890502D5013AF1
:10611000FAD113E092B1028892B242F48072028006
:10612000828892B242F44072828047F2305293F8F1
:10613000151411B1013AFAD100E012B901F05CF97D
:1061400004E0034B93F8160480F0010002B010BD88
:10615000A80A002010B5174C23681BB1FEF712FCEB
:10616000002323606B2180226820FFF7A7FF6420B3
:10617000FBF717FF192100226820FFF79FFF6B2113
:1061800003226820FFF79AFF372102226820FFF7D9
:1061900095FF094B1A211A786820FFF78FFF1B2102
:1061A00018226820FFF78AFFBDE8104068201C21F4
:1061B000102283E74C0500203D00002037B5062261
:1061C000044603216B461E2001F026F99DF801309C
:1061D0009DF80000154D43EA002000B201F064FF75
:1061E000296801F0B5FF02F079F99DF803302080AD
:1061F0009DF8020043EA002000B201F055FFA968B3
:1062000001F0A6FF02F06AF99DF80530A0809DF824
:10621000040043EA002000B201F046FF696801F083
:1062200097FF02F05BF9608003B030BD40000020B2
:1062300007B52320FBF7B5FE6820752101220DF17B
:10624000070301F0E9F828B19DF80700B0F16803F1
:106250005842584103B05DF804FB00BFF8B507464B
:1062600004F0A4FE044638B91A4B1B485A791B4B5C
:10627000013A53F8221028E038461949224604F022
:106280009DFE60B91748FBF78DFF174C54F8041FAB
:1062900019B1164800F0C1FCF8E7154805E00025E3
:1062A0000E4B53F8256026B91248BDE8F840FBF7BD
:1062B00079BF38463146224604F080FE0135002879
:1062C000EED1044B0C485D713146BDE8F84000F05A
:1062D000A4BC00BFA410002000E60008DCD1000828
:1062E000CCE4000814E60008D8D100080CE000084F
:1062F0007FE6000827E600083CE6000837B58288FC
:106300000446836810060D4606D529494FF4DA7015
:1063100091F86C1600FB0133D10504D525490A20FC
:10632000097800FB013302F03F02042A12D006D89C
:10633000012A0DD0022A2FD193F900102DE0102A46
:106340000AD0202A0AD0082A26D1B3F9001024E066
:10635000197822E0198820E019681EE0694618685B
:10636000FEF7A8FD0146144800F057FCF5B1E068BF
:1063700001F09AFE6946FEF79DFD01460F4800F0C8
:106380004CFC206901F090FE6946FEF793FD014642
:106390000A4800F042FC09E00021094800F03DFCF9
:1063A00025B10848E168226900F037FC03B030BD30
:1063B000A4100020A808002017E0000816E000083C
:1063C00052E600084EE600082DE9F0410024074699
:1063D0002546104B3946E65804EB0308304604F0D6
:1063E00021FE58B10C48314600F017FC4046002110
:1063F000FFF784FF094800F010FC01351434B4F5B0
:10640000166FE6D125B90648BDE8F041FBF7CABED4
:10641000BDE8F08138D40008ADE800087FE6000848
:1064200055E600082DE9F74F044604F0BFFD054688
:1064300020B1012818D123782A2B15D15548FBF714
:10644000B1FE0024544B5548E618E15800F0E5FB36
:1064500030462946FFF752FF14345148FBF7A2FE9D
:10646000B4F5166FEED192E020463D2104F091FD87
:10647000002800F08780034613F8012C202A01D160
:10648000013BF9E7451C2846C4EB030A04F0E3FD91
:1064900083462846FCF728F8002605461423734354
:1064A000DFF8F49053F8097003EB0908384604F05C
:1064B0007DFD03461A4620463946019304F07EFDD1
:1064C000019B002855D15FFA8AF29A4251D1D8F83F
:1064D0000C0001F0E9FD0146284601F0EBFF002821
:1064E00045D0D8F8100001F0DFFD0146284601F044
:1064F000D7FF00283BD0B8F804309B064FF01403B8
:1065000003FB0696B28858BF5D4614062946B36859
:1065100006D524484FF4DA7490F86C0604FB003377
:10652000D00504D520480A24007804FB003302F08B
:106530003F02042A0BD004D8013A012A0CD8197062
:106540000AE0102A05D0202A05D0082A04D1198093
:1065500002E0196000E01D603946144800F05DFB60
:106560003046002103B0BDE8F04FFFF7C7BE10482A
:1065700003E00136782E91D10E4803B0BDE8F04F0C
:10658000FBF710BE204603B0BDE8F04F1CE703B098
:10659000BDE8F08F6DE6000838D40008ADE80008CB
:1065A0007FE60008A4100020A808002082E600086A
:1065B0008DE6000855E600087FB5044604F0F6FCB9
:1065C000082824D100231F49E25C09681144497856
:1065D00001F00301022908BF203AE2540133082BDD
:1065E000F1D10025665D1848314604F0D2FC28B18F
:1065F00001356019314604F0CCFC18B11348FBF7A3
:10660000D1FD1CE0082DEDD12046FEF7B5FB10486A
:10661000FBF7C8FD00230F4A04A91A4492F8102181
:106620000A440949595C0133082B02F80C1CF2D1C9
:106630000023094801A98DF80C3000F0EEFA04B0EF
:1066400070BD00BF8800002015E30008ADE600081B
:10665000CDE60008A410002069E000082DE9F04311
:1066600089B0044604F0A2FCC6B2002E6CD18B485F
:10667000FBF798FD8A4C2069002101F0FDFE40BB2C
:1066800001368848314600F0C8FA206904A9FEF7AF
:1066900011FC0146844800F0C0FA606904A9FEF7C5
:1066A00009FC0146804800F0B8FAA06904A9FEF789
:1066B00001FC01467C4800F0B0FAE06904A9FEF74D
:1066C000F9FB0146794800F0A8FA0C2E04F11004F9
:1066D000D1D10025764C2F462B464FF00008B0450F
:1066E00004F1100415DA184654F8101C01F028FCC7
:1066F00054F80C1C8146284601F022FC54F8081C72
:106700000546384601F01CFC08F101084B460746D7
:10671000E5E76848019302950397FBF743FD0024E2
:1067200001ABE058644920F0004001F0CDFE634B1E
:10673000634A0434002814BF10461846FBF732FDA4
:106740000C2CEDD15F4891E020465F49052204F012
:1067500035FC38B9524B002203441030C0281A616E
:10676000F8D197E020465949042204F027FC064658
:106770002046002E40D1202104F00BFC002800F020
:106780008980451C284604F011FC34468046504B55
:1067900053F824600EB94F4868E0284631465FFA46
:1067A00088F204F00BFC671C20BB3D4B0021C21893
:1067B0001030C02811619C46F7D1474B002403EBF1
:1067C000C702D2F804E09846BEF1000F04D1434856
:1067D000314600F022FA55E018F837309C42F6DADC
:1067E00023010CEB0305103573440FCB013485E80E
:1067F0000F00F1E73C46CAE704F02DFC461E0B2EC5
:10680000074643DC2046202104F0C3FB054640B187
:10681000451C2846FBF768FE214B3F01D851012457
:1068200000E004462846202104F0B3FB054640B1B1
:10683000451C2846FBF758FE194B013403EB0613A1
:1068400058612846202104F0A4FB054640B1451CB0
:106850002846FBF749FE124B013403EB06139861FF
:106860002846202104F095FB18B91D48FBF79AFC37
:1068700010E00130FBF738FE094B032C03EB061642
:10688000F061F2D11748FFF7E9FE03E016480C214A
:1068900000F0C3F909B0BDE8F08300BFEAE60008E4
:1068A000A410002015E700081BE7000869E00008B5
:1068B000B81000201FE700080AD7233CE6E60008CE
:1068C000E2E600087FE600082EE7000834E700084B
:1068D000DCD1000827E60008C0CB000839E7000833
:1068E00049E70008D5E1000883E7000870B50446D1
:1068F00004F05CFB08B9204830E020461F4904F052
:10690000CFFB00242646254678B12CB1012C06D1B8
:1069100004F0A1FB064602E004F09DFB0546174982
:106920000020013404F0BCFBEEE70B2D05D9BDE8D7
:10693000704013480C2100F070B9012C08DC114B99
:10694000294633F915201048BDE8704000F065B9BC
:10695000A6F57A73B3F57A7F04D90C48BDE8704088
:1069600000F05BB90A482946324600F056F9054B5B
:1069700023F8156070BD00BFABE70008A4E1000874
:10698000E5E70008DC0400200BE8000823E8000825
:1069900045E80008F0B585B0074604F007FBC0B233
:1069A000E0B90446324B04F11C021B68192003EBCA
:1069B0008203591D8D785A79454305F561759B7998
:1069C0000095C978484300F5617001902146294837
:1069D000013400F022F9282CE4D146E0384604F0D6
:1069E0003AFB27283DDC224B00F11C061B68781C73
:1069F00003EB8606202100238DF80F3004F0C9FA3E
:106A0000751D044658B1441C204604F024FB15288B
:106A100005D870719DF80F3001338DF80F30204686
:106A2000202104F0B6FA044658B1441C204604F074
:106A300012FB0D2805D89DF80F30687001338DF8D2
:106A40000F302046A91C0DF10F02FDF777FD9DF8D0
:106A50000F30042B09D028460021042204F065FAE7
:106A600003E00548282100F0D8F805B0F0BD00BFCC
:106A7000340200205EE8000873E8000870B586B0B4
:106A8000054604F093FAC0B208BB044606236343EC
:106A9000444A03F58873126819201344591D4D7830
:106AA0009A7A454305F561755B7900958D78684361
:106AB00000F561700190C878029009793A48039115
:106AC0002146013400F0A9F80C2CDFD168E02846FB
:106AD00004F0C1FA0B285FDC06267043314B00F549
:106AE00088701E68202106440023681C8DF817302A
:106AF00004F04FFA741D054658B1451C284604F0B1
:106B0000AAFA032805D89DF81730607101338DF873
:106B100017302846202104F03CFA054658B1451CA0
:106B2000284604F098FA0D2805D870719DF81730A2
:106B300001338DF817302846611C0DF11702FDF75F
:106B4000FDFC202104F025FA054658B1451C2846D5
:106B500004F081FA0C2805D89DF81730E070013355
:106B60008DF817302846202104F013FA50B1013077
:106B700004F071FA0D2805D89DF817302071013303
:106B80008DF817309DF81730062B09D020460021CC
:106B9000062204F0CAF903E004480C2100F03DF895
:106BA00006B070BD3402002089E8000873E80008D0
:106BB00070B5064600240A4BE518AA8816420AD08A
:106BC000E158084800F029F828460021FFF796FB15
:106BD0000548FBF7E7FA1434B4F5166FEBD170BD36
:106BE00038D40008A9E800087FE60008436A8269F3
:106BF000D154436A02690133934228BF00234362A0
:106C0000436B23B11B68DB0706D4FEF7EBBE036DB5
:106C1000DA6842F08002DA6070470FB42DE9F04F75
:106C2000684A89B012AB1668674A53F8045B176864
:106C300004939B462978002900F0B880252902D0CA
:106C400001353046B0E06C78302C03D002354FF07F
:106C5000000903E0AC784FF001090335A4F13003DB
:106C6000092B4FF000081AD8A4F13003DAB2092A30
:106C700007D80A2B13DC0A2202FB083815F8014B4F
:106C8000F2E7A4F16103052B02D8A4F15703F0E762
:106C9000A4F14103052B02D8A4F13703E9E76C2CDA
:106CA00003BF2C78012201350022632C66D006D860
:106CB000252C77D0582C3FD0002C77D0BAE7732CF6
:106CC00063D002D8642C11D0B4E7752C02D0782C94
:106CD00032D0AFE70BF1040A05ACDBF800000A2163
:106CE00012B10022234613E0234620E00BF1040AF0
:106CF00005ACDBF8000072B1002806DA2D238DF810
:106D0000143040420DF1150300E023460A21002211
:106D1000FBF7A8FC0DE0002806DA2D238DF81430CF
:106D200040420DF1150300E023460A210022FBF743
:106D300071FCD34600941AE00BF1040303930DF1A8
:106D4000140ADBF80000102132B1583C6242624163
:106D50005346FBF787FC06E0B4F158035A425A4108
:106D60005346FBF757FCDDF80CB0CDF800A03046D9
:106D7000394642464B46FBF7B1FC5BE730469BF891
:106D800000100BF10404B8470AE0DBF8003030468D
:106D900000933946424600230BF10404FBF79EFCA6
:106DA000A34647E730462146B84743E7074B1868F4
:106DB00003681B6998470028F8D009B0BDE8F04F78
:106DC00004B070470C0500200805002008090020C9
:106DD000F0B5142285B007460E461648002104F08F
:106DE000A4F8154B00241A7AE0B2013412B1511EF6
:106DF0000A40F9E71C7DD1B2013214B1611E0C408A
:106E0000F9E7421A002A0DDD93E8070001AD85E895
:106E100007000A4C94E8070083E8070095E807009C
:106E200084E80700034A3846314605B0BDE8F04023
:106E3000FAF71ABFC40E0020100000201C0000202A
:106E40000E4B1A78562A16D15A88B2F5D26F12D143
:106E50001A79BE2A0FD193F88C260020EF2A0CD184
:106E600013F8012B5040064A9342F9D1D0F10100AA
:106E700038BF0020704700207047704700F80008B6
:106E800090FE00084A4B56222DE9F3411A704FF448
:106E9000D2625A80BE221A71EF2283F88C26002219
:106EA00083F88D2611461E46B35C0132B2F5D26FCF
:106EB00081EA0301F8D13E4B3E4A83F88D163E4BE2
:106EC00004275A6002F188325A600020013F17F00F
:106ED000FF075DD0384B3422384CDA60C4F3090325
:106EE0007BB1331903F17843A3F57843D3F80080DD
:106EF0004FF4005000230193FEF70AFA0428E5D16D
:106F00001BE04FF43020FEF703FA0428DED12A4DAF
:106F10004FF430202B6943F002032B616C612B6925
:106F200043F040032B61FEF7F3F92A6941F6FD7344
:106F3000134004282B61D4D0C8E71F4D4FF40050F4
:106F40002B6943F001032B611FFA88F32380FEF7BE
:106F5000DFF9042812D1A31C0193019B4FEA1848C2
:106F6000A3F800804FF40050FEF7D2F92B6941F6E8
:106F7000FE721A4004282A6106D0A7E72B6941F661
:106F8000FE721A402A61A1E70D4B04349C42A5D140
:106F9000094B04281A6942F080021A6102D1FFF7F6
:106FA0004FFF10B90A20FBF745F802B0BDE8F081A9
:106FB000A4100020230167450020024000F80008CB
:106FC00090FE000808B50448FBF7ECF8FFF75AFFFD
:106FD000BDE80840FEF7EBBCB3E800083F4A2DE9E6
:106FE000F84F916840F201130B4040F201118B42BF
:106FF00093460AD13A4B1A7D93F815905A75B9EB1E
:10700000020918BF4FF0010901E04FF001094FF0EC
:107010000008344B5FFA88F41B78A3425CD9324BEA
:10702000324E1B68324F23B93B685B8926F8143017
:107030004FE03A68072C94BF12F804A0A2462948F2
:1070400051469847DBF808300546DB0509D5B9F10C
:10705000000F06D0274B50461B6829461B68DB698A
:107060009847A5F2EE2240F2DC5392B29A4288BFD2
:107070003B68DBF8082088BF5D8942F201031340BA
:107080002BB31D4B1978164B01F0030202EB84025F
:1070900093F8760003EB4202D5821A4620B9032901
:1070A00015D9012183F8761002EBC403198BDD8A10
:1070B00002EB44020D44598B9B8B0D441D44ADB231
:1070C000A2F8785004232DB295FBF3F5ADB226F863
:1070D000145008F101089CE7BDE8F88FA4100020C7
:1070E000C40E0020D5040020BC070020620300204D
:1070F000FC0000200002002050080020094B30B5A1
:107100009D68094B05F480551868084B1C680023DE
:107110000DB1828800E0A28805495A520233182B2B
:10712000F6D130BDA4100020D4080020D8080020DB
:10713000DC04002008B50848FBF734F8074A0023B0
:107140001370074A1360074A1370FFF7D7FFBDE8B3
:107150000840FEF72CBC00BFBAE800081009002068
:107160000C0900205B170020F8B50024204BE0B28A
:107170001F78B8420CD21F4B33F810101E4B53F837
:1071800020301BB10B2801D8DB6898470134EDE7AC
:107190001A4B9B685B032AD50025194E2B46EAB291
:1071A000BA4224D2726854689C4218D02046FBF739
:1071B00014FBEFF31283502282F3128811494FF02F
:1071C000280CA28C0CFB001092B201324262A28AFF
:1071D000DBB292B242F00102A28283F3118856F828
:1071E000043F00221B6801351A802346D7E7F8BD0B
:1071F000341700203617002090060020A41000202D
:107200008C060020580F00202DE9F04F1421012892
:1072100034BF0646012601FB06F3DFF8D8A1DFF8EC
:10722000C0B10AEB03025AF803301069CBF8003002
:10723000694B15891E70694BB2F80A80DC6989B008
:107240002043546848EA0507D86102222761204696
:107250008DF80E1003A90193ADF80C708DF80F2076
:10726000FBF7F2FA019B4FF008099B46A268154212
:1072700003D10A20FAF78AFEF8E70A206561FAF7D7
:1072800085FE25610A20FAF781FEB9F10109EDD1E9
:10729000C4F814800A20FAF779FE65610A20FAF72B
:1072A00075FE25610A20FAF771FE0222C4F81080EB
:1072B00020468DF80F2003A91C228DF80E20ADF872
:1072C0000C70FBF7C1FA464B464A1C689442DBF847
:1072D000102008D142F40012CBF81020DBF8102067
:1072E00022F4001207E042F48002CBF81020DBF811
:1072F000102022F48002CBF81020A38803A823F4E6
:1073000040731B041B0CA38023889BB243F0010332
:107310002380A588FDF764FF25F03F050599324AD3
:107320002D04B1FBF2F22D0C1543ADB2A5802388DC
:10733000012523F001031B041B0C23802B4B03A806
:10734000B1FBF3F34FF496714A439BB24FF47A7159
:10735000002B92FBF1F208BF0123013292B243F4F9
:1073600000432284A38323889BB243F0010323803C
:10737000238823F4816323F002031B041B0C238066
:107380004FF480432381142303FB06A6737B002460
:107390008DF80C308DF80D408DF80E408DF80F50A3
:1073A000FDF72AFB337B9DF80F208DF80C308DF80C
:1073B0000D408DF80E401AB103A8FDF71DFB07E044
:1073C000590903F01F039D40094A203142F821501A
:1073D00009B0BDE8F08F00BF540F0020001002403C
:1073E000C00E00200054004040420F00804F1200A9
:1073F00000E100E010D4000808B5054B1A880132FE
:1074000092B21A80034B1878FFF7FEFE002008BDE9
:10741000BC040020540F002010B54000204CC0B226
:1074200020702048204C017020480021017001206C
:1074300020701F4C23601F4C23601F4B1A701F4B82
:107440001F4A107019701F490868194630B38388A5
:107450009C0515D40388DB050DD447F2305304880E
:10746000A40502D5013BFAD112E08BB103889BB28F
:1074700043F48073038083889BB243F4407383801A
:1074800047F23053107810B1013BFBD100E013B943
:10749000BDE81040B0E7087880F0010010BD00BFE3
:1074A000B00E0020B10E0020B30E0020B20E00205E
:1074B000B80E0020B40E0020BC0E0020BE0E00202E
:1074C000BD0E0020C00E0020244A13B513681446D8
:1074D000998A89B20191019911F4706F02D0204A02
:1074E00001211170019A12F4E06F2AD01A8B9A8848
:1074F00022F480621204120C9A80019A910520D421
:107500001A8892051DD41A88D0050FD51A88D1057E
:10751000FCD41A8892B242F400721A801A8892053A
:10752000FCD4104B1878FFF76FFE0AE01A8892B26D
:1075300042F400721A809A8822F440721204120CEB
:107540009A802268938A23F470631B041B0C938235
:10755000054B00221A7002B010BD00BFC00E002003
:10756000BE0E0020540F0020BD0E0020014802492D
:10757000FBF7F0B800080040D00F00200148024996
:10758000FBF7E8B800040040A80F00204FF080404F
:107590000149FBF7DFB800BF800F00200148024916
:1075A000FBF7D8B8002C0140580F002001480249D1
:1075B000FBF7D0B8002C0140580F002070B5214CCB
:1075C000D4F8F0201588ADB2A90618D5D4F8CC307F
:1075D0001BB1908880B2984711E0D4F8BC10928813
:1075E000D4F8B4004E1CD2B2C4F8BC604254D4F8F3
:1075F000BC10D4F8AC20914228BFC4F8BC302B0694
:107600001ED5D4F8C820D4F8C4100E4B8A4211D02D
:10761000511CD3F8B840C3F8C810A25CD3F8F000EE
:10762000D2B28280D3F8B020914209D30022C3F8AD
:10763000C82070BDD3F8F030DA6822F08002DA603A
:1076400070BD00BF580F00200F4BD3F844211188A4
:10765000090618D5D3F81C11D3F8180181420ED0B1
:10766000D3F80C01405C0131C0B29080D3F8042102
:10767000B1FBF2F002FB1011C3F81C117047D36884
:1076800023F08003D3607047580F00200C480D4B47
:107690004FF400525A60D0F828214FF6FE7311685B
:1076A0000B401360D0F81821D0F81C319A4202D058
:1076B000F430FEF797B9012380F83831704700BFE6
:1076C000580F002000000240FFF7FEBEFFF7FCBE8F
:1076D000FCF7EABFFCF7E8BF0F4B1A6842F0010263
:1076E0001A6059680D4A0A405A601A6822F084727A
:1076F00022F480321A601A6822F480221A605A68D2
:1077000022F4FE025A604FF41F029A60044B4FF0BD
:1077100000629A60704700BF001002400000FFF84E
:1077200000ED00E0024B1A6801321A60704700BF9A
:10773000A010002008B5084BB3F8D80093F89426A1
:107740000023D9B2914204D2044921F81300013335
:10775000F7E7FFF709FDFEE7A0100020361700202D
:1077600081F0004102E000BF83F0004330B54FEAF2
:1077700041044FEA430594EA050F08BF90EA020F5F
:107780001FBF54EA000C55EA020C7FEA645C7FEAF2
:10779000655C00F0E2804FEA5454D4EB5555B8BF15
:1077A0006D420CDD2C4480EA020281EA030382EA86
:1077B000000083EA010180EA020281EA0303362D18
:1077C00088BF30BD11F0004F4FEA01314FF4801CEB
:1077D0004CEA113102D0404261EB410113F0004FFD
:1077E0004FEA03334CEA133302D0524263EB4303B4
:1077F00094EA050F00F0A780A4F10104D5F1200E52
:107800000DDB02FA0EFC22FA05F2801841F10001AC
:1078100003FA0EF2801843FA05F359410EE0A5F180
:1078200020050EF1200E012A03FA0EFC28BF4CF0B1
:10783000020C43FA05F3C01851EBE37101F0004567
:1078400007D54FF0000EDCF1000C7EEB00006EEB74
:107850000101B1F5801F1BD3B1F5001F0CD34908FE
:107860005FEA30004FEA3C0C04F101044FEA445255
:1078700012F5800F80F09A80BCF1004F08BF5FEADC
:10788000500C50F1000041EB045141EA050130BDBC
:107890005FEA4C0C404141EB010111F4801FA4F15F
:1078A0000104E9D191F0000F04BF01460020B1FAB4
:1078B00081F308BF2033A3F10B03B3F120020CDAEC
:1078C0000C3208DD02F1140CC2F10C0201FA0CF0CA
:1078D00021FA02F10CE002F11402D8BFC2F1200C2F
:1078E00001FA02F120FA0CFCDCBF41EA0C019040E5
:1078F000E41AA2BF01EB0451294330BD6FEA04042E
:107900001F3C1CDA0C340EDC04F11404C4F1200218
:1079100020FA04F001FA02F340EA030021FA04F32A
:1079200045EA030130BDC4F10C04C4F1200220FA81
:1079300002F001FA04F340EA0300294630BD21FABF
:1079400004F0294630BD94F0000F83F4801306BF85
:1079500081F480110134013D4EE77FEA645C18BF79
:107960007FEA655C29D094EA050F08BF90EA020F10
:1079700005D054EA000C04BF1946104630BD91EA08
:10798000030F1EBF0021002030BD5FEA545C05D10B
:107990004000494128BF41F0004130BD14F580044A
:1079A0003CBF01F5801130BD01F0004545F0FE41BE
:1079B00041F470014FF0000030BD7FEA645C1ABFF3
:1079C000194610467FEA655C1CBF0B46024650EA2A
:1079D000013406BF52EA033591EA030F41F4002156
:1079E00030BD00BF90F0000F04BF0021704730B5DC
:1079F0004FF4806404F132044FF000054FF00001B1
:107A000050E700BF90F0000F04BF0021704730B571
:107A10004FF4806404F1320410F0004548BF404246
:107A20004FF000013EE700BF42004FEAE2014FEA9B
:107A300031014FEA02701FBF12F07F4393F07F4F76
:107A400081F06051704792F0000F14BF93F07F4FA8
:107A5000704730B54FF4607401F0004521F00041EB
:107A600020E700BF50EA010208BF704730B54FF071
:107A700000050AE050EA010208BF704730B511F076
:107A8000004502D5404261EB41014FF4806404F1AE
:107A900032045FEA915C3FF4DCAE4FF003025FEA30
:107AA000DC0C18BF03325FEADC0C18BF033202EBB8
:107AB000DC02C2F1200300FA03FC20FA02F001FA12
:107AC00003FE40EA0E0021FA02F11444C1E600BFB1
:107AD00070B54FF0FF0C4CF4E06C1CEA11541DBF64
:107AE0001CEA135594EA0C0F95EA0C0F00F0DEF82F
:107AF0002C4481EA030621EA4C5123EA4C5350EA14
:107B0000013518BF52EA033541F4801143F4801364
:107B100038D0A0FB02CE4FF00005E1FB02E506F0F5
:107B20000042E0FB03E54FF00006E1FB03569CF04A
:107B3000000F18BF4EF0010EA4F1FF04B6F5007F50
:107B400064F5407404D25FEA4E0E6D4146EB0606C2
:107B500042EAC62141EA55514FEAC52040EA5E504B
:107B60004FEACE2EB4F1FD0C88BFBCF5E06F1ED8F5
:107B7000BEF1004F08BF5FEA500E50F1000041EB2C
:107B8000045170BD06F0004646EA010140EA0200D9
:107B900081EA0301B4EB5C04C2BFD4EB0C0541EAFB
:107BA000045170BD41F480114FF0000E013C00F310
:107BB000AB8014F1360FDEBF002001F0004170BD34
:107BC000C4F10004203C35DA0C341BDC04F114044D
:107BD000C4F1200500FA05F320FA04F001FA05F2D9
:107BE00040EA020001F0004221F0004110EBD370A6
:107BF00021FA04F642EB06015EEA430E08BF20EAD2
:107C0000D37070BDC4F10C04C4F1200500FA04F374
:107C100020FA05F001FA04F240EA020001F0004106
:107C200010EBD37041F100015EEA430E08BF20EA79
:107C3000D37070BDC4F1200500FA05F24EEA020EC1
:107C400020FA04F301FA05F243EA020321FA04F0F0
:107C500001F0004121FA04F220EA020000EBD370A7
:107C60005EEA430E08BF20EAD37070BD94F0000FA7
:107C70000FD101F00046400041EB010111F4801FDB
:107C800008BF013CF7D041EA060195F0000F18BF8C
:107C9000704703F00046520043EB030313F4801FC8
:107CA00008BF013DF7D043EA0603704794EA0C0F82
:107CB0000CEA135518BF95EA0C0F0CD050EA410698
:107CC00018BF52EA4306D1D181EA030101F0004115
:107CD0004FF0000070BD50EA410606BF104619463D
:107CE00052EA430619D094EA0C0F02D150EA013649
:107CF00013D195EA0C0F05D152EA03361CBF10468A
:107D000019460AD181EA030101F0004141F0FE4128
:107D100041F470014FF0000070BD41F0FE4141F4AC
:107D2000780170BD70B54FF0FF0C4CF4E06C1CEAAC
:107D300011541DBF1CEA135594EA0C0F95EA0C0F61
:107D400000F0A7F8A4EB050481EA030E52EA03351C
:107D50004FEA013100F088804FEA03334FF080553D
:107D600045EA131343EA12634FEA022245EA11156A
:107D700045EA10654FEA00260EF000419D4208BF1B
:107D8000964244F1FD0404F5407402D25B084FEAC8
:107D90003202B61A65EB03055B084FEA32024FF474
:107DA00080104FF4002CB6EB020E75EB030E22BFD1
:107DB000B61A754640EA0C005B084FEA3202B6EB91
:107DC000020E75EB030E22BFB61A754640EA5C0040
:107DD0005B084FEA3202B6EB020E75EB030E22BFD0
:107DE000B61A754640EA9C005B084FEA3202B6EBD1
:107DF000020E75EB030E22BFB61A754640EADC0090
:107E000055EA060E18D04FEA051545EA16754FEAF1
:107E100006164FEAC30343EA52734FEAC2025FEA0F
:107E20001C1CC0D111F4801F0BD141EA00014FF09E
:107E300000004FF0004CB6E711F4801F04BF01436F
:107E40000020B4F1FD0C88BFBCF5E06F3FF6AFAE8B
:107E5000B5EB030C04BFB6EB020C5FEA500C50F11B
:107E6000000041EB045170BD0EF0004E4EEA11319E
:107E700014EB5C04C2BFD4EB0C0541EA045170BDA5
:107E800041F480114FF0000E013C90E645EA060EE9
:107E90008DE60CEA135594EA0C0F08BF95EA0C0F17
:107EA0003FF43BAF94EA0C0F0AD150EA01347FF45F
:107EB00034AF95EA0C0F7FF425AF104619462CE736
:107EC00095EA0C0F06D152EA03353FF4FDAE104699
:107ED000194622E750EA410618BF52EA43067FF4EA
:107EE000C5AE50EA41047FF40DAF52EA43057FF47A
:107EF000EBAE12E74A0011D212F5001211D20DD5E5
:107F00006FF47873B3EB62520ED44FEAC12343F09F
:107F1000004343EA505323FA02F070474FF0000049
:107F2000704750EA013002D14FF0FF3070474FF0F8
:107F30000000704780F0004002E000BF81F0004187
:107F400042001FBF5FEA410392EA030F7FEA226CFF
:107F50007FEA236C6AD04FEA1262D2EB1363C1BF8F
:107F6000D218414048404140B8BF5B42192B88BFFE
:107F7000704710F0004F40F4000020F07F4018BF21
:107F8000404211F0004F41F4000121F07F4118BF41
:107F9000494292EA030F3FD0A2F1010241FA03FCE9
:107FA00010EB0C00C3F1200301FA03F100F00043D1
:107FB00002D5494260EB4000B0F5000F13D3B0F199
:107FC000807F06D340084FEA310102F10102FE2A08
:107FD00051D2B1F1004F40EBC25008BF20F0010078
:107FE00040EA03007047490040EB000010F4000F26
:107FF000A2F10102EDD1B0FA80FCACF1080CB2EBB9
:108000000C0200FA0CF0AABF00EBC2505242184317
:10801000BCBFD0401843704792F0000F81F40001BC
:1080200006BF80F400000132013BB5E74FEA41038F
:108030007FEA226C18BF7FEA236C21D092EA030FFB
:1080400004D092F0000F08BF0846704790EA010F75
:108050001CBF0020704712F07F4F04D1400028BFA2
:1080600040F00040704712F100723CBF00F5000084
:10807000704700F0004343F0FE4040F400007047BA
:108080007FEA226216BF08467FEA23630146420266
:1080900006BF5FEA412390EA010F40F48000704779
:1080A0004FF0000304E000BF10F0004348BF40421F
:1080B0005FEA000C08BF704743F0964301464FF05B
:1080C00000001CE050EA010208BF70474FF00003B7
:1080D0000AE000BF50EA010208BF704711F00043F8
:1080E00002D5404261EB41015FEA010C02BF8446C8
:1080F0000146002043F0B64308BFA3F18053A3F527
:108100000003BCFA8CF2083AA3EBC25310DB01FA6D
:1081100002FC634400FA02FCC2F12002BCF1004FF1
:1081200020FA02F243EB020008BF20F00100704782
:1081300002F1200201FA02FCC2F1200250EA4C00D6
:1081400021FA02F243EB020008BF20EADC7070471C
:108150004FF0FF0C1CEAD0521EBF1CEAD15392EA2A
:108160000C0F93EA0C0F6FD01A4480EA010C400206
:1081700018BF5FEA41211ED04FF0006343EA501060
:1081800043EA5111A0FB01310CF00040B1F5000FA2
:108190003EBF490041EAD3715B0040EA010062F151
:1081A0007F02FD2A1DD8B3F1004F40EBC25008BF3B
:1081B00020F00100704790F0000F0CF0004C08BF59
:1081C00049024CEA502040EA51207F3AC2BFD2F126
:1081D000FF0340EAC250704740F400004FF0000334
:1081E000013A5DDC12F1190FDCBF00F0004070476E
:1081F000C2F10002410021FA02F1C2F1200200FAAC
:1082000002FC5FEA310040F1000053EA4C0308BF72
:1082100020EADC70704792F0000F00F0004C02BFC3
:10822000400010F4000F013AF9D040EA0C0093F03E
:10823000000F01F0004C02BF490011F4000F013B98
:10824000F9D041EA0C018FE70CEAD15392EA0C0F06
:1082500018BF93EA0C0F0AD030F0004C18BF31F071
:10826000004CD8D180EA010000F00040704790F047
:10827000000F17BF90F0004F084691F0000F91F0EB
:10828000004F14D092EA0C0F01D142020FD193EAB1
:108290000C0F03D14B0218BF084608D180EA010039
:1082A00000F0004040F0FE4040F40000704740F015
:1082B000FE4040F4400070474FF0FF0C1CEAD052E3
:1082C0001EBF1CEAD15392EA0C0F93EA0C0F69D03F
:1082D000A2EB030280EA010C49024FEA402037D0AA
:1082E0004FF0805343EA111143EA10130CF00040A1
:1082F0008B4238BF5B0042F17D024FF4000C8B4291
:1083000024BF5B1A40EA0C00B3EB510F24BFA3EB70
:10831000510340EA5C00B3EB910F24BFA3EB910340
:1083200040EA9C00B3EBD10F24BFA3EBD10340EA9A
:10833000DC001B0118BF5FEA1C1CE0D1FD2A3FF6E0
:1083400050AF8B4240EBC25008BF20F00100704795
:108350000CF0004C4CEA50207F32C2BFD2F1FF0338
:1083600040EAC250704740F400004FF00003013A69
:1083700037E792F0000F00F0004C02BF400010F40D
:10838000000F013AF9D040EA0C0093F0000F01F021
:10839000004C02BF490011F4000F013BF9D041EA43
:1083A0000C0195E70CEAD15392EA0C0F08D1420276
:1083B0007FF47DAF93EA0C0F7FF470AF084676E749
:1083C00093EA0C0F04D14B023FF44CAF08466EE722
:1083D00030F0004C18BF31F0004CCAD130F00042F0
:1083E0007FF45CAF31F000437FF43CAF5FE700BF48
:1083F0004FF0FF3C06E000BF4FF0010C02E000BF71
:108400004FF0010C4DF804CD4FEA40024FEA410312
:108410007FEA226C18BF7FEA236C11D001B052EAC8
:10842000530C18BF90EA010F58BFB2EB030088BF8E
:10843000C81738BF6FEAE17018BF40F001007047FD
:108440007FEA226C02D15FEA402C05D17FEA236CDF
:10845000E4D15FEA412CE1D05DF8040B704700BF26
:10846000844608466146FFE70FB5FFF7C9FF0028BD
:1084700048BF10F1000F0FBD4DF808EDFFF7F4FFF6
:108480000CBF012000205DF808FB00BF4DF808ED8F
:10849000FFF7EAFF34BF012000205DF808FB00BFB2
:1084A0004DF808EDFFF7E0FF94BF012000205DF8D4
:1084B00008FB00BF4DF808EDFFF7D2FF94BF012085
:1084C00000205DF808FB00BF4DF808EDFFF7C8FF7E
:1084D00034BF012000205DF808FB00BF4FEA4002D6
:1084E000B2F1FE4F0FD34FF09E03B3EB12620DD9E2
:1084F0004FEA002343F0004310F0004F23FA02F04C
:1085000018BF404270474FF00000704712F1610FF2
:1085100001D1420205D110F0004008BF6FF00040C9
:1085200070474FF00000704742000ED2B2F1FE4F8C
:108530000BD34FF09E03B3EB126209D44FEA002332
:1085400043F0004323FA02F070474FF000007047F9
:1085500012F1610F01D1420202D14FF0FF3070479A
:108560004FF00000704700BF73B96AB9002908BF17
:108570000028BCBF00204FF00041C4BF6FF0004195
:108580004FF0FF3000F03CB882B0EC462DE90050CF
:1085900000F006F8DDF804E002B00CBC704700BF44
:1085A0002DE9704F089E14461D468046894600F00E
:1085B00029F804FB01F3A4FB00AB00FB0532934454
:1085C000B8EB0A0869EB0B09C6E90089BDE8708FB2
:1085D0002DE9704F089E14461D468046894600F0DE
:1085E00061F900FB05F5A0FB04AB04FB0154A344B7
:1085F000B8EB0A0869EB0B09C6E90089BDE8708F82
:10860000704700BF00292DE9F00FC0F2A1800024BF
:10861000002BC0F29880154606460F46002B3FD12E
:108620008A4258D9B2FA82F34BB1C3F1200201FA5F
:1086300003F720FA02F29D4000FA03F61743290CD3
:10864000B7FBF1F201FB1277A8B200FB02F34FEA8D
:10865000164C4CEA0747BB4209D97F1902F1FF3C8F
:1086600080F00581BB4240F20281023A2F44FF1A9A
:10867000B7FBF1F301FB137100FB03F0B6B246EA5E
:108680000141884208D9491903F1FF3780F0F18090
:10869000884240F2EE80023B43EA0242002303E0BC
:1086A0008B420AD900231A461046194614B140429B
:1086B00061EB4101BDE8F00F7047B3FA83F8B8F100
:1086C000000F40F088808B4202D3824200F2E280A9
:1086D00000230122E8E712B90123B3FBF2F5B5FA52
:1086E00085F2002A3AD17F1B280C1FFA85FC012352
:1086F000B7FBF0F100FB11770CFB01F24FEA1648D3
:1087000048EA0747BA4207D97F1901F1FF3802D278
:10871000BA4200F2C4804146BF1AB7FBF0F200FB38
:1087200012700CFB02FCB6B246EA0040844507D941
:10873000401902F1FF3702D2844500F2AE803A467A
:1087400042EA0142B0E7E443524263EB430362E78B
:10875000404261EB41014FF0FF3459E79540C2F1CF
:10876000200927FA09F126FA09F99740280CB1FBEC
:10877000F0F800FB18111FFA85FC0CFB08F349EA1E
:1087800007094FEA194747EA01418B4206FA02F608
:1087900008D9491908F1FF327AD28B4278D9A8F169
:1087A00002082944C91AB1FBF0F300FB13170CFBB4
:1087B00003F21FFA89F949EA0747BA4207D97F1934
:1087C00003F1FF3160D2BA425ED9023B2F44BF1A97
:1087D00043EA08438CE7C8F1200225FA02F103FAC4
:1087E00008FC27FA02F320FA02F207FA08F741EA36
:1087F0000C0C4FEA1C49B3FBF9F109FB11331FFACA
:108800008CFA0AFB01FB17433A0C42EA03439B45EF
:1088100005FA08F008D913EB0C0301F1FF3235D249
:108820009B4533D902396344CBEB0303B3FBF9F225
:1088300009FB12330AFB02FABFB247EA0347BA4503
:1088400008D917EB0C0702F1FF331BD2BA4519D92F
:10885000023A674442EA0145A5FB0001CAEB07075B
:108860008F424FF000030AD305D02A461CE7624628
:10887000FDE63B4610E706FA08F68642F5D26A1E88
:10888000002311E71A46E5E70B46A0E71146CBE7C0
:10889000904687E74346424606E7023A50E70239E8
:1088A0002F4439E72DE9F00F144605460E46002BFC
:1088B00043D18A4253D9B2FA82F757B1C7F12006A1
:1088C00020FA06F601FA07F302FA07F400FA07F5B0
:1088D0001E43210CB6FBF1F201FB1266A0B200FBB5
:1088E00002F32F0C47EA0646B34209D9361902F1C2
:1088F000FF3780F0FD80B34240F2FA80023A26440E
:10890000F61AB6FBF1F301FB136100FB03F0ADB205
:1089100045EA0141884208D9091903F1FF3680F080
:10892000E980884240F2E680023B43EA02420023AB
:1089300010461946BDE8F00F70478B424CD8B3FA89
:1089400083F6002E4FD18B4202D3824200F2DD80AB
:10895000BDE8F00F0023012210461946704712B9F6
:108960000124B4FBF2F4B4FA84F2002A40F08280CD
:10897000091B260CA7B20123B1FBF6F006FB101170
:1089800007FB00F24FEA154C4CEA01418A4207D935
:10899000091900F1FF3C02D28A4200F2C880604609
:1089A000891AB1FBF6F206FB121107FB02F7ADB212
:1089B00045EA0145AF4208D92C1902F1FF3180F098
:1089C0009B80A74240F29880023A42EA0042104659
:1089D0001946BDE8F00F704700231A4610461946A5
:1089E000BDE8F00F7047C6F1200522FA05F703FA3B
:1089F00006F421FA05F301FA06FB20FA05F53C43DB
:108A00004FEA1448B3FBF8FC08FB1C331FFA84F947
:108A100009FB0CFA45EA0B0B4FEA1B4545EA0343F9
:108A20009A4502FA06F204D91B190CF1FF356FD3EF
:108A3000AC46CAEB0303B3FBF8F508FB153309FB9F
:108A400005F91FFA8BFB4BEA0347B94504D93F19D7
:108A500005F1FF3362D31D4645EA0C4CACFB022303
:108A6000C9EB07079F424FF000054AD346D0624644
:108A70002B465DE79440C2F1200921FA09FC9140A0
:108A800020FA09F9260CBCFBF6F806FB18CCA7B2B5
:108A900007FB08F349EA01094FEA194141EA0C4C86
:108AA000634500FA02F509D91CEB040C08F1FF320A
:108AB0003BD2634539D9A8F10208A444C3EB0C0C9E
:108AC000BCFBF6F306FB13C107FB03F21FFA89F99F
:108AD00049EA01418A4207D9091903F1FF3022D23C
:108AE0008A4220D9023B2144891A43EA084343E7DA
:108AF0003A4605E7334618E70A4666E7B040904233
:108B0000B5D20CF1FF32002312E7334632460FE7AD
:108B10009A458DD9ACF1020C23448AE7B9459AD91C
:108B2000023D274498E70346DEE79046C6E7023851
:108B3000214435E74FEA4102B2F1E04324BFB3F5E7
:108B4000001CDCF1FE5C0DD901F0004C4FEAC002C4
:108B50004CEA5070B2F1004F40EB830008BF20F0A8
:108B60000100704711F0804F21D113F13872BCBF62
:108B700001F00040704741F480114FEA5252C2F1B7
:108B80001802C2F1200C10FA0CF320FA02F018BF00
:108B900040F001004FEAC1234FEAD32303FA0CFC53
:108BA00040EA0C0023FA02F34FEA4303CCE77FEAE2
:108BB000625307D150EA01331EBF4FF0FE4040F42C
:108BC0004000704701F0004040F0FE4040F40000DB
:108BD000704700BF1C481D49026800608A4200F0CF
:108BE0001D80002100F004B8194B5B58435004313C
:108BF0001848194B42189A42FFF4F6AF174A00F092
:108C000003B8002342F8043B154B9A42FFF4F9AF36
:108C1000FEF762FD00F038F8FFF7FEBF114E124874
:108C200030601248016821F070610160410201600A
:108C30000F4C182020600F490F4808600F48D0F8EB
:108C400000D0406800470000F04F0020EFBEADDECE
:108C500054F4000800000020F4000020F800002078
:108C600070170020181002400900000004000140A5
:108C7000140C0140000C01404434434400F0FF1F39
:108C8000FFF7FEBF000000002DE9804893B0F7F722
:108C90003FFA914E914CD6F80880002318F0080F47
:108CA0002370374600F0E78063681B7A042B00F2DC
:108CB000E080DFE803F00303058AB100237AD9E0FE
:108CC000627A864B002A00F0D48000225A7293F810
:108CD0002020100700F1CD80D97A9A7A01F00700A0
:108CE00042EA00225A621A7B02F03F00400140EA49
:108CF000D1019962597B890041EA92119A7B02F075
:108D0000010041EA8021D962D97B01F00F00C00146
:108D100040EA52021A631A7C02F07F00000140EA26
:108D200011115963597C490041EAD212997C01F032
:108D3000030042EA40229A63DA7C02F01F008001BD
:108D400040EA9101D963197DC90041EA5212997D27
:108D50001A645A7D01F0070042EA00225A64DA7D63
:108D600002F03F00400140EAD1019964197E890078
:108D700041EA92115A7E02F0010041EA8021D96451
:108D8000997E01F00F00C00140EA52021A65DA7EB6
:108D900002F07F00000140EA11115965197F490076
:108DA00041EAD212597F01F0030042EA40229A655B
:108DB0009A7F02F01F00800140EA9101D965D97FB6
:108DC000C90041EA52121A6651E094F86420434BFC
:108DD000002A4ED0002283F8642093F86620012AEE
:108DE00047D193F88A20102A84BF102283F88A2062
:108DF00094F88A103A4A0023D8B2884202F102025B
:108E000035D212F8010C12F8025C40EA052535480B
:108E100040F823500133EFE794F8CC202F4B42B3B6
:108E2000002283F8CC2093F8CD20A82A21D193F8F2
:108E3000E050F5B9294901EB450393F8D00093F8C8
:108E4000D13003EB0020FEF7CDFD1FA3D3E90023B3
:108E5000FEF768FF1EA3D3E90023FEF785FCFFF7AA
:108E600049F8214B43F825000135082DE2D10123B3
:108E700000E00023237018F4804F08D094F80431E8
:108E800023B1164B002283F8042101232370237899
:108E900043B118F4807F05D0104BD3F808311B681C
:108EA0001B689847DFF844802278D8F8003032B940
:108EB0000A4AD2F80C219A1AD243D20F00E00122BA
:108EC000B2B1F9F707FDB2E09A99999999991940C9
:108ED0000000000000707740A4100020F80000207F
:108EE0006001002084010020DC01002050170020D8
:108EF000D4F810A1A54D0AF10101C4F81011BAF17E
:108F0000000F40F09080D5F81421110740F18F80B8
:108F1000D5F818219A1A002AC0F2898003F5C339BE
:108F200005F58E7009F1A009C5F81891FDF746F90D
:108F3000974B05F58E7001461A78F8F785FD95F880
:108F4000220105F58E7110F0040F17D0C5F8249199
:108F50005346FA180025A2F8FE508C4ACD5A02F565
:108F6000947E23F80E5002F5977E23F80E500233BC
:108F7000062BEED120F0040082F8220194F834216F
:108F8000824BA2B1B3F81C01B6F8FE20821AA3F8F6
:108F90001C21B3F81E01B6F80021821AA3F81E2185
:108FA000B3F82001B6F80221821AA3F82021D4F8E0
:108FB0002431764A002B3AD07648C3EB0909814523
:108FC00002F5947502F5977019D8734BDA6882F43C
:108FD0000052DA600023CA5A35F903E017B2BE45E1
:108FE000C4BFDFF8C8E123F80E2030F903E0BE4526
:108FF000BCBF6A4FDA530233062BECD117E00023D3
:10900000C2F8243135F903E0C15EFA1871444FF01B
:10901000020E734491FBFEF1062BA2F8FE10F1D173
:10902000F9F74CFC03E00129C8BFC5F81021F8F797
:10903000DFFEB389C8F800002BB1D4F83821821ABA
:10904000002AFFF626AE1844504F7379C4F8380151
:10905000049307F5A870D4F84431D4F83C519847EC
:1090600007F5A870014694F85621F8F7EDFC4C4B33
:109070001B88002B00F0B980D7F858314FF000085A
:109080001B7807F5AE7903934746454A1288B2F537
:109090007A7F0292434A04D1002142F80810C9F8AD
:1090A00010104149C85F52F80810014442F80810F6
:1090B000FEF7FAFFD9F8102083460132012AC9F8D9
:1090C000102007D10022C9F80400C9F80000C9F82F
:1090D00008202CE0D9F800C061468DE80410FEF7A6
:1090E0002DFF009A82461046FEF7DEFF01465046ED
:1090F000FFF7E2F8DDF804C001466046FEF720FF06
:1091000002461146C9F8040058460092FEF716FFC1
:1091100001465046FFF71CF8D9F80810FEF710FF7B
:10912000009AC9F80C00C9F80020C9F808001E49C7
:10913000029B002201F1540B012B7A5227F80B20DD
:10914000DFF85CA044D1D9F81000012808DD01380F
:10915000FEF7AAFF0146D9F80C00FFF7ADF800E0D2
:10916000002002F015FA039B02460BB3184600924A
:10917000FEF79AFF009A01461046FFF7A5F9B8B12D
:109180004FF47A73AAF800302FE000BFF8000020F7
:109190005A1700207FC3C901001001402602002099
:1091A00058170020900200204802002020020020D2
:1091B000B54A4FF47A7158F802200A2002F5FA7283
:1091C00092FBF1F22BF807200F210122F8F7F3FEB2
:1091D0000237062F08F1040809F114097FF455AF8E
:1091E000029F07F1FF39AAF800900023A74F07F567
:1091F000A87207F5D271985A595A411A99520233F6
:10920000062BF3D1D7F8143113F0020300F00A83D0
:10921000D7F8B03107F5DC70984707F5DC700146E8
:1092200097F8BE21F8F710FCB7F8C03107F5DC78E5
:10923000002B45D00022D7F8C4011346934F38F9CC
:1092400002C0B7F8C01107F5E47EB1F5C87F04BFCE
:1092500000214EF803105EF803108C4F61444EF865
:109260000310043300210C2B28F80210815202F164
:109270000202E3D1B7F8C031012B1CD1D7F8C831B5
:109280004FF4C872C83393FBF2F30380D7F8CC31A4
:10929000C83393FBF2F34380D7F8D031C83393FB44
:1092A000F2F27B4B1B88D21A8280A5F85410A5F8E5
:1092B0005610F9F703FBB4F8C031013BA4F8C031F4
:1092C000B3685A0779D5B4F8D421704B322A13D138
:1092D000D3F8C4211188A3F8D61151889288A3F835
:1092E000D811A3F8DA21B5F85420A3F8DC21B5F899
:1092F0005620A3F8DE2101E0002A3CD00021D4F85A
:10930000C4610A46614838F901E0B0F8D43100F58B
:10931000F077322B04BF0023BB50B8585B4B70442E
:10932000B850043200200C2A28F80100705201F1D4
:109330000201E7D1B3F8D421012A17D183F8ED2136
:10934000052283F8EE21B3F8D62183F8EC013280B0
:10935000B3F8D8217280B3F8DA21B280B3F8DC21F7
:10936000B3F8DE31A5F85420A5F85630B4F8D4315E
:10937000013BA4F8D43194F8EF21444BEAB1D3F87F
:10938000E061D3F8C4113220002296FBF0F683F896
:10939000EF210E80D3F8E46196FBF0F64E80D3F80F
:1093A000E83193FBF0F03A4B1B88C01A8880A5F88F
:1093B0005420A5F85620F9F781FAD4F8C431B4F84E
:1093C000B8111A8800268A1AA4F8B821B4F8BA117C
:1093D0005A88B1468A1AA4F8BA219B88B4F8BC21ED
:1093E000D31AA4F8BC31F8F703FDD4F8F0310546E0
:1093F000C31A18460293FEF753FED4F8F4110390F3
:10940000FEF7A6FED4F8F881C4F8F05198F800A051
:10941000059035461F4F785FFEF746FE0599FEF72B
:1094200097FE09A98851BAF1000F35D05046FEF7D2
:109430003BFE01464FF07E50FEF73EFF02461146CE
:1094400007F1AC0B4FF07E500092FEF777FD56F817
:109450000B10FEF77DFE07F168018446485FCDF8EA
:1094600004C0FEF721FE009AB8371146FEF770FEE1
:10947000DDF804C001466046FEF762FD4BF80600C9
:10948000FFF72CF878530CE090020020F800002041
:10949000000000204802002007F1B8026837E95BAD
:1094A000A952AD4F0436EA5F0235062D02FB029940
:1094B000B0D1AA4D4FF0640A2A880AFB09F352433F
:1094C00093FBF2FAAAF1490A07F1080009A91FFA69
:1094D0008AFAF8F7A5FEBAF13B0FD8F8046010D964
:1094E000B4F91C02FEF7E0FDD4F8186201463046DC
:1094F000FEF7EAFF9A4F94F8223168B343F008036D
:109500002CE04FF07E513046FEF71AFD01464FF039
:109510007E50FEF7D1FE4FF0000B8246914B304655
:1095200053F81B100193FEF713FE024637F90B00A8
:109530000092FEF7B9FD009A01461046FEF700FDC5
:109540005146FEF705FE019B43F81B000BF1020B91
:10955000BBF1060FE2D1C3E723F008033146D4F88C
:10956000140287F8223102F011F80746C4F82002ED
:10957000D4F81002D4F818B200F10046D4F814025E
:109580000146FEF7E5FD594682465846FEF7E0FDE6
:1095900001465046FEF7D4FC01F0FAFF0146304682
:1095A00001F0F4FF70490646C4F824023846FEF77D
:1095B000CFFD01F01FFF6C49A4F828023046FEF7EA
:1095C000C7FD01F017FFD4F81431A4F82A021B07D5
:1095D00039D5664809A9F8F723FED8F808904FF066
:1095E0007E514846FEF7ACFC01464FF07E50FEF738
:1095F00063FE4FF0000B8246594D484605F50B734C
:1096000053F81B100193FEF7A3FD05F58E7102467A
:1096100031F90B000092FEF747FD009A0146104613
:10962000FEF78EFC5146FEF793FD019B43F81B00AD
:109630000BF1020BBBF1060FDED11846F8F7A8FEBE
:10964000A5F8380241E0DFF814A109A90AF10400E5
:10965000F8F7E6FD6868D5F808B00146FEF778FD32
:10966000D5F80C90594605465846FEF771FD01465F
:109670002846FEF765FC494605464846FEF768FD64
:1096800001462846FEF75CFC01F082FF00210546FA
:10969000FEF7F2FEA0B9DAF804002946FEF70CFE48
:1096A0002946CAF80400DAF80800FEF705FE294644
:1096B000CAF80800DAF80C00FEF7FEFDCAF80C0044
:1096C0002B48F8F765FEA4F838022A490398FEF7FC
:1096D0003FFD07F10047814606F10046B4F9380224
:1096E0000C970D96FEF7E0FC234900F10040FEF7D1
:1096F0002FFD0E90B4F90802FEF7D6FC0F90B4F9D6
:109700000A02FEF7D1FC1090B4F90C02FEF7CCFC73
:109710000CA911900FA8F8F783FD98F80130104DAF
:10972000012B2DD1154B1B785E070ED4D5F83C329A
:10973000402093FBF0F0181AFEF7B6FC1199FEF7E3
:10974000FFFBFEF7CBFEC5F83C02054BD3F83C020D
:10975000402390FBF3F015E0000300200000002000
:10976000F8000020080300204C3D0F442403002093
:1097700004000020BD37863535FA8E3C5C1700208A
:10978000A94B1888FEF790FC01461198FEF7D6FB0E
:10979000D4F8441211904846FEF7D2FB01464846E1
:1097A000FEF78AFDD4F84052064629461198FEF786
:1097B000C5FB01463046FEF7CBFC01462846FEF7C6
:1097C000BFFB0646C4F840020F98D4F8487201F077
:1097D00011FED4F854522978F8F7A4FF3844C4F89D
:1097E00048021098D4F84C7201F004FE2978F8F77A
:1097F00099FF3844C4F84C023046D4F8507201F056
:10980000F9FD6978F8F78EFF884B38441A68029F93
:10981000C4F850023A441A60D4F858320133C4F8FC
:10982000583205E0A7F8B831A7F8BA31A7F8BC312B
:109830007F4CB4F85031A4F85C32B4F85231A4F83B
:109840005E32049B012B0ED1B4F96222B4F954317B
:1098500003EB4203032293FBF2F39BB2A4F86032C2
:10986000A4F8623203E0B4F85431A4F86032F8F797
:10987000BFFA704BD4F890521860D4F86432C4F830
:109880006402C31A9BB20293A4F86832B4F970025E
:109890002B8998420EDBB0F5FA6FAF7907DAC21A5E
:1098A0005743A3F5FA6397FBF3F7643703E0C7F177
:1098B000640700E06427604BD4F83C61B3F81A8178
:1098C00093F9EC3000215B429BB2CDF80C800493FD
:1098D00034460A46594BDDF80CE031F90390CEEBE3
:1098E000090303F2F31C40F2E63EF44503D8002BD3
:1098F000B8BF5B4201E04FF4FA73022ADFF830E1AF
:1099000033D096F85DC1BCF1000F04D06345CCBFE5
:10991000CCEB030300234FF0640C93FBFCF80EEB3D
:10992000480A6FF0630B0BFB083BBAF894A20EEBEE
:10993000480EBEF996820FFA8AFECEEB080E0EFB99
:109940000BFEDFF804819EFBFCFEF24421F808A028
:1099500095F804E003FB0EFE394B9EFBF3F36344E2
:109960009BB27B4393FBFCFC1CE096F85EC1BCF110
:10997000000F04D06345CCBFCCEB03030023DDF81C
:10998000108003FB08FCAEF8A6C295F805E083EA58
:10999000E37CACEBE37C0CFB0EFC294B9CFBF3FC67
:1099A0000CF1640C06EB020E9EF80480254B0CFBB8
:1099B00008F84FF0640E98FBFEF802F8038094F864
:1099C0000EA003F103080CFB0AFA9AFBFEFA02F858
:1099D00008A094F818A003F106080CFB0AFC9CFBF5
:1099E000FEFCDDF80CE002F808C0F145A3F2AA285D
:1099F00007DA08F2A22331F803E0CEF1000E21F8D5
:109A000003E00132032A01F1020104F101047FF4B1
:109A100061AF094CB4F81C31984217DBB0F5FA6F0E
:109A2000A8BF4FF4FA6012E0000000205417002095
:109A3000F800002050170020A4100020620300202E
:109A40000CFEFFFFA20300209A0300201846C01A54
:109A50004FF47A725043C3F5FA63B0FBF3F3642614
:109A600093FBF6F208EB42016FF0630000FB023358
:109A7000B1F8B41208EB4202B2F9B6020AB2821A85
:109A8000534393FBF6F6B8F8CC3231445806B24D46
:109A9000A8F8A8123DD5B5F8CE32B5F83802C01AEC
:109AA00000B2FEF701FBAD49FEF752FB064601F09E
:109AB0006BFC0746304601F0DBFC0646B5F9A40214
:109AC000FEF7F2FA8146B5F9A202FEF7EDFA394641
:109AD0008246FEF73DFB314683464846FEF738FB9B
:109AE00001465846FEF72AFAFEF7F8FC3946A5F873
:109AF000A2024846FEF72CFB314607465046FEF7C9
:109B000027FB01463846FEF71BFAFEF7E7FCA5F8EF
:109B1000A402A26840F602031340002B66D0D8F8D6
:109B2000D062029B06211E4498F8D4328A4D01333C
:109B3000DBB2B3FBF1F088F8D43201FB103313F041
:109B4000FF07C8F8D06251D1910712D5F8F734F861
:109B500095F8D522B5F8D632934207D3D5F8D83246
:109B60009B7893428CBF0023012300E03B4688F89A
:109B7000DC32A3681A0536D598F8F132D8F8E0122D
:109B800008EB4303B3F8F402082391FBF3F280B22D
:109B90008A1A024492FBF3F39BB240F6E441594324
:109BA000D8F8D83240F6FF70B1FBF0F1D888C8F889
:109BB000E022091A4FF47A7251439B8891FBF3F12A
:109BC0004E43674B96FBF2F2C8F8FC12D3E9000152
:109BD000801841EBE271C3E90001624A0023FEF7FD
:109BE000C3FCC8F808030023C8F8D032D8F80C33F7
:109BF000594A13F4805318BF012382F81033A36825
:109C000098F8DC6213F4807F574C2CD0D8F81433CA
:109C100020781B68C0F380005B684F4D984758B1AF
:109C2000012385F81833D5F814331B68DB6898478F
:109C300010B1022385F81833D8F814331B689B68D9
:109C4000984730B123785B0703D4434B022283F853
:109C50001823D8F814331B689B69984718B13E4BFA
:109C6000002283F8182398F818233B4B022A02D1CC
:109C70004C204E2114E0012A06D153204D214C22C4
:109C80000B46FAF7C5FC1FE093F81023012A04D114
:109C90005320014602464D23F3E726B153204D21C0
:109CA0000A464423EDE7B3F8CC22170603D5532028
:109CB0004D210246E4E793F8EE211AB11920FAF794
:109CC0007DFC01E083F819632278550704D5274B02
:109CD0004FF400525A6171E0D8F80C33D80703D41E
:109CE000214942F001020A70B8F8C02122B11A4A93
:109CF000D2F81421910705D41D4A1288003218BFEA
:109D0000012200E0012242B1184AD16881F40051D9
:109D1000D160227822F00102227098F822211207E5
:109D200003D4227822F001022270DB0203D52378CB
:109D300023F00103237023780E4A13F0010F1BD088
:109D40000023C8F81C3303F180434FF4005103F59E
:109D5000883319611FE000BFF800002035FA8E3CFF
:109D6000F8030020407E05005C1700200010014031
:109D70005817002050170020D8F81C13136851B949
:109D80007E4903F5F42303F59073C1F81C337C4B33
:109D90004FF400515961D8F81C33126873B1D21ACC
:109DA000002A0BDB764A03F5F423D16803F59073A0
:109DB00081F40051D160714AC2F81C33714B1B7899
:109DC0001BB1F9F7FDFD00F066BD6F4C94F84A3009
:109DD000012B40F05B85694D2368C5F8B843C5F891
:109DE000BC33664ED6F8BC03354603685B689847BB
:109DF000002800F04585D6F8BC0303689B689847A7
:109E0000D6F8B83393F84820E2B9B0F124077A4283
:109E10007A4183F84820002AE3D15C4B1B785D0728
:109E2000DFD4232802D1F9F7CBFDDAE7D6F8C03327
:109E30001B7D8342D5D1564A564B1A60564A574B22
:109E4000DA60CEE7012A05D14D2814BF0022022294
:109E500000F012BD022A05D13C2814BF00220322C3
:109E600000F00ABD032A0BD140284FF0000200F297
:109E700003851A71DA7158719871042200F0FCBCE4
:109E8000042A07D19A7983F8490050409871052235
:109E900000F0F2BC052AA4D159791A799142997936
:109EA00006D941409971511C19711344187298E7F1
:109EB000814240F0DD8493F84970682F00F067829A
:109EC00000F21B812C2F00F0868448D8242F00F04C
:109ED00067842BD8202F00F04A82222F00F0908335
:109EE000012F40F0A1842C20F8F7F6F80020F8F7B5
:109EF000C4F83846F8F7C1F80020F8F7BEF8432058
:109F0000F8F7BBF84C20F8F7B8F84620F8F7B5F8A2
:109F10004C20F8F7B2F83846F8F7AFF80020F8F719
:109F2000ACF80020F8F7A9F8002665E1282F00F02A
:109F30003F842A2F00F04984262F40F07584184E64
:109F40000320F8F7C9F8B6F9E600F8F7C8F8B6F94B
:109F5000E800F8F7C4F8B6F9EA0000F033BC642F63
:109F600000F071811ED8342F00F06A83402F00F07A
:109F70004D84322F40F0588400F041BCF80000209E
:109F8000001001405B170020180400205C1700201F
:109F9000EFBEADDEF04F00200400FA0500ED00E05A
:109FA000A4100020662F00F0798100F2AE810B2012
:109FB000F8F792F8B6F96802F8F791F8B6F8C40322
:109FC00000B2F8F78CF8D6F81431C3F3C000C3F32D
:109FD0008002800040EA4200C3F340021043C3F312
:109FE000401240EAC20003F010031843F8F777F874
:109FF000B6F8CC22D6F80C3312F0010F0CBF0027B4
:10A00000022712F0020F0CBF4FF000084FF00408B7
:10A0100012F0040F0CBF4FF0000E4FF0100E12F0B4
:10A02000400F0CBF0020202012F0100F0CBF0021A9
:10A030004FF4007112F0200F02970CBF00274FF46D
:10A04000806703F48026CDF80C8002F0080B03F43F
:10A050000058CDF810E0059003F4803E03F4002092
:10A0600003F4807A0691079703F4801103F4003714
:10A0700003F4805903F4004C03F0C00343EA0B03DC
:10A0800043EA0A0343EA090343EA080343EA0C03E9
:10A0900043EA0E033B43334303430B43D249DDF80A
:10A0A000088091F800E00498CEF3800E43EA0E0396
:10A0B000DDF80CE043EA080343EA0E030599034385
:10A0C000069F0B43DDF81C8012F4807F43EA0703F0
:10A0D0000CBF00254FF4006543EA080312F4007F2B
:10A0E00043EA05030CBF00224FF400121A43BF4B92
:10A0F000002093F8C6630346B9E0732F00F018837D
:10A1000051D86E2F00F0908110D86C2F00F057813D
:10A1100000F26381692F40F0878396F8DD03002603
:10A12000400000F0FE00F7F7D7FF3CE1702F00F091
:10A13000C881C0F0A181722F40F07683AC4F162009
:10A14000F7F7CAFF0020F7F7CAFFB7F9D000F7F713
:10A15000C6FFB7F9D200F7F7C2FFB7F9D400F7F797
:10A16000BEFFD6F83C31B3F9A801F7F7B8FF0020DD
:10A17000F7F7B5FF0020F7F7D7FFD6F83C31B3F972
:10A1800052000A2390FBF3F0F7F7A9FF97F80401B8
:10A19000F7F773FF97F80601F7F76FFF97F80501D8
:10A1A000F7F76BFFC2E2782F00F0BB800DD8752F58
:10A1B00000F01A82C0F06D82772F40F0358396F858
:10A1C000C603F7F789FF0026A3E2F02F00F0DA823A
:10A1D000FE2F00F0B882A02F40F026830C20F7F766
:10A1E0007BFF844B1868F7F79FFF834B1868F7F7DE
:10A1F0009BFF824B1868D8E2814B1B68985D013643
:10A20000F7F73BFF042EF7D10020F7F768FF002691
:10A210007C4B985D0136F7F730FF0B2EF8D1002606
:10A22000794B985D0136F7F728FF082EF8D1072003
:10A23000F7F723FF0026754B985D0136F7F71DFFF2
:10A24000072EF8D172E20720694EF7F745FFE620A6
:10A25000F7F713FF7079F7F710FF0020F7F70DFFFE
:10A2600096F82631002B0CBF04200C209DE2B3424F
:10A270000CD267495F5C012101FA07F7174218BF4A
:10A28000994003F1010318BF0843F0E7F7F74CFFCB
:10A29000574B93F86C06F7F7F0FEE3E21220F7F75E
:10A2A0001BFF5C4B1B88B3F5806F21D900275A4BED
:10A2B000F85E082390FBF3F00237F7F710FF062F44
:10A2C000F5D1B6F95C02F7F70AFFB6F95E02F7F7C7
:10A2D00006FFB6F96002F7F702FFB6F91C01F7F7BF
:10A2E000FEFEB6F91E01F7F7FAFEB6F9200169E2A3
:10A2F000B6F90802F7F7F3FEB6F90A02F7F7EFFE30
:10A30000B6F90C02F7F7EBFEDBE71020F7F7E4FEF7
:10A310000026424B985D0136F7F7AFFE102EF8D1BC
:10A32000A0E23820F7F7D8FE0027D5F83C3107F136
:10A330002C06F6003344B3F90600F7F7D0FED5F843
:10A340003C3101373344B3F90800F7F7C8FED5F8BC
:10A350003C313344B3F90A00F7F7C1FED5F83C317C
:10A360001E44307BF7F789FE082FDED17AE2082001
:10A37000F7F7B2FE0026D5F83C3103EBC60393F89D
:10A380006D010136F7F779FE082EF4D16AE210204C
:10A39000F7F7A2FE0026224B985D0136F7F76DFE17
:10A3A000102EF8D15EE295F8DD339E4280F05A829D
:10A3B0001C4B33F91600F7F792FE0136F3E706203F
:10A3C000F7F78AFEB6F92802F7F789FEB6F92A02EE
:10A3D000F7F785FEB6F93802F4E10620F7F77CFEC0
:10A3E0000020F7F7A1FEBAE15C170020F80000207A
:10A3F000A4100020E8F7FF1FECF7FF1FF0F7FF1F86
:10A400007800002098DD0008A4DD0008ADDD00081C
:10A41000BF04002000000020000300206200002094
:10A4200036170020620300200720F7F755FE96F844
:10A43000D502F7F722FED6F808034FF6FF77B842A9
:10A44000A8BF384620EAE07000B2F7F748FEB6F938
:10A45000E003F7F744FEC34DC34BD5F8FC0293F875
:10A460000C310028B8BF40420BB10A235843B84210
:10A47000A8BF384600B2A5E10720F7F72DFED6F8B1
:10A4800090321878F7F7F9FDD6F890325878F7F748
:10A49000F4FDD6F890321879F7F7EFFDD6F8903240
:10A4A0005879F7F7EAFDD6F890329879F7F7E5FD95
:10A4B000D6F890329878F7F7E0FDD6F89032D87851
:10A4C000E9E61E20F7F708FED6F83C3100261B7897
:10A4D000022B73D1A348A549D0F83C3103EB860386
:10A4E000586AFDF735FE00F085FFFA28A8BFFA206C
:10A4F00020EAE070C0B2F7F7C0FD9A49D1F83C31CC
:10A500009B4903EB8603186BFDF722FE00F072FFF8
:10A51000FA28A8BFFA2020EAE070C0B2F7F7ADFD34
:10A52000904A9449D2F83C3103EB8603D86BFDF78F
:10A530000FFE00F05FFF6428A8BF642020EAE070EF
:10A54000C0B20136F7F799FD032EC3D1072ED5F817
:10A550003C311FD1986C8549FDF7FAFD00F04AFFA8
:10A56000FA28A8BFFA2020EAE070C0B2F7F785FD0C
:10A57000D5F83C317D49D86CFDF7EAFD00F03AFF93
:10A58000FA28A8BFFA2020EAE070C0B2F7F775FDFC
:10A5900000200DE033441879F7F76FFDD5F83C3112
:10A5A0003344987BF7F769FDD5F83C313344187E86
:10A5B0000136F7F762FD0A2EC8D153E1D5F83C31D8
:10A5C00033441879F7F759FDD5F83C313344987B7B
:10A5D000F7F753FDD5F83C313344187E0136F7F7D1
:10A5E0004CFD0A2EEAD13DE12F20F7F775FD624EB2
:10A5F00016F8010F002800F03581F7F73EFDF7E768
:10A60000A020F7F769FD0026D5F83C3106F11C02C1
:10A6100003EB82035F1D594A5B790C2101FB032385
:10A62000187AF7F72AFD7878F7F727FDB878F7F763
:10A6300024FD0136F878F7F720FD282EE4D111E14A
:10A640004820F7F749FD00274FF0060909FB07F9F5
:10A65000D5F83C3109F58879994499F80A00F7F75B
:10A660000CFD99F80500F7F708FD99F80600F7F7D3
:10A6700004FD99F80700F7F700FD99F80800F7F7CF
:10A68000FCFC013799F80900F7F7F7FC0C2FDBD138
:10A69000E8E04FF000090126002795F8C6339F42F5
:10A6A00024DA374BF95C0023344A03EB020B9A5C43
:10A6B0008A4204D00C33B3F58A7FF5D114E0DBF87D
:10A6C000040000F073FC80460EB9B24601E08144FC
:10A6D0000AE0C24508DADBF8042012F80A00F7F7AE
:10A6E000CCFC0AF1010AF4E70137D6E7002E00F0AE
:10A6F000B9805FFA89F0F7F7EFFC0026CCE71F4A34
:10A7000099189A5C82420DD00C33B3F58A7FF6D14A
:10A71000013695F8C6339E4280F0A480184BF05C59
:10A720000023ECE7087AF7F7A8FCF1E70020B2E590
:10A730000820F7F7D1FC0126F0B20136F7F79DFCAF
:10A74000092EF9D18EE00820F7F7C6FC0020F7F7B4
:10A75000C6FC0020F7F7C3FC0020F7F7C0FC002080
:10A7600030E000BFF8000020A410002000002041CD
:10A770000000C84200007A445FCA000890CA00087E
:10A78000BF0400200420F7F7A7FCD6F83C31B3F94A
:10A790005600F7F7A4FCD6F83C31B3F9540011E0A9
:10A7A0000420F7F799FCB04B9868F7F7BDFC59E027
:10A7B000AD4E0420F7F790FCB6F90801F7F78FFCCF
:10A7C000B6F90A01F7F78BFC4CE00120F7F784FC9F
:10A7D000A54B58795FE5A44E0720F7F77DFC96F866
:10A7E0001801F7F74AFCB6F91E01F7F778FCB6F93D
:10A7F0001A01F7F774FCB6F91C01F7F770FC012099
:10A80000F7F76AFC984B93F8200144E50820F7F726
:10A8100063FC0026944B334493F810010136F7F79C
:10A820002CFC082EF6D11DE0C82F00F04A8340F220
:10A830004881D02F00F0328240F29081D42F00F076
:10A840001D8300F2FB82D22F40F0F182874B1B78F0
:10A8500003F0040303F0FF06002B00F0DD8200206C
:10A86000F7F73AFC824BD3F8B8339879F7F705FC41
:10A870007F4B0022D3F8B83383F84820FFF7B1BAF2
:10A8800096F8FC3313B17B4A7B4BDA607B4B4C343C
:10A890009C427FF49BAA764CD4F8483113B104F261
:10A8A000FE309847D4F81431714A13F0080F6E4EF9
:10A8B00038D0B2F8A61201F145039BB28A2B2DD8ED
:10A8C000B2F8CC325F0729D5B2F83802B2F8E233D9
:10A8D00094F82251C21A92B293B218B2B330BCBFEC
:10A8E00002F5B4739BB21AB2B32AC4BFA3F5B47312
:10A8F0009BB22D0796F8EC005D4A13D540B240425A
:10A900004343D2F83C011BB2007B43436FF01D0070
:10A9100093FBF0F31944A2F8A61203E0B4F838321E
:10A92000A4F8E233D4F83C71514D97F86491B9F131
:10A93000000F51D0B5F8CC329A074DD0D5F810029F
:10A94000D5F814320146D5F81882B5F8A8A20193BB
:10A95000FDF7FEFB019B834619461846FDF7F8FB01
:10A9600001465846FDF7ECFA414683464046FDF75E
:10A97000EFFB01465846FDF7E3FA00F009FE0146F9
:10A980004046FDF799FC3E498046FDF789FDF8B940
:10A99000404600F0ABFDD5F80014FDF7D9FB00F000
:10A9A00029FDB0F5617FA8BF4FF46170FDF77CFB16
:10A9B0003449FDF781FC00F05BFD05464846FDF794
:10A9C00073FB2946FDF7C4FB00F014FD80B200E0E4
:10A9D00000205044A4F8A8022B4B381D1D68D4F861
:10A9E000901207F15403B6F8F620A847FAF7A2FC34
:10A9F000D4F80434002B60D01D4B93F80834013B8D
:10AA0000142B55D8DFE803F00B5454275754541F28
:10AA10005454545454445454545454274400D4F873
:10AA20000C345B782BB1194B00205989F7F7F2FEF3
:10AA300043E00E4B1B7803F0040303F0FF00002BF0
:10AA4000F1D10146F2E7114C0020E188F7F7E2FE70
:10AA500001202189EAE70D4C00202189F7F7DAFE71
:10AA600001206189E2E700BFA41000205C170020EC
:10AA7000F80000200400FA0500ED00E0B00400201A
:10AA80008FC2753CEFB6B044740000206200002015
:10AA9000C04C0020E188F7F7BDFE01202189F7F7BF
:10AAA000B9FE02206189F7F7B5FE0320A189BDE751
:10AAB000B3689B0601D5F7F7B9FEFCF755FBFEF727
:10AAC000E8B82B2F07D10020F7F706FBF7F7B8F807
:10AAD000B14B5871C3E636D8252F10D1AE4E0020A9
:10AAE000F7F7FAFA0023B360F7F7B4F80746F7F779
:10AAF000B1F8B36807EB00400343B360AFE650D84A
:10AB0000212F00F0EC81232F40F0F681F7F798F821
:10AB100027281ED8D6F83C3100F11C0703EB870725
:10AB2000F7F78EF89D4B7E1D03F58A72197A8142E4
:10AB300003D00C339342F9D10BE01B787B71F7F70C
:10AB40007FF8707026E0352F6AD1F7F779F80B2877
:10AB50004AD901200021F7F7A1FA80E6CD2F00F0B5
:10AB6000A98000F20981CA2F00F0AE80CC2F40F0FE
:10AB7000C381D6F89062F7F763F83070F7F760F8A2
:10AB80007070F7F75DF83071F7F75AF87071F7F7F2
:10AB900057F8B071F7F754F8B070F7F751F8F07054
:10ABA0005DE6272F10D10020F7F796FAF7F752F855
:10ABB000794EA6F8E600F7F74DF8A6F8E800F7F7A3
:10ABC00049F8A6F8EA004AE6292F40F095810020CE
:10ABD000F7F782FAF7F73EF86F4EA6F80801F7F795
:10ABE00039F8A6F80A013AE606277843D6F83C7108
:10ABF00000F588700744F7F723F80328A9D8B8723E
:10AC0000F7F71EF87871F7F71BF8B871F7F718F82F
:10AC1000F871F7F715F83872F7F712F878721EE640
:10AC200022D82D2F14D10020F7F756FAF7F708F89D
:10AC3000594E86F81801F7F70DF8A6F81E01F7F738
:10AC400009F8A6F81A01F7F705F8A6F81C0106E6B8
:10AC5000332F40F051810020F7F73EFAF6F7F0FF6E
:10AC60004D4B83F82001FAE5412F0DD10020F7F775
:10AC700033FA0026F6F7E4FF474B33440136082E3B
:10AC800083F81001F6D1EAE5442F40F03581002029
:10AC9000F7F722FA012386F8FC33E0E5404B1B78F6
:10ACA00058073FF5DCADF8F79DFFFCF7EBF8F8F738
:10ACB00091FBD4E53A4B1B7859073FF5D0AD4FF4E3
:10ACC000C873A6F8C031CAE5D6F83C713B78022BB0
:10ACD00042D10026F6F7B4FFFDF7E2F93149FDF75E
:10ACE000EBFA7862F6F7ACFFFDF7DAF92E49FDF7DB
:10ACF000E3FA3863F6F7A4FFFDF7D2F92B49FDF725
:10AD0000DBFA0136032EF86307F10407E2D1072EC0
:10AD1000D5F83C7112D1F6F793FFFDF7C1F921493F
:10AD2000FDF7CAFAB864F6F78BFFFDF7B9F91D49CC
:10AD3000FDF7C2FAF864F6F783FF09E0F6F780FF43
:10AD400037443871F6F77CFFB873F6F779FF387639
:10AD500001360A2EDBD182E5013F0026F6F770FFAF
:10AD600001373871F6F76CFFB873F6F769FF0136F3
:10AD70000A2E3876F2D172E5CE2F19D1084B1B7806
:10AD80005A073FF56CAD96F8223143F0040386F87C
:10AD9000223164E562000020A410002090CA00085F
:10ADA0005C170020000020410000C84200007A44E7
:10ADB000CF2F40F0A180F6F74DFFF6F74BFF514F34
:10ADC000A7F8D000F6F746FFA7F8D200F6F742FF43
:10ADD000D6F83C61A7F8D400F6F73CFFA6F8A80126
:10ADE000F6F738FFF6F736FFF6F734FFF6F732FFDF
:10ADF00000EB80004000A6F85200F6F721FF87F82C
:10AE00000401F6F71DFF87F80601F6F719FF87F82A
:10AE10000501F6F715FF22E5F6F712FF394B022878
:10AE200083F86C067FF641AF83F86C663DE7D32F5D
:10AE300062D1F6F70FFFA6F8E20310E5EF2F0AD173
:10AE4000D6F83C61F6F706FFA6F85600F6F702FFC3
:10AE5000A6F8540003E5FA2F05D12B4B1B785B07AE
:10AE60007FF523AF48E0D62F46D10026F6F7F2FE55
:10AE7000264B98530236102EF8D1F0E40027D5F86F
:10AE80003C61F6F7E7FE06EBC706A6F86601F6F7A3
:10AE9000E1FEA6F86801F6F7DDFEA0F57A73072853
:10AEA0009BB298BF86F86D01B3F57A7F98BFA6F87C
:10AEB0006A01F6F7C5FE0137082F86F86C01DED16E
:10AEC000CDE40026F6F7C6FE114B03F26A2290533A
:10AED0000236102EF6D1012283F80421BFE40026A9
:10AEE000D5F83C71F6F7ACFE07EBC6070136082E25
:10AEF00087F86D01F4D1B2E401200021F7F7CEF814
:10AF0000B0E400BFA41000205C170020DC04002087
:10AF1000F8000020AFF3008010B50023934203D067
:10AF2000CC5CC4540133F9E710BD0244034693429C
:10AF300002D003F8011BFAE7704700000D4B70B513
:10AF40001D680022845C2B195B7803F00303012B3E
:10AF50008B5C08BF2034EE18767806F00306012ECD
:10AF600008BF2033E41A02D10132002BEAD1204677
:10AF700070BD00BF8800002010B50446224613783B
:10AF80000134002BFAD1CC5CD4540133002CFAD11B
:10AF900010BDC9B2024610F8013B1BB18B42F9D17A
:10AFA000104670470029FBD018467047034613F837
:10AFB000012B002AFBD1181A013870470F4BF0B54E
:10AFC0001E680023934215D0C55C7419647804F0A0
:10AFD0000304012CCC5C08BF203537197F7807F0BB
:10AFE0000307012F08BF20342D1B04D10133002C8F
:10AFF000E8D100E000252846F0BD00BF8800002011
:10B0000010B5034632B111F8014B013A03F8014B78
:10B01000002CF7D11A44934203D0002103F8011BFE
:10B02000F9E710BD30B503780BB1044604E00B78A6
:10B03000002B18BF002030BD22461078013438B1F3
:10B040000023C85C28B1D55C8542F5D10133F8E70F
:10B0500030BD104630BD00210A2200F001B92DE9B3
:10B06000F04E82468B461F46144612B90020BDE8BA
:10B07000F08E002BFAD00026A642F7D2A5196D0853
:10B0800007FB05B950464946089B9847002802DB54
:10B0900003D06E1C25462C46EEE74846BDE8F08EF0
:10B0A000174B2DE9F0411D680646AC6D0F46FCB903
:10B0B000502000F0E3F8A8658460AB6D0460446044
:10B0C0001C61DC60AB6D9C615C61AB6DDC629C62A1
:10B0D000AB6D5C631C63AB6DDC639C63AB6D5C64EC
:10B0E0001C64AB6DDC649C64AB6D1C77AB6D5C6207
:10B0F00030463946AA6D0123BDE8F04100F002B8A0
:10B10000EC000020F0B508B9106828B3044614F824
:10B11000015B0F4617F8016B3EB1B542FAD10BB196
:10B120002046F3E714600370F0BD4DB91560284662
:10B13000F0BD17F8016BAE4207D0002EF9D11C46C6
:10B14000234613F8015B0F46F3E715B10021217088
:10B1500000E02B461360F0BDF0BD000084463F4880
:10B160002DE9F04FD0F800800E46344614F8015B0C
:10B1700008EB0500407800F0080000F0FF0708B178
:10B180002646F2E72D2D03D1B41C7578012703E084
:10B190002B2D04BF7578B41C33F010000DD1302D69
:10B1A00008D1207800F0DF00582851D165781023AD
:10B1B000023402E0002B08BF0A23002F0CBF6FF0FF
:10B1C000004A4FF0004ABAFBF3F903FB19AA002624
:10B1D000304608EB050B9BF801B01BF0040F01D0C3
:10B1E000303D0BE01BF0030B1BD0BBF1010F14BF74
:10B1F0004FF0570B4FF0370BCBEB05059D4210DAA4
:10B20000B6F1FF3F0AD0484506D801D1554503DCC9
:10B2100003FB0050012601E04FF0FF3614F8015BFC
:10B22000D7E7731C0CD1002F4FF022030CBF6FF037
:10B2300000404FF00040CCF800302AB9BDE8F08F54
:10B2400007B1404242B106B1611E1160BDE8F08F06
:10B25000002B08BF0823B0E7BDE8F08F880000206E
:10B2600030B51346044A05460C4610682946224666
:10B27000BDE83040FFF772BFEC000020024B0146F2
:10B28000186800F003B800BFEC00002070B5CD1CBA
:10B2900025F0030508350C2D38BF0C25002D06467A
:10B2A0003FDB8D423DD3214B1C6818462146A1B19E
:10B2B0000B685B1B0ED40B2B03D90B60CC18CD5045
:10B2C0001FE08C4202D1626802601AE04B68636042
:10B2D0000C4616E00C464968E9E7154C23681BB993
:10B2E000304600F027F820602946304600F022F86A
:10B2F000431C014615D0C41C24F0030484420AD127
:10B30000256004F10B00231D20F00700C31A0BD0A9
:10B310005A42E25070BD3046611A00F00BF801301D
:10B32000EED10C233360002070BD00BF64170020F5
:10B330006017002038B5064C0023054608462360F8
:10B3400000F008F8431C02D1236803B12B6038BD1C
:10B350006C170020094A136863B118446946884293
:10B3600002D8106018467047054B0C221A604FF047
:10B37000FF307047034B1360EFE700BF68170020F2
:10B380006C1700207017002000B5194A20F0004308
:10B39000934283B0014617DDB3F1FF4F04DBFCF7A6
:10B3A000CDFD03B05DF804FB694600F037FB00F00B
:10B3B0000302012A0098019911D0022A0AD09AB1F9
:10B3C000012201F0EFF8ECE7002100F0EFFC03B000
:10B3D0005DF804FB00F0EAFC00F10040E1E701F059
:10B3E000E1F800F10040DCE700F0E0FCD9E700BF45
:10B3F000D80F493F30B5C0F3C754A4F17F031E2BCB
:10B4000083B0014620DC581C1BDB162B4FEAD1759C
:10B4100009DDC1F3160040F40000963CA04005B1E0
:10B42000404203B030BD114B53F825402046FCF795
:10B4300087FD019001982146FCF780FD20F0004334
:10B4400033B9002003B030BDFDF748F803B030BD7C
:10B45000C0F31604C0F3C75044F40004C0F19600D2
:10B4600024FA00F0002DDCD0DAE700BF40F000083D
:10B4700000B51D4A20F00043934283B0014618DD19
:10B48000B3F1FF4F04DBFCF759FD03B05DF804FB9B
:10B49000694600F0C3FA00F00300012818D0022822
:10B4A0000ED0D0B10098019900F080FC00F100406E
:10B4B000EBE70021002201F075F803B05DF804FB12
:10B4C00000980199012201F06DF800F10040DCE7DD
:10B4D0000098019900F06AFCD7E7009801990122D1
:10B4E00001F060F8D1E700BFD80F493F70B58AB0CE
:10B4F000054600F09BF8224C064694F900300133D3
:10B5000003D0284601F02CFA10B930460AB070BDBD
:10B51000284601F0DBF94FF07E51FCF7D5FF0028FB
:10B52000F3D0184901220023284600920893019184
:10B53000FCF77AFA02460B461348CDE90423CDE91D
:10B54000022301F0A7F894F90030CDE90601022B9F
:10B550000BD0684601F09CF838B1089B53B9DDE97F
:10B560000601FDF7E7FA0AB070BD01F073FA212376
:10B570000360F2E701F06EFA089B0360EFE700BF9B
:10B58000F000002048F0000850F0000800F0B6B9C4
:10B5900070B58AB0054600F0B5FB224C064694F91A
:10B5A0000030013308D0284601F0DAF920B12846EE
:10B5B0000021FCF76BFF10B930460AB070BD1A4984
:10B5C000012200232846019100920893FCF72CFAEF
:10B5D0002478CDE90401CDE902017CB900220023E1
:10B5E000CDE90623684601F053F888B1089BA3B95A
:10B5F000DDE90601FDF79EFA0AB070BD00200021CA
:10B6000002460B46FCF78EFB022CCDE90601E9D180
:10B6100001F020FA21230360E8E701F01BFA089B00
:10B620000360E5E7F000002054F00008F8B520F0D2
:10B630000043B3F17E5F044610D008DCB3F17C5FB9
:10B6400011DAB3F10C5F00F384809D48F8BD014628
:10B65000FCF774FC0146FCF72FFEF8BD002840F310
:10B66000CD800020F8BD0028C0F2CA8001464FF00E
:10B670007E50FCF763FC4FF07C51FCF769FD0446FB
:10B6800000F040FB8F4906462046FCF761FD8E49DD
:10B69000FCF756FC2146FCF75BFD8C49FCF74EFCA1
:10B6A0002146FCF755FD8A49FCF74AFC2146FCF788
:10B6B0004FFD8849FCF742FC2146FCF749FD8649CD
:10B6C000FCF73EFC2146FCF743FD84490546204635
:10B6D000FCF73EFD8249FCF731FC2146FCF738FDC2
:10B6E0008049FCF72DFC2146FCF732FD7E49FCF732
:10B6F00025FC2146FCF72CFD4FF07E51FCF720FC89
:10B7000001462846FCF7D8FD3146FCF721FD26F41A
:10B710007F6525F00F05074629462846FCF718FDEA
:10B7200001462046FCF70AFC294604463046FCF751
:10B7300007FC01462046FCF7BFFD01463846FCF7F2
:10B74000FFFB01462846FCF7FBFB0146FCF7F8FB34
:10B75000F8BD0146FCF7FCFC5A490546FCF7F8FC2D
:10B760005949FCF7EDFB2946FCF7F2FC5749FCF779
:10B77000E5FB2946FCF7ECFC5549FCF7E1FB2946C3
:10B78000FCF7E6FC5349FCF7D9FB2946FCF7E0FC43
:10B790005149FCF7D5FB2946FCF7DAFC4F49064630
:10B7A0002846FCF7D5FC4E49FCF7C8FB2946FCF7B8
:10B7B000CFFC4C49FCF7C4FB2946FCF7C9FC4A49BD
:10B7C000FCF7BCFB2946FCF7C3FC4FF07E51FCF7AD
:10B7D000B7FB01463046FCF76FFD01462046FCF7FB
:10B7E000B7FC01464148FCF7A9FB01462046FCF79F
:10B7F000A5FB01463E48FCF7A1FBF8BD3D48F8BD5E
:10B800004FF07E51FCF79CFB4FF07C51FCF7A0FC05
:10B810002C490446FCF79CFC2B49FCF791FB214684
:10B82000FCF796FC2949FCF789FB2146FCF790FCC4
:10B830002749FCF785FB2146FCF78AFC2549FCF7E4
:10B840007DFB2146FCF784FC2349FCF779FB21466C
:10B85000FCF77EFC0646204600F054FA1F490546D8
:10B860002046FCF775FC1E49FCF768FB2146FCF7F7
:10B870006FFC1C49FCF764FB2146FCF769FC1A4984
:10B88000FCF75CFB2146FCF763FC4FF07E51FCF7B4
:10B8900057FB01463046FCF70FFD2946FCF758FCE4
:10B8A0001249FCF74BFB01462846FCF749FB0146D1
:10B8B000FCF746FB01461048FCF740FBF8BD00BF13
:10B8C000DB0FC93F08EF1138047F4F3A4611243D82
:10B8D000A80A4E3E90B0A63EABAA2A3E2EC69D3D7B
:10B8E0006133303F2D57014039D119406821A233CF
:10B8F000DA0FC93FDB0F4940DA0F494021F000421F
:10B90000B2F1FF4FF8B5044614DC20F00045B5F164
:10B91000FF4F06460EDCB1F17E5F3AD08F1707F07D
:10B92000020747EAD07755B9022F2FD0032F2FD126
:10B930003148F8BD08462146FCF702FBF8BDFAB1D4
:10B94000B2F1FF4F29D0B5F1FF4F19D0AA1AD21585
:10B950003C2A19DC002938DB2046FCF7ADFC00F05E
:10B96000B5FF00F09DFE012F2CD0022F22D0002F1A
:10B970002FD02249FCF7E4FA2149FCF7DFFAF8BDA1
:10B98000002E15DB1F48F8BD1E48ECE71C48F8BD2B
:10B99000F8BDBDE8F84000F083BEB5F1FF4F19D007
:10B9A000022FF3D0032FC3D0012F1BD00020F8BDEE
:10B9B0001548F8BD1149FCF7C3FA01461048FCF7D9
:10B9C000BDFAF8BD00F10040F8BD3C32C4DA0020F9
:10B9D000C9E7F8BD022F0CD0032F08D0012F04D0E7
:10B9E0000A48F8BD4FF00040F8BD0948F8BD0948C5
:10B9F000F8BD0948F8BD00BFDB0F49C02EBDBB3301
:10BA0000DB0F4940DB0FC93FDB0FC9BFDB0F493FED
:10BA1000DB0F49BFE4CB16C0E4CB16402DE9F04F55
:10BA2000AB4A20F00044944289B006460D4664DDDE
:10BA3000A84A94421CDC0028A74940F3EC80FCF79C
:10BA40007DFAA64B24F00F049C42064664D0A4491C
:10BA5000FCF774FA014628603046FCF76FFAA049FB
:10BA6000FCF76CFA01236860184609B0BDE8F08F56
:10BA70009C4A944262DDB4F1FF4F46DAE715863FF7
:10BA8000A4EBC7542046FCF729FDFCF70DFB034649
:10BA9000014620460593FCF751FA4FF08741FCF729
:10BAA00057FB8046FCF71AFDFCF7FEFA01460446F8
:10BAB00040460694FCF742FA4FF08741FCF748FBFA
:10BAC00000210790FCF7D8FC002800F0C580204634
:10BAD0000021FCF7D1FC002814BF01230223824877
:10BAE0000221019000913A4605A8294600F022FA69
:10BAF000002EC0F2A780034603E000222860002346
:10BB00004A60184609B0BDE8F08F0146FCF716FA06
:10BB1000002368602860F4E77449FCF70FFA744961
:10BB20000446FCF70BFA014628602046FCF706FAAB
:10BB30006F49FCF703FA01236860E2E700F0C6FEF4
:10BB40006C490746FCF704FB4FF07C51FCF7F8F911
:10BB5000FCF7C4FC8246FCF7A7FA5F498346FCF772
:10BB6000F7FA01463846FCF7E9F95D498046584640
:10BB7000FCF7EEFABAF11F0F81464946404618DC41
:10BB80005D4B0AF1FF3253F8223024F0FF029A4253
:10BB90000FD0FCF7D3F907462F6039464046FCF733
:10BBA000CDF94946FCF7CAF9002E686056DB5346CA
:10BBB000A7E7FCF7C3F9E315C0F3C7529A1A082A9E
:10BBC0000746E9DD494958460393FCF7C1FA0746A1
:10BBD00039464046FCF7B2F9044621464046FCF798
:10BBE000ADF93946FCF7AAF9414907465846FCF732
:10BBF000AFFA3946FCF7A2F9814649462046FCF7E0
:10BC00009DF9039BC0F3C7529B1A192B074641DCD1
:10BC10002860A046C1E7FCF793F9304B24F00F04ED
:10BC20009C42064623D02E49FCF78AF9014628603B
:10BC30003046FCF783F92A49FCF782F94FF0FF33CD
:10BC400068605EE795E80C0003F1004102F10042F4
:10BC500043422A60696054E7032340E707F1004745
:10BC600000F100402F606860CAF1000349E71F49F6
:10BC7000FCF766F91E490446FCF762F901462860A4
:10BC80002046FCF75BF91A49FCF75AF94FF0FF33ED
:10BC9000686036E719495846FCF75AFA07463946AC
:10BCA0002046FCF74BF9804641462046FCF746F912
:10BCB0003946FCF743F9124904465846FCF748FA5E
:10BCC0002146FCF73BF981464946404661E700BF03
:10BCD000D80F493FE3CB1640800FC93FD00FC93F73
:10BCE00043443537800F4943DCF0000800443537C2
:10BCF00008A3852E84F9223F5CF0000800A3852E5E
:10BD000032318D2420F00042B2F1FF4FF8B50446E5
:10BD100003462DD25AB300283DDBB2F5000F4FEA9F
:10BD2000E0502CD37F38C3F31603C20743F400035B
:10BD300048BF5B00002740105B003E4619244FF0CF
:10BD40008072B5189D4202DC5B1BAE181744013CA3
:10BD50004FEA43034FEA5202F3D113B107F0010354
:10BD60001F447F1007F17C5707EBC050F8BDF8BDAA
:10BD70000146FCF7EDF92146FCF7E2F8F8BD14F4B2
:10BD800000020FD15B00190202F10102FAD5C2F1E3
:10BD900001021044C6E70146FCF7D0F80146FCF763
:10BDA0008BFAF8BD01221044BCE700BF2DE9F8432F
:10BDB00020F00046B6F1485F05460F4649DAFCF729
:10BDC0008DFB002800F09D8029462846FCF7C0F92D
:10BDD0004E490446FCF7BCF94D49FCF7B1F8214641
:10BDE000FCF7B6F94B49FCF7A9F82146FCF7B0F986
:10BDF0004949FCF7A5F82146FCF7AAF94749FCF7A1
:10BE00009DF82146FCF7A4F94549FCF799F821462D
:10BE1000FCF79EF9804620464FF07C51FCF798F9DC
:10BE2000414606462046FCF793F939460446284623
:10BE3000FCF78EF901462046FCF780F801463046B3
:10BE4000FCF77CF801464FF07E50FCF777F8BDE830
:10BE5000F8830146FCF77CF92C490446FCF778F995
:10BE60002B49FCF76DF82146FCF772F92949FCF7DC
:10BE700065F82146FCF76CF92749FCF761F8214683
:10BE8000FCF766F92549FCF759F82146FCF760F9FB
:10BE90002349FCF755F82146FCF75AF9214B804617
:10BEA0009E42B8DD204B9E4227DC06F17F4631469C
:10BEB0004FF07E50FCF742F8814620464FF07C510F
:10BEC000FCF746F93146FCF739F84146064620466C
:10BED000FCF73EF9394604462846FCF739F9014695
:10BEE0002046FCF72BF801463046FCF727F80146C0
:10BEF0004846FCF723F8BDE8F883DFF834900B4E92
:10BF0000DBE74FF07E50BDE8F88300BF4ED747AD6A
:10BF1000F6740F317CF29334010DD037610BB63AD1
:10BF2000ABAA2A3D9999993E0000483F0000903EF7
:10BF30000000383F2DE9F04FDFB00B93013B029337
:10BF4000D31E48BF131DB84C06466898DB1054F842
:10BF5000204023EAE3730C93DB4302EBC303089412
:10BF60000693089C029B0C9A1D190991C3EB0207CA
:10BF70001DD4699C3D4404EB870901354FF000084E
:10BF800022AC0AE059F80800FCF78EF80137AF42FE
:10BF900044F8080008F1040809D0002FF2DA01374C
:10BFA0000020AF4244F8080008F10408F5D1089ACF
:10BFB000002AC0F2DF82089A0B9B02F101089C0064
:10BFC00022AF4FEA880827440025029A002AC0F2CF
:10BFD000F28105EB070B4FF000094FF0000A56F80D
:10BFE00009005BF8041DFCF7B3F801465046FBF767
:10BFF000A7FF09F10409A1458246F0D14AA840F8FB
:10C0000005A004354545E0D1089A0EAB03EB820349
:10C010000D9391464FEA89030793079A5EAB134449
:10C02000B9F1000F53F850AC23DD0DF134084AAFDD
:10C03000174490440DAD4FF06E515046FCF788F810
:10C04000FCF74CFAFCF730F84FF087418346FCF7D9
:10C050007FF801465046FBF771FFFCF73FFA59465F
:10C0600045F8040F57F8040DFBF76AFF4545824673
:10C07000E1D15046069900F08DFC4FF0785105460D
:10C08000FCF766F800F026FC4FF08241FCF760F800
:10C0900001462846FBF752FF0546FCF71FFA824689
:10C0A000FCF702F801462846FBF748FF069A80464F
:10C0B000002A40F3678109F1FF310EA850F82130C2
:10C0C000C2F1080043FA00F202FA00F01B1A0698C7
:10C0D0009244C0F1070743FA07F70EA840F8213051
:10C0E000002F32DDB9F1000F0AF1010A40F375812A
:10C0F0000EAB079A19461144002507E0C2F580707F
:10C1000012B143F8040C01258B420BD053F8042BD9
:10C11000002DF3D0C2F1FF028B4243F8042C4FF004
:10C120000105F3D1069B002B0DDD012B00F03281C0
:10C13000022B08D109F1FF330EA951F8232002F098
:10C140003F0241F82320022F70D040460021FCF727
:10C1500093F9002800F08380089A09F1FF35AA427C
:10C160000DDC079A0EAB0D981344002253F8041D02
:10C17000834242EA0102F9D1002A40F0E481089B9F
:10C180000EA85A1E50F82230002B40F0F18100EB2F
:10C190008202012352F8041D01330029FAD04B44D6
:10C1A00099450A933DDADDF82CA022AACA44DDF8AD
:10C1B000308002EB8A02C844C9EB0309131D0392C5
:10C1C0000593699A079B4FEA89094AAF02EB8808F1
:10C1D000CDF810901F44002558F8040FFBF764FFBA
:10C1E000029B039A002B50514FF0000B13DBDDF83C
:10C1F00014A04FF00009AA4456F809005AF8041D8B
:10C20000FBF7A6FF01465846FBF79AFE09F1040921
:10C21000A1458346F0D1049A0435954247F804BFFE
:10C22000DAD1DDF82890F5E6F4F3000841464FF046
:10C230007E50FBF783FE8046002D86D006994FF096
:10C240007E5000F0A7FB01464046FBF777FE804694
:10C2500040460021FCF710F900287FF47DAF069BD3
:10C2600040465942CDF808A000F094FB4FF08741BA
:10C270000446FCF71FF9002800F07F814FF06E5153
:10C280002046FBF765FFFCF729F9FBF70DFF4FF0A0
:10C2900087410546FBF75CFF01462046FBF74EFE53
:10C2A000FCF71CF90EAB43F829002846FCF716F9F9
:10C2B000069C09F1010508340EA9069441F82500F1
:10C2C00006994FF07E5000F065FB002D04464FDBD1
:10C2D0006E1C4FEA8508C6EB867A0DF138094AAB29
:10C2E000C1444FEA8A0A98444FF0000B59F80B00FA
:10C2F000FBF7DAFE2146FBF72BFF4FF06E5148F8B3
:10C300000B002046FBF724FFABF1040BD34504469A
:10C31000ECD1DFF88C92DDF820A00024B346039521
:10C320000497BAF1000FB8BF002515DB0026374689
:10C33000002501E0A7420FDC58F8061059F8060066
:10C34000FBF706FF01462846FBF7FAFD0137BA4521
:10C35000054606F10406EDDA5EA800EB840301341D
:10C36000A345A8F1040843F8A05CDAD1039D049F1B
:10C37000689C032C00F29880DFE814F0CB009C004E
:10C380009C00310010D109F1FF330EA951F8237040
:10C390003F12A5E609F1FF330EA850F8232002F062
:10C3A0007F0240F82320CEE64FF07C51FCF782F864
:10C3B00058B90746C9E64FF0000A4AA840F805A058
:10C3C000043545457FF401AE1EE6B9F1000F4FF08C
:10C3D00002070AF1010A3FF78BAE0025A2E6002D05
:10C3E00040F3DC804FEA850B5EAB36AE05F1FF3AD9
:10C3F0005B4406EB8A0A53F8A08C54465B4635AA88
:10C40000BB462F4600E0C84654F80459414628462A
:10C4100001920093FBF794FD814649462846FBF7BD
:10C420008DFD4146FBF78CFD019AC4F804909442BF
:10C43000A060009BE7D13D46012D5F469B4640F33F
:10C44000AD805EAB9B445BF8A04C00E044465AF8DC
:10C45000049921464846FBF773FD8046414648460D
:10C46000FBF76CFD2146FBF76BFD5645CAF80480CF
:10C47000CAF80800EAD16C1C06EB840400200836D8
:10C4800054F8041DFBF75CFDB442F9D1002F7ED0B7
:10C49000369A379B099C00F1004002F1004203F1FB
:10C4A0000043A06022606360029A02F007005FB060
:10C4B000BDE8F08F002DB8BF00200ADB36AE6C1C43
:10C4C000002006EB840454F8041DFBF739FDB44248
:10C4D000F9D1002F35D000F10043099C01462360BB
:10C4E0003698FBF72BFD002D08DD36AC04EB8505F7
:10C4F00054F8041FFBF724FDAC42F9D10FB100F151
:10C500000040099A5060029A02F007005FB0BDE84F
:10C51000F08F002D39DB6C1C36AE002006EB840456
:10C5200054F8041DFBF70CFDB442F9D10FB100F132
:10C530000040099A1060029A02F007005FB0BDE85F
:10C54000F08F0346C9E7069A0EAC54F82530083A36
:10C55000CDF808A00692002B7FF4B2AE04EB850361
:10C5600053F8041D013D083A0029F9D00692A7E6C8
:10C57000012314E60B9B9C0046E52046FBF7AEFF2B
:10C580000EAA4D4642F829009AE60020CEE7099C03
:10C59000369A379BA0602260636085E7002075E7CC
:10C5A00000F400082DE9F84320F00043B3F1485FA0
:10C5B00004460F46904603DAFBF790FF002857D059
:10C5C00021462046FBF7C4FD21460546FBF7C0FD8A
:10C5D000294906462846FBF7BBFD2849FBF7AEFC78
:10C5E0002946FBF7B5FD2649FBF7AAFC2946FBF7D0
:10C5F000AFFD2449FBF7A2FC2946FBF7A9FD224920
:10C60000FBF79EFC8146B8F1000F22D038464FF070
:10C610007C51FBF79DFD494680463046FBF798FD6F
:10C6200001464046FBF78AFC2946FBF791FD394657
:10C63000FBF784FC154905463046FBF789FD0146AA
:10C640002846FBF77DFC01462046FBF777FCBDE85A
:10C65000F88349462846FBF77BFD0C49FBF76EFC47
:10C660003146FBF775FD2146FBF76AFCBDE8F88310
:10C670002046BDE8F88300BFD3C92E2F342FD73210
:10C680001BEF3836010D50398988083CABAA2A3E89
:10C690000020704700200149704700BF0000F87F6C
:10C6A0002DE9F04120F00045B5F1A14F04460646C2
:10C6B00008DBB5F1FF4F6FDC002840F3A0806F4826
:10C6C000BDE8F0816E4B9D4277DCB5F1445F68DBDD
:10C6D0004FF0FF3721462046FBF73AFD01468046E2
:10C6E000FBF736FD67490546FBF732FD6649FBF768
:10C6F00027FC2946FBF72CFD6449FBF721FC294662
:10C70000FBF726FD6249FBF71BFC2946FBF720FDE2
:10C710006049FBF715FC2946FBF71AFD5E49FBF75C
:10C720000FFC4146FBF714FD5C4980462846FBF7A9
:10C730000FFD5B49FBF702FC2946FBF709FD594950
:10C74000FBF7FCFB2946FBF703FD5749FBF7F6FB1C
:10C750002946FBF7FDFC5549FBF7F0FB2946FBF7A3
:10C76000F7FC7B1C014640464CD0FBF7E9FB214619
:10C77000FBF7EEFC4E4B4F4D53F82710FBF7DEFB5B
:10C780002146FBF7DBFB014655F82700FBF7D6FBFC
:10C79000002E30DBBDE8F0810146FBF7D1FBBDE8A0
:10C7A000F0814549FBF7CCFB4FF07E51FBF78CFE47
:10C7B00000288DD02046BDE8F08100F087F83F4B7F
:10C7C00004469D4229DCA3F5D0039D4244DC01468A
:10C7D000FBF7B6FB4FF07E51FBF7B0FB4FF080410B
:10C7E00005462046FBF7ACFB01462846FBF764FDF7
:10C7F000002704466EE700F10040BDE8F0813048B4
:10C80000BDE8F081FBF79CFB2146FBF7A1FC01464C
:10C810002046FBF793FBBDE8F0812A4B9D4214DCD8
:10C820004FF07F51FBF78AFB4FF07F5105462046C2
:10C83000FBF78EFC4FF07E51FBF782FB014628464A
:10C84000FBF73AFD0227044644E701461E48FBF782
:10C8500033FD032704463DE74FF07E51FBF76EFBA7
:10C860004FF07E5105462046FBF76AFB01462846FD
:10C87000FBF722FD012704462CE700BFDB0FC93F71
:10C88000FFFFDF3ED769853C59DA4B3D356B883D6C
:10C890006E2EBA3D2549123EABAAAA3E21A215BD75
:10C8A0006BF16E3D95879D3D388EE33DCDCC4C3E82
:10C8B0002CF400083CF40008CAF24971FFFF973FCE
:10C8C000DB0FC9BFFFFF1B40000080BF20F000400E
:10C8D000704700BF2DE9F04120F00047FD0D7F3D7E
:10C8E000162D064613DC002D80461BDB194F2F4109
:10C8F000074214D01849FBF723FB0021FBF7E4FDA6
:10C9000068B1002E1BDB28EA0700BDE8F081B7F113
:10C91000FF4F04D30146FBF713FBBDE8F08130461F
:10C92000BDE8F0810C49FBF70BFB0021FBF7CCFDC8
:10C930000028F4D0002E08DB0020BDE8F0814FF481
:10C94000000343FA05F5A844DDE7002FE7D00348CC
:10C95000BDE8F081FFFF7F00CAF24971000080BF8F
:10C9600030F0004001D102207047A0F50003B3F180
:10C97000FE4F01D204207047054B421E9A4201D857
:10C9800003207047B0F1FF4358425841704700BF41
:10C99000FEFF7F0038B530F00044024603460D46E6
:10C9A00014D0B4F1FF4F0DD2B4F5000F0FD3E40D46
:10C9B0002C44FE2C2EDC002C1DDD23F0FF4343EA2B
:10C9C000C45038BD0146FBF7BBFA38BD38BD4FF047
:10C9D0009841FBF7BDFB194B02469D4207DBC0F3B4
:10C9E000C7540346193CE3E7154800F02DF81449F5
:10C9F000FBF7AEFB38BD14F1160F13DA4CF25033CF
:10CA00009D421146F0DD0F4800F01EF80D49FBF77E
:10CA10009FFB38BD11460B4800F016F80949FBF79B
:10CA200097FB38BD04F1190023F0FF4343EAC050DF
:10CA30004FF04C51FBF78CFB38BD00BFB03CFFFF03
:10CA40006042A20DCAF2497101F0004120F000409D
:10CA500008437047014B1868704700BFEC00002086
:10CA6000524F4C4C3B50495443483B5941573B4132
:10CA70004C543B506F733B506F73523B4E61765238
:10CA80003B4C4556454C3B4D41473B56454C3B0086
:10CA900000000000BADD00080000000001000000F6
:10CAA000BFDD00080100000002000000C6DD000834
:10CAB0000200000003000000CFDD000803000000BA
:10CAC00004000000D5DD000805000000050000009E
:10CAD000DADD00080600000006000000E4DD0008C2
:10CAE0000700000007000000EDDD0008080000005E
:10CAF00008000000F6DD0008090000000900000041
:10CB0000FFDD00080A0000000A00000009DE00083E
:10CB10000B0000000B00000013DE00080C000000FA
:10CB20000C0000001DDE00080D0000000D000000DC
:10CB300025DE00080E0000000E0000002DDE0008BB
:10CB40000F0000000F00000035DE0008100000009C
:10CB5000100000003EDE000811000000110000007F
:10CB600045DE000812000000120000004FDE000841
:10CB7000130000001300000057DE0008140000003E
:10CB80001400000062DE000815000000150000001F
:10CB90006CDE000816000000160000000000000017
:10CBA000FF000000ADDD0008A4DD000898DD0008EE
:10CBB000001001400020100200100140004010024F
:10CBC00000000000000000000301000018D1000870
:10CBD00004000000D8D000080400000098D000082D
:10CBE0000201000078D000080001000000000000F1
:10CBF0000600000018D0000806000000B8CF0008AA
:10CC000001010000000000000400000078CF0008CF
:10CC10000600000018CF00080800000098CE0008A9
:10CC20000800000018CE00080800000098CD000899
:10CC300001010000000000000001000000000000F1
:10CC400000010000000000000400000058CD0008B2
:10CC500006000000F8CC0008000100000000000001
:10CC600002010000D8CC0008010100000000000013
:10CC70000000000000000000C0CC0008B4CC000898
:10CC8000B2CC0008B0CC000819170008D51600086F
:10CC9000B1160008891600087916000879240008E2
:10CCA0000517000821160008F9160008EB16000801
:10CCB000FFFFFFFF000106030D0307030C03FFFF47
:10CCC00000020102020203020802090206030D0328
:10CCD00007030C03FFFF00000000803F000000007E
:10CCE00000000000000080BF0000803F0000000046
:10CCF000000000000000803F0000803F000080BF77
:10CD00000000803F000080BF0000803F000080BF27
:10CD1000000080BF0000803F0000803F0000803F97
:10CD20000000803F0000803F0000803F0000803F07
:10CD3000000080BF000080BF0000803F00000000B6
:10CD400000000000000000000000803F0000000024
:10CD500000000000000000000000803F0000000014
:10CD60000000803F0000803F0000803F000080BF47
:10CD7000000080BF000000000000803F00000000B5
:10CD80000000803F000080BF0000803F0000803F27
:10CD9000000080BF000000800000803F0000803F56
:10CDA000000000BF0000803F0000803F000000BF87
:10CDB000000080BF0000803F0000803F000080BF77
:10CDC0000000003F0000803F0000803F0000003F67
:10CDD0000000803F0000803F0000803F0000003FD7
:10CDE000000080BF000080BF0000803F000080BFC7
:10CDF000000000BF000080BF0000803F000000BFB7
:10CE00000000803F000080BF0000803F0000803FA6
:10CE10000000003F000080BF0000803FF704353F66
:10CE2000F70435BF0000803F0000803FF70435BFA6
:10CE3000F70435BF0000803F0000803FF70435BF96
:10CE4000F704353F0000803F0000803FF704353F86
:10CE5000F704353F0000803F0000803F00000000E5
:10CE6000000080BF000080BF0000803F000080BF46
:10CE700000000000000080BF0000803F00000000B4
:10CE80000000803F000080BF0000803F0000803F26
:10CE900000000000000080BF0000803F000080BF55
:10CEA0000000803F000080BF0000803F000080BF86
:10CEB000000080BF0000803F0000803F0000803FF6
:10CEC0000000803F0000803F0000803F0000803F66
:10CED000000080BF000080BF0000803F000080BFD6
:10CEE0000000803F0000803F0000803F000080BFC6
:10CEF000000080BF000080BF0000803F0000803F36
:10CF00000000803F000080BF0000803F0000803FA5
:10CF1000000080BF0000803F0000803F000000BF95
:10CF2000D0B35D3F0000803F0000803F000000BFA5
:10CF3000D0B35DBF0000803F0000803F0000003F95
:10CF4000D0B35D3F000080BF0000803F0000003F85
:10CF5000D0B35DBF000080BF0000803F000080BFF5
:10CF600000000000000080BF0000803F0000803F04
:10CF7000000000000000803F0000803F0000000033
:10CF80000000803F000080BF0000803F000080BFA5
:10CF9000000080BF000000000000803F0000000093
:10CFA0000000803F0000803F0000803F0000803F85
:10CFB000000080BF000000000000803FD0B35DBFD4
:10CFC0000000003F0000803F0000803FD0B35DBF05
:10CFD000000000BF000080BF0000803FD0B35D3F75
:10CFE0000000003F0000803F0000803FD0B35D3F65
:10CFF000000000BF000080BF0000803F0000000074
:10D00000000080BF0000803F0000803F0000000063
:10D010000000803F000080BF0000803F0000000053
:10D02000A8AAAA3F0000803F0000803F000080BF08
:10D03000B0AA2ABF000080BF0000803F0000803FF0
:10D04000B0AA2ABF000080BF0000803F000000009F
:10D05000A8AAAA3F000080BF0000803F000080BF58
:10D06000B0AA2ABF0000803F0000803F0000803F40
:10D07000B0AA2ABF0000803F0000803F0000803F30
:10D0800000000000000000000000803F000080BFA2
:10D0900000000000000000000000803F000080BF92
:10D0A0000000803F000080BF0000803F000080BF84
:10D0B000000080BF0000803F0000803F0000803FF4
:10D0C0000000803F0000803F0000803F0000803F64
:10D0D000000080BF000080BF0000803F0000000013
:10D0E0000000803F000080BF0000803F000080BF44
:10D0F000000000000000803F0000803F0000803FF3
:10D10000000000000000803F0000803F00000000A1
:10D11000000080BF000080BF0000803F00000000D2
:10D12000A8AAAA3F000000000000803F000080BFC6
:10D13000B0AA2ABF000000000000803F0000803F2E
:10D14000B0AA2ABF000000000000000080250000F7
:10D1500000C2010006000000010000008025000060
:10D1600000C20100070000000100010200010300ED
:10D17000010400010500010600010700010800018B
:10D180000900010A00010B00010C010341E2000843
:10D1900046E200084AE200085DE200084FE20008AB
:10D1A00055E2000859E2000800000000D5E100083F
:10D1B000F5E10008FDE1000805E200080DE20008C5
:10D1C00014E200081FE2000827E200082FE200082E
:10D1D00037E200083CE200080000000067E20008B7
:10D1E0006BE2000871E2000877E200087AE20008CA
:10D1F00081E2000884E2000889E2000895E2000864
:10D2000098E200089EE20008A5E20008AFE20008EC
:10D21000B9E20008C2E20008D0E20008DCE200083F
:10D22000E3E20008E9E20008F6E2000801E3000892
:10D230000EE30008000000001E1E64646464646461
:10D240009001C800C800C800C800C800C800C800D5
:10D25000C80064000000C800C800C800C800320050
:10D26000020000008025000000C201000000000054
:10D27000200000008025000000C201000100000025
:10D28000400000008025000000C2010000000000F6
:10D29000010000008025000000C201000000000025
:10D2A000100000008025000000C201000003000003
:10D2B0000400000080250000004B0000000000007A
:10D2C0000800000000E1000000E100000004000090
:10D2D000ED6B00085517000825170008055B0008CE
:10D2E00077170008015B000857E500085EE50008B5
:10D2F00063E5000874E500087EE5000889E500089C
:10D3000094E5000855E200089FE500084FE2000898
:10D31000A8E50008B2E50008C0E50008C3E500087C
:10D32000D3E50008DAE50008E3E50008EDE50008CC
:10D33000F5E5000800000000B0E30008B9E30008CC
:10D340007D6A0008DDE30008E1E300089569000854
:10D35000F7E30008FCE300085D660008ECE1000864
:10D3600010E400082D3F00082DE4000832E4000816
:10D370004937000861E40008D5E10008357100086C
:10D3800066E400086EE400086D5E000882E40008B0
:10D3900086E40008C963000899E40008D5E10008A4
:10D3A000A93300089EE40008A2E40008B96500085B
:10D3B0000AE40008BEE400085D620008D1E4000849
:10D3C000D7E40008ED680008EDEC0008F2E400087E
:10D3D000FD36000801E50008F2E400087932000893
:10D3E0000DE5000812E50008C56F000830E70008E9
:10D3F00022E500082564000850E5000844E500081F
:10D40000D1320008B3EA0008D5E10008493200082B
:10D4100000540040000C0140400080001F2000002C
:10D420000000200000580040000C014000040008EB
:10D430002122000000004000E6E80008440000004F
:10D44000B01000200000000028230000EFE80008D2
:10D4500041000000B21000200000000001000000A8
:10D46000FDE8000844000000BE110020B0040000E8
:10D47000A406000004E9000844000000C0110020D8
:10D4800000000000D00700000EE900084400000082
:10D49000C211002000000000D007000018E90008B9
:10D4A00042000000C4110020000000001200000033
:10D4B00025E9000842000000C5110020010000001D
:10D4C000FF00000030E9000842000000C611002003
:10D4D000000000000100000045E9000844000000D1
:10D4E0007411002000000000D007000052E900087D
:10D4F000440000007611002000000000D00700006A
:10D500005FE90008440000007811002000000000DE
:10D51000D00700006BE90008440000007A110020E9
:10D5200000000000D00700007BE900084400000074
:10D530007C11002000000000D00700008CE90008EA
:10D54000440000007E11002000000000D007000011
:10D5500097E900084400000080110020000000004E
:10D56000D0070000ACE90008440000008211002050
:10D5700032000000007D0000BBE90008440000000C
:10D580008411002032000000F2010000CAE9000806
:10D5900041000000C7110020000000000100000051
:10D5A000D7E9000841000000C81100200000000079
:10D5B00001000000EAE9000841000000C911002054
:10D5C00000000000B4000000F6E90008410000007F
:10D5D000CA110020000000006400000002EA0008F8
:10D5E00042000000CB110020FFFFFFFF0100000000
:10D5F00018EA000841000000CC11002000000000E3
:10D60000090000002FEA000841000000CD110020B1
:10D61000000000000900000046EA00084100000088
:10D62000E0110020300000007E00000057EA0008F2
:10D6300050000000D0110020B004000000C2010022
:10D6400064EA000850000000D4110020B00400007B
:10D6500000C2010071EA000841000000BC11002076
:10D66000000000000300000083EA00084100000001
:10D67000E4110020000000000300000096EA00080A
:10D6800041000000E5110020000000000100000042
:10D69000A7EA000841000000E61100200000000099
:10D6A00001000000BBEA000860000000E811002053
:10D6B000A6FFFFFF5A000000D3EA00086000000048
:10D6C000EC1100204CFFFFFFB4000000EBEA000863
:10D6D00041000000F01100200000000001000000E7
:10D6E00004EB000841000000F111002000000000E0
:10D6F000010000000FEB000844000000B211002000
:10D7000000000000204E000020EB00084100000057
:10D71000A811002000000000FF0000002BEB000813
:10D7200041000000A91100200A00000032000000A2
:10D7300041EB000841000000AA1100200A0000008F
:10D740003200000057EB000844000000AC1100203C
:10D7500001000000102700006BEB000844000000EF
:10D76000AE110020000000007206000080EB0008EF
:10D7700041000000B0110020000000000100000086
:10D780009EEB000841000000861100200000000010
:10D7900008000000A9EB00084100000087110020EC
:10D7A0000000000008000000B3EB0008410000008A
:10D7B000881100200000000008000000BDEB0008F8
:10D7C000480000008A1100204CFFFFFF68010000A4
:10D7D000CEEB0008480000008C1100204CFFFFFF3A
:10D7E00068010000E0EB0008480000008E110020F6
:10D7F0004CFFFFFF68010000F0EB00084400000050
:10D800009A110020640000008403000006EC000868
:10D810004400000092110020000000000001000000
:10D820000FEC0008410000009811002000000000EB
:10D83000800000001FEC000844000000941100204C
:10D8400064000000E803000030EC00084400000021
:10D850009611002064000000E803000042EC00087C
:10D86000810000005313002001000000FA000000B6
:10D8700054EC000881000000541300200000000058
:10D88000010000004BEC0008810000005113002053
:10D89000000000002000000069EC0008810000008A
:10D8A00052130020000000006400000076EC000825
:10D8B00081000000581300200000000096000000C6
:10D8C00090EC0008840000005613002001000000C6
:10D8D00084030000AAEC0008420000009011002020
:10D8E000FFFFFFFF01000000C0EC00088200000005
:10D8F000A2130020FFFFFFFF01000000CEEC000894
:10D9000082000000A31300200000000001000000BE
:10D91000E0EC00088100000044120020000000003C
:10D9200002000000F5EC00080101000012170020C1
:10D9300000000000FA000000FDEC000801010000FA
:10D9400013170020000000006400000005ED00082F
:10D950000101000014170020000000006400000016
:10D960000DED000801010000151700200000000067
:10D970006400000016ED00080101000016170020E9
:10D98000000000006400000026ED00080101000016
:10D990001717002000000000640000002FED0008B1
:10D9A00001010000181700200000000064000000C2
:10D9B00038ED0008040100001A170020E8030000F9
:10D9C000D007000047ED0008810000009A130020F6
:10D9D00000000000C800000056ED000881000000B3
:10D9E0009B13002000000000C800000069ED000843
:10D9F000840000009C130020E8030000D007000012
:10DA00007BED0008840000009E13002064000000ED
:10DA1000D00700008DED000884000000A013002056
:10DA200064000000B80B00009FED000881000000BA
:10DA3000A413002000000000FF000000ACED00086F
:10DA40004100000091110020000000000A000000C9
:10DA5000B9ED0008810000004C1200200000000019
:10DA6000FA000000C8ED00088100000054120020F8
:10DA70000000000064000000D7ED000881000000F5
:10DA8000551200200000000064000000E5ED0008D1
:10DA9000A00000005012002001000000140000004F
:10DAA000F5ED000881000000681200200000000071
:10DAB0000100000004EE0008880000004A12002067
:10DAC000D4FEFFFF2C01000013EE000888000000C8
:10DAD00048120020D4FEFFFF2C01000021EE0008B8
:10DAE00081000000581200200000000030000000FB
:10DAF0002FEE0008A00000005C12002000000000D3
:10DB0000010000003EEE0008A000000060120020AE
:10DB100000000000010000004AEE0008A000000024
:10DB200064120020000000000100000056EE000812
:10DB30008800000046120020B0B9FFFF50460000E8
:10DB400066EE000881000000F411002000000000D3
:10DB50000200000075EE000881000000F9110020AD
:10DB600000000000C80000007DEE000881000000F9
:10DB70000312002000000000C8000000D8EB0008DD
:10DB8000810000000D12002000000000C80000000D
:10DB900085EE000881000000F81100200000000060
:10DBA000C80000008CEE0008810000000212002076
:10DBB00000000000C8000000C7EB00088100000062
:10DBC0000C12002000000000C800000093EE0008C6
:10DBD00081000000FA11002000000000C8000000D1
:10DBE00099EE0008810000000412002000000000EF
:10DBF000C8000000EAEB0008810000000E120020BF
:10DC000000000000C80000009FEE0008A000000017
:10DC10001C1200200000000064000000A8EE0008B4
:10DC2000A000000028120020000000006400000096
:10DC3000B1EE0008A0000000341200200000000037
:10DC400064000000BAEE0008A000000018120020D6
:10DC50000000000064000000C2EE0008A000000008
:10DC6000241200200000000064000000CAEE00083A
:10DC7000A00000003012002000000000640000003E
:10DC8000D2EE0008A00000002012002000000000DA
:10DC900064000000D9EE0008A00000002C12002053
:10DCA0000000000064000000E0EE0008A00000009A
:10DCB000381200200000000064000000E7EE0008B9
:10DCC000A000000040120020000000000A00000038
:10DCD000F5EE0008A00000003C120020000000004B
:10DCE0000A00000001EF000881000000FB11002085
:10DCF00000000000C800000007EF000881000000DD
:10DD00000512002000000000C80000000DEF000810
:10DD1000810000000F12002000000000C800000079
:10DD200013EF000881000000FF1100200000000038
:10DD3000C80000001BEF000881000000091200204D
:10DD400000000000C800000023EF00088100000070
:10DD50001312002000000000C80000002BEF000894
:10DD6000810000000112002000000000C800000037
:10DD700031EF0008810000000B12002000000000BD
:10DD8000C800000037EF00088100000015120020D5
:10DD900000000000C80000004465632031342032D8
:10DDA0003031340032333A35363A34310063353964
:10DDB0003562663800434A4D310041524D3B0041C7
:10DDC0004E474C453B00484F52495A4F4E3B00424C
:10DDD00041524F3B004D41473B004845414446526C
:10DDE00045453B004845414441444A3B0043414D81
:10DDF000535441423B0043414D545249473B004735
:10DE0000505320484F4D453B0047505320484F4CFE
:10DE1000443B0050415353544852553B0042454502
:10DE20005045523B004C45444D41583B004C454405
:10DE30004C4F573B004C4C49474854533B004341DF
:10DE40004C49423B00474F5645524E4F523B004FC4
:10DE500053442053573B0054454C454D455452596B
:10DE60003B004155544F54554E453B00534F4E4196
:10DE7000523B00000000004000080140010000008B
:10DE8000001C0028000000400008014002000000C3
:10DE9000041C0028000000400008014004000000AD
:10DEA000081C002800000040000801400800000095
:10DEB0000C1C002800040040000801404000000045
:10DEC000001D002800040040000801408000000000
:10DED000041D002800040040000C01400100000067
:10DEE000081D002800040040000C01400200000052
:10DEF0000C1D0028002C014000080140000100001A
:10DF0000001B0128002C014000080140000800000F
:10DF10000C1B012800080040000C014040000000DC
:10DF2000001E002800080040000C01408000000096
:10DF3000041E002800080040000C01400001000001
:10DF4000081E002800080040000C014000020000EC
:10DF50000C1E0028303132333435363738394142DF
:10DF6000434445464748494A4B4C4D4E4F50515209
:10DF7000535455565758595A00004F201004430225
:10DF8000400108436C65616E666C696768742F2593
:10DF900073202573202F20257320282573290072D4
:10DFA00061746570726F66696C652025640D0A0086
:10DFB00053797374656D20557074696D653A2025C9
:10DFC00064207365636F6E64732C20566F6C74618C
:10DFD00067653A202564202A20302E3156202825D6
:10DFE00064532062617474657279290D0A0043508C
:10DFF000552025644D487A2C2064657465637465EA
:10E00000642073656E736F72733A2000257320006D
:10E0100041434348573A202573002E256300437936
:10E02000636C652054696D653A2025642C20493263
:10E0300043204572726F72733A2025642C20636FFF
:10E040006E6669672073697A653A2025640D0A0057
:10E05000417661696C61626C6520636F6D6D616EA4
:10E0600064733A0D0A0025730925730D0A006D616A
:10E0700073746572007261746573000D0A232076F3
:10E08000657273696F6E0D0A000D0A232064756D49
:10E0900070206D61737465720D0A000D0A23206D86
:10E0A000697865720D0A006D697865722025730DB7
:10E0B0000A00636D697820256400636D6978202506
:10E0C0006420302030203020300D0A000D0A0D0A67
:10E0D0002320666561747572650D0A00666561745A
:10E0E000757265202D25730D0A0066656174757261
:10E0F000652025730D0A000D0A0D0A23206D61703D
:10E100000D0A006D61702025730D0A000D0A232091
:10E1100064756D702070726F66696C650D0A000D14
:10E120000A232070726F66696C650D0A000D0A2360
:10E13000206175780D0A000D0A232061646A7261FE
:10E140006E67650D0A000D0A232064756D702072DC
:10E15000617465730D0A000D0A2320726174657085
:10E16000726F66696C650D0A000D0A456E74657202
:10E17000696E6720434C49204D6F64652C2074798B
:10E1800070652027657869742720746F2072657424
:10E1900075726E2C206F72202768656C70270D0ACF
:10E1A000000D0A2320000D1B5B4B001B5B324A1B3A
:10E1B0005B313B314800556E6B6E6F776E20636F3D
:10E1C0006D6D616E642C20747279202768656C70A7
:10E1D00027000820080041455452313233340052A0
:10E1E0006573657474696E6720746F206465666119
:10E1F000756C7473004144584C333435004D5055A0
:10E2000036303530004D4D413834357800424D417F
:10E21000323830004C534D333033444C4843004D7A
:10E22000505536303030004D505536353030004D79
:10E230005055393135300046414B45004E6F6E65C3
:10E24000004759524F00414343004241524F00534F
:10E250004F4E415200475053004750532B4D4147BA
:10E2600000434A4D435500545249005155414450D2
:10E270000051554144580042490047494D42414CE4
:10E28000005936004845583600464C59494E475FBC
:10E2900057494E47005934004845583658004F43B7
:10E2A000544F5838004F43544F464C415450004F40
:10E2B00043544F464C41545800414952504C414EF2
:10E2C000450048454C495F3132305F4343504D0073
:10E2D00048454C495F39305F4445470056544149F1
:10E2E0004C340048455836480050504D5F544F5FFD
:10E2F000534552564F004455414C434F505445529C
:10E300000053494E474C45434F50544552004355E6
:10E3100053544F4D00414552543132333435363722
:10E32000386162636465666768002E000D0A526595
:10E33000626F6F74696E6700456E61626C65642020
:10E3400066656174757265733A2000417661696C27
:10E3500061626C652066656174757265733A200050
:10E36000496E76616C6964206665617475726520BA
:10E370006E616D650D0A0047505320756E617661C0
:10E38000696C61626C650D0A00534F4E41522075F5
:10E390006E617661696C61626C650D0A0044697337
:10E3A00061626C65642000456E61626C656420008A
:10E3B00061646A72616E67650073686F772F736559
:10E3C000742061646A7573746D656E742072616E19
:10E3D0006765732073657474696E6773006175781F
:10E3E0000073686F772F736574206175782073658B
:10E3F0007474696E677300636D697800646573692E
:10E40000676E20637573746F6D206D697865720037
:10E41000726573657420746F2064656661756C74D1
:10E420007320616E64207265626F6F740064756D35
:10E4300070007072696E7420636F6E6669677572C2
:10E4400061626C652073657474696E677320696EB0
:10E450002061207061737461626C6520666F726DFB
:10E4600000657869740066656174757265006C6931
:10E470007374206F72202D76616C206F722076612C
:10E480006C0067657400676574207661726961620B
:10E490006C652076616C75650068656C70006D61F7
:10E4A00070006D617070696E67206F662072632006
:10E4B0006368616E6E656C206F72646572006D6971
:10E4C000786572206E616D65206F72206C6973745F
:10E4D000006D6F746F72006765742F736574206DC3
:10E4E0006F746F72206F75747075742076616C75BF
:10E4F0006500696E64657820283020746F203229A9
:10E50000007261746570726F66696C650073617624
:10E5100065007361766520616E64207265626F6F5D
:10E5200074006E616D653D76616C7565206F72205B
:10E53000626C616E6B206F72202A20666F72206C95
:10E540006973740073686F772073797374656D20D5
:10E550007374617475730052585F50504D00564289
:10E56000415400494E464C494748545F4143435F3C
:10E5700043414C0052585F53455249414C004D4F66
:10E58000544F525F53544F5000534552564F5F54AF
:10E59000494C5400534F465453455249414C004650
:10E5A00041494C534146450054454C454D45545214
:10E5B000590043555252454E545F4D455445520003
:10E5C00033440052585F504152414C4C454C5F50CF
:10E5D000574D0052585F4D535000525353495F41BD
:10E5E0004443004C45445F535452495000444953FE
:10E5F000504C4159004F4E4553484F54313235002D
:10E6000043757272656E74206D697865723A202563
:10E61000730D0A00417661696C61626C65206D69F9
:10E62000786572733A2000496E76616C6964206D7A
:10E630006978657220747970650D0A004D69786596
:10E64000722073657420746F2025730D0A002025D5
:10E650006420256400556E6B6E6F776E2076617254
:10E660006961626C65206E616D650D0A00437572AB
:10E6700072656E742073657474696E67733A200DE9
:10E680000A0025732073657420746F200056616C36
:10E6900075652061737369676E6D656E74206F7543
:10E6A00074206F662072616E67650D0A004D757388
:10E6B0007420626520616E79206F72646572206FCC
:10E6C000662041455452313233340D0A004375728D
:10E6D00072656E742061737369676E6D656E743AEE
:10E6E00020004E4709004F4B0900437573746F6D4E
:10E6F000206D697865723A200D0A4D6F746F72094A
:10E7000054687209526F6C6C0950697463680959D6
:10E7100061770D0A002325643A0900257309005327
:10E72000616E69747920636865636B3A090072658C
:10E73000736574006C6F6164004C6F616465642084
:10E740002573206D69780D0A0057726F6E67206E11
:10E75000756D626572206F6620617267756D656E9A
:10E7600074732C206E656564732069647820746806
:10E770007220726F6C6C20706974636820796177A5
:10E780000D0A004D6F746F72206E756D6265722098
:10E790006D757374206265206265747765656E209F
:10E7A0003120616E642025640D0A00557361676530
:10E7B0003A0D0A6D6F746F7220696E646578205B24
:10E7C00076616C75655D202D2073686F77205B6FB7
:10E7D00072207365745D206D6F746F722076616C4A
:10E7E00075650D0A004E6F2073756368206D6F7438
:10E7F0006F722C207573652061206E756D62657275
:10E80000205B302C2025645D0D0A004D6F746F7203
:10E810002025642069732073657420617420256449
:10E820000D0A00496E76616C6964206D6F746F72B9
:10E830002076616C75652C20313030302E2E3230D0
:10E8400030300D0A0053657474696E67206D6F7403
:10E850006F7220256420746F2025640D0A00617595
:10E86000782025752025752025752025752025758E
:10E870000D0A00696E6465783A206D7573742062C4
:10E8800065203C2025750D0A0061646A72616E671F
:10E890006520257520257520257520257520257571
:10E8A0002025752025750D0A0073657420257320B9
:10E8B0003D2000536176696E67000D0A4C656176F4
:10E8C000696E6720434C49206D6F64652C20756E1E
:10E8D0007361766564206368616E676573206C6F31
:10E8E00073742E0D0A006C6F6F7074696D6500652E
:10E8F0006D665F61766F6964616E6365006D696402
:10E900005F7263006D696E5F636865636B006D6164
:10E91000785F636865636B00727373695F636861D6
:10E920006E6E656C00727373695F7363616C650012
:10E93000696E7075745F66696C746572696E675F25
:10E940006D6F6465006D696E5F7468726F74746C6E
:10E9500065006D61785F7468726F74746C65006DCA
:10E96000696E5F636F6D6D616E640033645F6465D3
:10E97000616462616E645F6C6F770033645F6465CD
:10E98000616462616E645F686967680033645F6ECA
:10E9900065757472616C0033645F646561646261A3
:10E9A0006E645F7468726F74746C65006D6F746F01
:10E9B000725F70776D5F7261746500736572766FF8
:10E9C0005F70776D5F726174650072657461726407
:10E9D00065645F61726D0064697361726D5F6B691C
:10E9E0006C6C5F73776974636800736D616C6C5FE6
:10E9F000616E676C6500666C6170735F73706565EE
:10EA00006400666978656477696E675F616C7468D5
:10EA10006F6C645F6469720073657269616C5F70CA
:10EA20006F72745F315F7363656E6172696F0073DB
:10EA3000657269616C5F706F72745F325F7363657A
:10EA40006E6172696F007265626F6F745F63686197
:10EA5000726163746572006D73705F626175647278
:10EA600061746500636C695F62617564726174658D
:10EA70000073657269616C72785F70726F76696439
:10EA800065720074656C656D657472795F70726F24
:10EA900076696465720074656C656D657472795F22
:10EAA0007377697463680074656C656D65747279F9
:10EAB0005F696E76657273696F6E006672736B79EB
:10EAC0005F64656661756C745F6C6174746974759C
:10EAD0006465006672736B795F64656661756C74FA
:10EAE0005F6C6F6E676974756465006672736B79CD
:10EAF0005F636F6F7264696E617465735F666F7276
:10EB00006D6174006672736B795F756E6974006213
:10EB10006174746572795F636170616369747900AF
:10EB2000766261745F7363616C6500766261745FC5
:10EB30006D61785F63656C6C5F766F6C746167653F
:10EB400000766261745F6D696E5F63656C6C5F76A1
:10EB50006F6C746167650063757272656E745F6D6A
:10EB6000657465725F7363616C650063757272656D
:10EB70006E745F6D657465725F6F66667365740051
:10EB80006D756C74697769695F63757272656E74AF
:10EB90005F6D657465725F6F757470757400616C1C
:10EBA00069676E5F6779726F00616C69676E5F613C
:10EBB000636300616C69676E5F6D616700616C69BA
:10EBC000676E5F626F6172645F726F6C6C00616C24
:10EBD00069676E5F626F6172645F70697463680019
:10EBE000616C69676E5F626F6172645F7961770003
:10EBF0006D61785F616E676C655F696E636C696E8D
:10EC00006174696F6E006779726F5F6C7066006D1A
:10EC10006F726F6E5F7468726573686F6C640067A3
:10EC200079726F5F636D70665F666163746F7200A7
:10EC30006779726F5F636D70666D5F666163746F35
:10EC40007200616C745F686F6C645F6465616462BC
:10EC5000616E6400616C745F686F6C645F666173A1
:10EC6000745F6368616E6765007961775F64656191
:10EC70006462616E64007468726F74746C655F6363
:10EC80006F7272656374696F6E5F76616C75650033
:10EC90007468726F74746C655F636F7272656374AD
:10ECA000696F6E5F616E676C65007961775F636F36
:10ECB0006E74726F6C5F646972656374696F6E0005
:10ECC0007961775F646972656374696F6E007472ED
:10ECD000695F756E61726D65645F736572766F00F2
:10ECE00064656661756C745F726174655F70726F84
:10ECF00066696C650072635F726174650072635F60
:10ED00006578706F007468725F6D69640074687212
:10ED10005F6578706F00726F6C6C5F7069746368A8
:10ED20005F72617465007961775F72617465007408
:10ED300070615F72617465007470615F62726561B9
:10ED40006B706F696E74006661696C736166655F94
:10ED500064656C6179006661696C736166655F6F9B
:10ED600066665F64656C6179006661696C73616693
:10ED7000655F7468726F74746C65006661696C734A
:10ED80006166655F6D696E5F757365630066616975
:10ED90006C736166655F6D61785F7573656300674D
:10EDA000696D62616C5F666C616773006163635F6C
:10EDB0006861726477617265006163635F6C70663D
:10EDC0005F666163746F720061636378795F646525
:10EDD000616462616E64006163637A5F646561644B
:10EDE00062616E64006163637A5F6C70665F637515
:10EDF000746F6666006163635F756E61726D6564F2
:10EE000063616C006163635F7472696D5F706974E4
:10EE10006368006163635F7472696D5F726F6C6CCD
:10EE2000006261726F5F7461625F73697A6500622C
:10EE300061726F5F6E6F6973655F6C7066006261AF
:10EE4000726F5F63665F76656C006261726F5F63AD
:10EE5000665F616C74006D61675F6465636C696EA9
:10EE60006174696F6E007069645F636F6E74726F56
:10EE70006C6C657200705F706974636800695F70C4
:10EE80006974636800705F726F6C6C00695F726FA9
:10EE90006C6C00705F79617700695F7961770070F1
:10EEA0005F70697463686600695F7069746368663F
:10EEB00000645F70697463686600705F726F6C6C89
:10EEC0006600695F726F6C6C6600645F726F6C6C79
:10EED0006600705F7961776600695F7961776600C7
:10EEE000645F79617766006C6576656C5F686F72E8
:10EEF000697A6F6E006C6576656C5F616E676C65D4
:10EF000000705F616C7400695F616C7400645F61C4
:10EF10006C7400705F6C6576656C00695F6C65761B
:10EF2000656C00645F6C6576656C00705F76656C1F
:10EF300000695F76656C00645F76656C0000202078
:10EF40002020202020202028282828282020202099
:10EF50002020202020202020202020202020881059
:10EF600010101010101010101010101010100404B9
:10EF700004040404040404041010101010101041C0
:10EF80004141414141010101010101010101010131
:10EF900001010101010101010110101010101042C6
:10EFA0004242424242020202020202020202020201
:10EFB00002020202020202020210101010200000DF
:10EFC0000000000000000000000000000000000041
:10EFD0000000000000000000000000000000000031
:10EFE0000000000000000000000000000000000021
:10EFF0000000000000000000000000000000000011
:10F000000000000000000000000000000000000000
:10F0100000000000000000000000000000000000F0
:10F0200000000000000000000000000000000000E0
:10F0300000000000000000000000000000000000D0
:10F040000000004B000000CB61636F73660000009E
:10F05000000000007371727466000000000FC93F69
:10F06000000F494000CB9640000FC9400053FB40C1
:10F0700000CB164100ED2F41000F494100316241A4
:10F0800000537B41003A8A4100CB9641005CA3418A
:10F0900000EDAF41007EBC41000FC94100A0D54149
:10F0A0000031E24100C2EE410053FB4100F2034255
:10F0B000003A0A420083104200CB164200141D425F
:10F0C000005C234200A5294200ED2F420036364263
:10F0D000007E3C4200C74242000F4942A2000000AD
:10F0E000F9000000830000006E0000004E000000E8
:10F0F000440000001500000029000000FC00000092
:10F100002700000057000000D1000000F5000000BB
:10F1100034000000DD000000C0000000DB00000043
:10F120006200000095000000990000003C00000013
:10F13000430000009000000041000000FE000000BD
:10F140005100000063000000AB000000DE00000082
:10F15000BB000000C500000061000000B700000017
:10F16000240000006E0000003A0000004200000091
:10F170004D000000D2000000E0000000060000008A
:10F18000490000002E000000EA0000000900000015
:10F19000D1000000920000001C000000FE000000F2
:10F1A0001D000000EB0000001C000000B10000008A
:10F1B00029000000A70000003E000000E800000059
:10F1C0008200000035000000F50000002E00000065
:10F1D000BB0000004400000084000000E9000000C3
:10F1E0009C0000007000000026000000B400000039
:10F1F0005F0000007E0000004100000039000000B8
:10F2000091000000D60000003900000083000000DB
:10F210005300000039000000F40000009C000000D2
:10F22000840000005F0000008B000000BD000000B3
:10F23000F9000000280000003B0000001F00000053
:10F24000F800000097000000FF000000DE00000052
:10F2500005000000980000000F000000EF00000013
:10F260002F000000110000008B0000005A00000079
:10F270000A0000006D0000001F0000006D0000008B
:10F28000360000007E000000CF00000027000000D4
:10F29000CB00000009000000B70000004F00000094
:10F2A000460000003F000000660000009E000000D5
:10F2B0005F000000EA0000002D0000007500000063
:10F2C00027000000BA000000C7000000EB000000AB
:10F2D000E5000000F10000007B0000003D000000A0
:10F2E0000700000039000000F70000008A0000005D
:10F2F0005200000092000000EA0000006B000000D5
:10F30000FB0000005F000000B10000001F000000D3
:10F310008D0000005D0000000800000056000000A5
:10F32000030000003000000046000000FC00000068
:10F330007B0000006B000000AB000000F00000004C
:10F34000CF000000BC000000200000009A00000078
:10F35000F4000000360000001D000000A9000000BD
:10F36000E300000091000000610000005E0000006A
:10F37000E60000001B00000008000000650000001F
:10F3800099000000850000005F00000014000000EC
:10F39000A000000068000000400000008D00000098
:10F3A000FF000000D8000000800000004D000000B9
:10F3B000730000002700000031000000060000007C
:10F3C000060000001500000056000000CA00000002
:10F3D00073000000A8000000C900000060000000E9
:10F3E000E20000007B000000C00000008C00000074
:10F3F0006B0000000400000007000000090000008E
:10F400000000C93F0000F0390000DA370000A233E5
:10F410000000842E0000502B0000C2270000D022E4
:10F420000000C41F0000C61B000044176937AC3140
:10F4300068212233B40F14336821A2333863ED3EC0
:0CF44000DA0F493F5E987B3FDA0FC93FAE
:08F44C00B891FF7F01000000F0
:10F45400000100000000803F0000000000000000E8
:10F464000000000000000000000000000100000097
:10F47400000000000000000000127A0000000000FC
:10F48400000000000102030406070809010300004C
:10F494000000803F0000803F0000803F010000002A
:10F4A400000102030401020304060708090204061A
:10F4B4000800DC05DC05DC05DC05DC05DC05DC0519
:10F4C400DC050000493F0008B5DD0008030000002A
:10F4D40000A24A0461E200083DEF000800000000B9
:10F4E4000000000000000000000000000000000018
:10F4F40000000000000000000000000048E20008D6
:10F5040000000000000000000000000000000000F7
:10F5140000000000000000000000000000000000E7
:10F5240000000000000000000000000000000000D7
:10F534000000000000000000000000008C0000201B
:04F5440001000000C2
:0400000508000000EF
:00000001FF
